:020000040800F2
:1028000080840020DD290008758E000839850008C5
:10281000198B0008F53B0008DD9800080000000057
:102820000000000000000000000000004529000832
:10283000753C00080000000089290008C58E0008CA
:10284000F7290008F7290008F7290008F7290008E8
:10285000F7290008F7290008F7290008F7290008D8
:10286000F7290008F7290008F7290008F7290008C8
:10287000F7290008F93B0008F7290008F7290008A4
:10288000F7290008F7290008F7290008F7290008A8
:10289000F7290008F7290008F7290008F729000898
:1028A000F7290008618F0008F7290008F7290008B8
:1028B000718F0008F7290008818F0008F7290008A8
:1028C000F7290008F7290008F7290008F729000868
:1028D000F7290008D5960008F7290008E5960008B2
:1028E000F7290008F7290008F7290008F729000848
:1028F000F7290008F7290008F7290008F729000838
:10290000F7290008F7290008F7290008F729000827
:10291000D9900008F7290008F7290008F7290008CE
:10292000F7290008F7290008093C0008F7290008E2
:10293000DFF80CD000F0E8FE0048004721BA00089C
:1029400080840020224B19680868B0E8F00F80F3FB
:102950000988BFF36F8F4FF0000080F311884EF0AD
:102960000D0E70470000000006480068006880F304
:10297000088862B661B6BFF34F8FBFF36F8F00DF79
:1029800000BF00BF08ED00E0EFF30980BFF36F8FD9
:102990000F4B1A6820E9F00F106008B54FF0500097
:1029A00080F31188BFF34F8FBFF36F8F0DF028FABC
:1029B0004FF0000080F31188BDE8084019680868EE
:1029C000B0E8F00F80F30988BFF36F8F704700BF46
:1029D000B4100020EFF305807047000006488047E0
:1029E00006480047FEE7FEE7FEE7FEE7FEE7FEE7F4
:1029F000FEE7FEE7FEE7FEE75F8F000831290008EB
:102A0000202A04DB203A21FA02F00021704721FA43
:102A100002F3D040C2F120029140084319467047AA
:102A2000004870478413010810B50446FFF7F8FF0B
:102A30000068005D00F0010010BDA0F141011929FE
:102A400000D82030704740EA01039B0703D009E01B
:102A500008C9121F08C0042AFAD203E011F8013B8A
:102A600000F8013B521EF9D27047D2B201E000F8E3
:102A7000012B491EFBD270470022F6E710B5134622
:102A80000A4604461946FFF7F0FF204610BD30B550
:102A900005462A460B4612F8010B13F8014B08B104
:102AA000A042F8D01CB1002802D06D1CF1E72846E6
:102AB00030BD10B5044604E00B7800F8013B03B1CB
:102AC000491C521EF8D2204610BDCAB2401E10F852
:102AD000011F8A4202D00029F9D100207047421C10
:102AE00010F8011B0029FBD1801A7047034611F82A
:102AF000012B00F8012B002AF9D11846704730B598
:102B000005460020034600E05B1C934205D2EC5CC6
:102B1000C85C201A01D1002CF6D130BD70B50F4D24
:102B200000B92868002412E00A4602E09E4203D061
:102B3000521C1378002BF9D1DAB2224305D02BB105
:102B400024B1002100F8011B04E00446401C067873
:102B5000002EE9D12860204670BD00002012002020
:102B60000FB400B58DB010A909900B9000914FF0F3
:102B7000FF300A9000200C90054806900548079009
:102B80006A4609A80F9900F045FC0DB05DF814FBEA
:102B9000313400084F3400082DE9FF5F1D464FF027
:102BA000FF3BD5E9014691465F464FF00008A96911
:102BB0007F1C01988847296A824688470028F6D1F9
:102BC000BAF1FF3F0CD024F4C064002E19DD60067A
:102BD00014D5BAF12B0F09D0BAF12D0F0ED103E0A5
:102BE000584604B0BDE8F09F44F48064A9697F1C96
:102BF00001988847761E8246002E02DDBAF1300F1A
:102C000003D0B9F1000F26D032E0A969761E44F452
:102C100000747F1C019888478246002E05DDBAF1BA
:102C2000780F06D0BAF1580F03D0B9F1000F10D0C9
:102C30001EE0B9F1000F02D0B9F1100F18D1A96947
:102C4000761E24F400747F1C019888478246102069
:102C500002E0082000E00A20814609E008FB09089C
:102C6000A969761E44F400747F1C01988847824647
:102C7000002E05DD4946504600F0B8FB0028EDDA8D
:102C8000E96901988847A00502D46FF00100A8E720
:102C9000E00725D1600613D5600502D5C8F1000014
:102CA00000E0404629680A1D2A600968220501D50E
:102CB000087015E0220701D5088011E008600FE0D8
:102CC0002868011D29600068210502D580F8008070
:102CD00006E0210702D5A0F8008001E0C0F80080DE
:102CE00038467EE770B5064606F078FE046805466D
:102CF0000A220021304600F0BBFB2C6070BDF0B40E
:102D000080EA0102D40F4200B2EB410F02D2024628
:102D1000084611464A0042D0C30DDDB2C1F3C75286
:102D2000AD1A202D35DAC1F3160141F4000204B1C9
:102D30005242C5F1200602FA06F12A411044B3EBD3
:102D4000D05F23D0C4B1012DA0EBC35009DCF0BC8F
:102D50004FF0004202EAC352DBB200F5000000F07F
:102D6000C8BB400000F1807000EBC350A0F1807040
:102D700040EAD170490009E0490841EAC071A0EB7E
:102D8000C35000F50000400800EBC350F0BC00F059
:102D9000A7BB6142012202EB4101001BF6E7F0BC38
:102DA000704781F00041AAE780F00040A7E780EA81
:102DB000010210B502F00043400022D04A001FD0AB
:102DC000010E01EB1261C0F35600C2F3560240F44B
:102DD000000042F40002A0FB022000047F3914042A
:102DE00000D0401C50EA124001D44000491EC2B23B
:102DF0000C0604EBD010401C4008802A02D003E0EF
:102E0000002010BD20F00100002900DA0020184346
:102E100010BD30B480EA010202F0004530F00042FB
:102E200021F0004013D090B1C30DD40DC2F31601B0
:102E3000C0F31600E41A41F4000140F400027D34AE
:102E4000914201D3641C00E04900002C02DA30BC3E
:102E5000002070474FF400000023914201D3891AEB
:102E6000034340084FEA4101F7D151B1914202D1E9
:102E70004FF0004105E002D24FF0010101E06FF098
:102E8000010103EBC450284430BC00F029BB2DE9FC
:102E9000FE4F804681EA0300C00F0C46009021F0EF
:102EA000004123F00045B8EB0200A94105D240469D
:102EB000214690461C460B46024623F00040104334
:102EC00047D0270DC7F30A00C3F30A510290401AF6
:102ED000019040286BDAC3F3130040F4801B009884
:102EE000924620B10023D2EB030A63EB0B0B01984F
:102EF0005946C0F14002504600F057FA06460D46CA
:102F000050465946019A00F05FFA10EB0800614103
:102F1000002487EA115284EAE7731A4340D0009AEA
:102F200062B3019A012A4FEA075215DC001B61EBDC
:102F300002014FF0004202EA0752CDE90042001CB4
:102F400041F5801132462B4600F010FB03B0BDE87E
:102F5000F08F40462146F9E7001B61EB0201001C9F
:102F600041F5801300185B412018A2F5001747EBCC
:102F7000030140EAD570B6196D4111E06D084FEAC2
:102F8000360645EAC0754FEA0752001B61EB0201A5
:102F9000001C41F5801149084FEA300000195141E9
:102FA00032462B4603B0BDE8F04F00F0D0BA00988F
:102FB000012240000023D0EB020263EBE073009893
:102FC00021464FEAE074B8EB000061EB0401E9E749
:102FD00083F000435BE781F0004158E72DE9FE4FA5
:102FE00081EA030404F0004421F0004100944FF012
:102FF000000B23F0004350EA01045ED052EA0304C0
:103000005BD0C3F30A54C1F30A552C44A4F2F33441
:103010000194A0FB0254C1F3130141F48011C3F3E6
:10302000130343F4801301FB024400FB034E840AA4
:10303000970A44EA815447EA8357A4FB076802953C
:103040008D0A05FB07854FEA932C04FB0C542705DA
:10305000029D4FEA065847EA1637B5EB08056EEBB6
:10306000070C870E920E47EA811742EA8312A7FBEC
:103070000201B6EB0B0164EB00042B0D43EA0C33A9
:103080005E1844EB1C50DA465146E7FB0201C5F3DB
:1030900013044FEA0B3343EA14534FEA0432019C02
:1030A00043EA0603A4F10C040294009CCDE900B4A9
:1030B00000F05CFA03B0BDE8F08F00200146F9E7AC
:1030C0002DE9F04D81EA030404F0004B21F00045A6
:1030D00014464FF0000A23F0004150EA050220D0C8
:1030E00054EA01021DD0C5F30A570246C5F3130383
:1030F000C1F31300C1F30A5640F4801543F4801362
:10310000A7EB0608101BD64608F2FD3873EB050046
:1031100002D308F1010801E092185B41B8F1000FF9
:1031200003DA00200146BDE8F08D00204FF4801145
:10313000064684460EE0171B73EB050705D3121BEA
:1031400063EB050306434CEA010C49084FEA3000E3
:1031500092185B4150EA0107EDD152EA030012D008
:1031600082EA040083EA0501084305D0101BAB4145
:1031700006D20122002306E000224FF0004302E0C5
:103180006FF0010253101AEB06004CEB085110EBE4
:103190000A0041EB0B01BDE8F04D00F0D8B9C10FBA
:1031A00080EAE0700844CA079623002100F0A1B924
:1031B00096230022114600F09CB90EB5C10F80EA9B
:1031C000E0700844CA07002140F233438DE80E0046
:1031D0000A460B4600F0CAF903B000BD0EB540F236
:1031E000334102910021CDE900110A460B4600F05F
:1031F000BDF903B000BD20F00040C10DC0F31600C2
:1032000040F400007F2901DA00207047962903DC92
:10321000C1F19601C840704796398840704770B533
:10322000C1F30A5201F000450024C1F3130140F23A
:10323000FF3341F480119A4201DA002070BD40F260
:1032400033439A42A2F2334203DC5242FFF7D8FBE7
:1032500000E090402C43F1D0404270BD00F00042AD
:1032600030F000400AD0C10D01F56071C0F31600C6
:1032700042EA0151C208400711437047002001464D
:103280007047000030B5041E71F1000404DB4FF0FC
:103290000044404264EB0101141E73F1000405DB9D
:1032A0001C464FF00043524263EB04038B4208BFBD
:1032B000824230BD30B5041E71F1000404DB4FF0D2
:1032C0000044404264EB0101141E73F1000405DB6D
:1032D0001C464FF00043524263EB0403994208BF7F
:1032E000904230BD01F0004330B421F0004150EA7B
:1032F000010206D00A0DA2F56072C1F31301002A83
:1033000002DC30BC00207047440F44EAC104C10015
:10331000E01830BC00EBC25000F0E2B830B50B460C
:10332000014600202022012409E021FA02F59D42F5
:1033300005D303FA02F5491B04FA02F52844151EC9
:10334000A2F10102F1DC30BD2DE9F05F054600205D
:1033500092469B4688460646814640241BE0284606
:10336000414647462246FFF74BFB53465A46C01A92
:10337000914110D311461846224600F016F82D1A36
:1033800067EB01084F4622460120002100F00DF8AE
:1033900017EB00094E41201EA4F10104DFDC484672
:1033A00031462A464346BDE8F09F202A04DB203AF6
:1033B00000FA02F1002070479140C2F1200320FA88
:1033C00003F3194390407047202A06DBCB17203ABD
:1033D00041FA02F043EAE07306E041FA02F3D0401A
:1033E000C2F1200291400843194670473A2800D2A2
:1033F000303820F02002412A01D3A2F13700884260
:1034000001D34FF0FF307047026811441378016018
:1034100018467047D1600449516104491162002186
:103420001161114600F082B909340008292A000808
:10343000426842B1016811F8013B23B1521EC0E954
:103440000012184670470121C160881E704742680B
:103450005AB1C368016843B983688B4205D0491EDD
:10346000521CC0E90012002070474FF0FF30704737
:103470002DE9F04791460F4680460446002614F891
:10348000015B2DB1FFF7CCFA0068405DC007F6D1B3
:103490002B2D02D02D2D18D0641E4A4639462046C9
:1034A00000F0DAFA27B13968A14201D1C7F80080EB
:1034B00071054FF002040BD54042002803DD06F0F1
:1034C0008DFA0460A007BDE8F08746F48066E4E763
:1034D0000028F8DA06F082FA04606FF00040F2E7A4
:1034E0000029A8BF7047401C490008BF20F0010018
:1034F000704710B4B0FA80FC00FA0CF050EA0104F6
:1035000004BF10BC704749B1CCF1200421FA04F487
:1035100011FA0CF118BF012121430843A3EB0C0160
:10352000CB1D4FEA00614FEA102042BF002010BCC3
:10353000704700EBC35010440029A4BF10BC704773
:10354000401C490008BF20F0010010BC704710B5B6
:10355000141E73F1000408DA401C41F100019218B6
:103560005B411A4301D120F0010010BD2DE9F04D5F
:1035700092469B4611B1B1FA81F202E0B0FA80F2B4
:1035800020329046FFF711FF04460F4640EA0A003A
:1035900041EA0B0153465A46084313D0114653EAF9
:1035A000010019D0C8F140025046FFF729FA05463C
:1035B0000E46504659464246FFF7F7FE084305D0EF
:1035C000012004E020463946BDE8F08D0020054387
:1035D00046EAE0762C4337430A986305E40AA0EBF9
:1035E00008000022FD0A44EA47540A3002D50020B0
:1035F0000146E9E7010510196941DDE908450019AF
:103600006941BDE8F04DA2E770B521F000430343E6
:103610000CD0C1F30A550024D5EB040564EB040378
:10362000D617AD1AB34102DB0020014670BD201849
:1036300041EB025170BD2DE9F04D00231A461B1AD3
:103640008A4103DB00200146BDE8F08DC1F30A5238
:10365000C1F3130141F480154FF0000BD10702D1E3
:1036600000186D41521E0027044640F2FF113846F3
:1036700001EB620A3E468046024600204FF480116C
:10368000FFF7BEF9C2197141BB1846EB0100B4EB5C
:10369000030C75EB000C04D3E41A65EB0005174628
:1036A0000E46241908F101006D4180463428E3DDFF
:1036B000F91946EB0600091BA84103D24FF0FF326F
:1036C000134601E0002213461BEB070046EB0A51AC
:1036D000BDE8F04DFFF73BBFC1F30A52C1F3130140
:1036E00040F2FF3341F480119A4202DA0020014691
:1036F000704740F233439A42A2F2334202DC524214
:10370000FFF77EB9FFF751BE064C074D06E0E068B3
:1037100040F0010394E8070098471034AC42F6D318
:10372000FFF70AF99C150108BC1501082DE9F34FB4
:103730008BB04FF0000801F10C000C464FF0010B6C
:1037400046460DF1080A01906269012101989047EF
:10375000051E2DD0252D2CD0216A8847C0B1626965
:10376000012101989047216A88470028F7D1411E1E
:1037700062690198904700E0761CA1690B98884720
:10378000216A88470028F7D1E1690B988847DBE771
:10379000A1690B9888470746A84201D1761CD3E758
:1037A000E1690B9888477F1C02D1B8F1000F6FD0F8
:1037B00046E1002762693D463946019890472A282C
:1037C00004D162690121019890470125DFF88492B4
:1037D0006269012101989047A0F130010A290AD2BB
:1037E0004F45E5DC07EB870100EB4107303FDFD4B5
:1037F00045F01005ECE7E90601D46FF000476C28AE
:103800000AD04C2814D0682815D06A280DD0742806
:103810001CD07A281AD01DE06269012101989047D6
:103820006C2802D045F0040514E045F002050DE0D7
:1038300045F020050AE06269012101989047682857
:1038400002D045F0080505E045F4006562690121F4
:1038500001989047C4E9015765283DD019DC5828E4
:103860007AD00CDC452837D004DC252826D0412826
:1038700031D131E046282FD047282CD12CE05B28CD
:1038800077D0612828D063287CD0642823D15AE0DF
:10389000D0E06F2848D008DC66281DD067281BD0F0
:1038A000692821D06E2816D127E0702845D07328CA
:1038B00068D0752847D078280DD14DE0A1690B98C4
:1038C0008847054625283FF469AFE1690B9888478A
:1038D0006D1C3FF46AAFB3E023466A466FF0010007
:1038E0000B99AFF300809EE045F040006060A807B0
:1038F00023464FF0000236D43EE0E8077FF447AF9E
:103900002068011D21600068290501D506701BE7AC
:10391000290701D5068017E7A90703D5F117C0E9E4
:10392000006111E706600FE745F040006060A807FE
:1039300023464FF0080216D41EE040F60E0125EA99
:103940000100606016E045F040006060A807234673
:103950004FF00A0207D40FE045F040006060A8076E
:1039600008D5234610226FF001000B99AFF30080B9
:1039700059E007E0234610226FF001000B99FFF792
:103980000BF950E04FF000094F464B46632802D038
:103990005B2806D040E0E80601D40120A0600127A2
:1039A0003AE062690121019890475E2805D14FF005
:1039B00001096269494601989047216939B9002196
:1039C0000A46534643F82120491C0829FADBB0B3C4
:1039D000216969B9C11700EBD16253110AEB830168
:1039E00022F01F02821A01200B68904003430B60F3
:1039F00062690121019890475D28E8D1B9F1000F73
:103A000009D00020514651F82020D24341F820200F
:103A1000401C0828F7DB02AB224600976FF001003C
:103A20000B99AFF3008000280CDA401C08D1BBF1E1
:103A3000000F05D04FF0FF300DB0BDE8F08FFFE76D
:103A40004046F9E7E90701D108F1010806444FF0C3
:103A5000000B79E6CCCCCC0C2DE9F05F82460078E7
:103A6000002715468B460AF10104B946302801D0DB
:103A70009DB113E014F8010B0127782803D05828D2
:103A800001D045B10AE00DB1102D07D10027102556
:103A900014F8010B02E0082500E00A250026B046D4
:103AA0000EE005FB080005FB06F1012701EB1046BF
:103AB0001FFA80F8B6F5803F00D3B94614F8010B21
:103AC0002946FFF793FC0028EBDABBF1000F05D085
:103AD0000FB1641E00E05446CBF80040B9F1000F6E
:103AE00006D005F07BFF02210160C81EBDE8F09FF3
:103AF00048EA0640FAE770B58C1810F8015B15F03B
:103B0000070301D110F8013B2A1106D110F8012B4F
:103B100003E010F8016B01F8016B5B1EF9D12B0774
:103B200005D40023521E0DD401F8013BFAE710F82A
:103B3000013BCB1A921C03E013F8015B01F8015B17
:103B4000521EF9D5A142D8D3002070BD70B50446ED
:103B5000002540F6B8322149214804F07BFC20487A
:103B60000068C06840F010001D490968C86026E080
:103B7000012008F00DF92046FEF7B1FF0646334656
:103B8000224640F6B83115480BF08AFB00B10125FA
:103B9000052314A240F6B83110480BF081FB00B1A8
:103BA000022512480088642805DA10480088401C65
:103BB0000E49088003E000200C4908800325002DF1
:103BC000D6D000200A49087005480068C06820F077
:103BD000100003490968C860284670BDA021002074
:103BE000582D00204552524F520000006E10002008
:103BF000A210002000BFFEE710B5024802F098FCBA
:103C000010BD0000742E002010B5024802F090FC98
:103C100010BD0000302E002030B590F84050012437
:103C2000AC40C56B6C60046863604468102C04D1C0
:103C30000468A2600468E16003E00468A1600468AD
:103C4000E26030BD01B5084A5068084A1268084B66
:103C5000B2FBF3F2009B02FB03F100BF024A526881
:103C6000121A8A42FAD308BD001000E0B0100020FA
:103C700040420F007047000070B504460D46002614
:103C800040F6B8321549164804F0E4FB14480068C1
:103C9000C06840F0100012490968C86002E00120C5
:103CA00008F076F80F4800780028F8D00C48006833
:103CB000C06820F010000A490968C860002009495E
:103CC000087029462046FEF7E2FE064640F6B83167
:103CD0002046FEF7D1FE304670BD0000A021002036
:103CE000582D0020A210002070B504460025204663
:103CF00000F0B6FE0546AAB24FF47A732146024898
:103D000004F0C0FB70BD0000582D002070B59AB0C3
:103D10000026642101A8FEF7AFFE00240025A74875
:103D200000780C2874D2DFE800F0061F29425B7689
:103D30009DB6CFF0EEEDA2A0FFF7D6FFA2A1A4485A
:103D4000FFF79AFF05461DB1A2A005F0DBFD04E0D8
:103D5000601CC4B2A5A005F0D5FD1CB9012097498F
:103D6000087000E0002426E300F0AAFE04461CB917
:103D700002209249087000E000241CE3A2A0FFF793
:103D8000B3FF91A19248FFF777FF05461DB1A0A0B0
:103D900005F0B8FD04E0601CC4B2A3A005F0B2FDBC
:103DA0001CB903208549087000E0002403E3A6A0A5
:103DB000FFF79AFFA7A18648FFF75EFF05461DB1F2
:103DC000AAA005F09FFD04E0601CC4B2ACA005F001
:103DD00099FD1CB904207949087000E00024EAE24A
:103DE000ACA0FFF781FF01F0D1FB794800F040FE65
:103DF00006461EB1AAA005F085FD04E0601CC4B211
:103E0000ABA005F07FFD24B905206C49087001E0E6
:103E1000D0E20024CFE2ABA0FFF766FF01F0B6FBD3
:103E2000ABA16B48FEF733FE20B9AAA16848FEF7A4
:103E30002EFE18B1A8A005F065FD04E0601CC4B218
:103E4000B3A005F05FFD40F6B8316148FEF714FEFF
:103E50000020BC4908701CB906205849087000E0D1
:103E60000024A8E2B8A0FFF73FFF57A15848FFF78A
:103E700003FF05461DB1B8A005F044FD04E0601C39
:103E8000C4B2BFA005F03EFD1CB907204B49087025
:103E900000E000248FE2C3A0FFF726FF4AA14C48B0
:103EA000FFF7EAFE05461DB1C2A005F02BFD04E0B8
:103EB000601CC4B2C8A005F025FD1CB908203F490C
:103EC000087000E0002476E21E22CBA101A805F0D4
:103ED00041FD01A8FFF708FF3BA13D48FFF7CCFEDD
:103EE00005461DB1CBA005F00DFD04E0601CC4B279
:103EF000D1A005F007FD1CB909203049087000E089
:103F0000002458E23AE019E0FFE7D3A0FFF7ECFE07
:103F10002DA12F48FFF7B0FE05461DB1D6A005F034
:103F2000F1FC04E0601CC4B2DDA005F0EBFC1CB9A0
:103F30000A202249087000E000243CE2E148838A1C
:103F40000246E1A101A805F005FD01A8FFF7CCFE9E
:103F5000E3A0FFF7FBFD0646012E03D1E4A005F028
:103F6000D1FC04E0601CC4B2EDA005F0CBFC1CB990
:103F70000B201249087000E000241CE2D1483E30BA
:103F8000A0F11403A0F12802F0A1009001A805F00F
:103F9000E1FC01A8FFF7A8FE0BA10D48FFF76CFE9E
:103FA0000546F0A10A48FFF767FE05461DB1F1A0DE
:103FB00005F0A8FCF7E1601CC4B2F1E16B10002031
:103FC00041540D0A000000004F4B0D0A0000000094
:103FD000A02100204D6F64756C6520737461747549
:103FE00073206E6F726D616C0D0A00004D6F647509
:103FF0006C65207374617475732061626E6F726D8D
:10400000616C0D0A00000000415445300D0A0000AB
:1040100043616E63656C206D6F64756C65206563CC
:10402000686F0D0A000000004661696C65642074C9
:104030006F2063616E63656C206D6F64756C6520C5
:104040006563686F0D0A000041542B4350494E3F91
:104050000D0A00002B4350494E3A20524541445925
:104060000D0A0D0A4F4B0D0A0000000053494D2068
:1040700063617264206E6F726D616C0D0A000000E6
:1040800053494D20636172642061626E6F726D618D
:104090006C0D0A0041542B4353510D0A00000000DF
:1040A0007369676E616C206E6F726D616C0D0A00D2
:1040B0007369676E616C2061626E6F726D616C0D09
:1040C0000A00000041542B435245473F0D0A0000AF
:1040D0003100000035000000546865206D6F647584
:1040E0006C65207375636365737366756C6C79209A
:1040F00072656769737465726564206F6E20746899
:10410000652047534D206E6574776F726B0D0A0002
:10411000546865206D6F64756C65206661696C65B7
:104120006420746F207265676973746572206F6EA6
:10413000207468652047534D206E6574776F726BED
:104140000D0A0000A210002041542B514944454162
:1041500043543D310D0A0000537563636573736604
:10416000756C6C792064697361626C6564206D6F35
:1041700062696C65207363656E650D0A000000005E
:104180004661696C656420746F2064697361626C58
:1041900065206D6F62696C65207363656E650D0ADD
:1041A0000000000041542B51494143543D310D0A58
:1041B000000000005375636365737366756C6C79FA
:1041C00020656E61626C6564206D6F62696C65204C
:1041D0007363656E650D0A004661696C65642074E1
:1041E0006F20656E61626C65206D6F62696C652021
:1041F0007363656E650D0A0041542B514D5443465F
:10420000473D22716D7470696E67222C302C2564D5
:104210000D0A00004D515454206865617274626546
:104220006174207365742073756363657373667559
:104230006C6C790D0A0000004661696C656420743D
:104240006F20736574204D515454206865617274F9
:10425000626561740D0A000041542B514D54434670
:10426000473D22726563762F6D6F6465222C302C7A
:10427000302C310D0A0000004461746120726563C6
:10428000656976696E67206D6F646520736574205B
:104290007375636365737366756C6C792E0D0A00B4
:1042A0004661696C656420746F2073657420646175
:1042B000746120726563656976696E67206D6F64ED
:1042C000650D0A001010002041542B514D544F50E1
:1042D000454E3D302C222573222C25640D0A00000A
:1042E0002B514D544F50454E3A20302C3000000099
:1042F0005375636365737366756C6C79206F706555
:104300006E65642061206E6574776F726B20666FD6
:104310007220746865206D6F64756C650D0A00000D
:104320004661696C656420746F206F70656E2061F2
:10433000206E6574776F726B20666F72207468658B
:10434000206D6F64756C650D0A00000041542B519F
:104350004D54434F4E4E3D302C25732C25732C2548
:10436000730D0A002B514D54434F4E4E3A20302CC2
:10437000302C30005375636365737366756C6C79AC
:1043800020636F6E6E656374656420746F2074685B
:1043900065204D515454207365727665720D0A0084
:1043A00006A005F0AFFA1CB90C200E49087000E019
:1043B000002400E000BF00BF1AB070BD4661696C08
:1043C000656420746F20636F6E6E65637420746F14
:1043D00020746865204D515454207365727665725F
:1043E0000D0A00006B10002070B59AB000243C4DFF
:1043F000642101A8FEF740FB00263A480078052812
:1044000069D2DFE800F003204F565F0005F1420358
:1044100035A2642101A805F085FA01A8FFF764FC24
:1044200036A0FFF793FB0446012C04D1002437A0EB
:1044300005F068FA02E03EA005F064FA14B9012024
:104440002849087048E005F1560342A2642101A8FA
:1044500005F068FA01A8FFF747FC43A0FFF776FBD9
:104460000446012C16D1002443A005F04BFA05F1B7
:104470006C024BA14F48FEF773FB012804D14EA0FC
:10448000E96E05F03FFA08E0601CC4B250A005F0E8
:1044900039FA02E056A005F035FA14B902201149A4
:1044A000087019E05C485D49086003200D490870F8
:1044B00012E005F053F90646012E02D10420094905
:1044C000087009E001205649087005F009FA052036
:1044D0000449087000E000BF00BF1AB070BD0000C2
:1044E000941100201C12002041542B51465450437B
:1044F00057443D222573220D0A0000002B514654DB
:10450000504357443A20302C3000000046494E4971
:1045100053482120536574207468652066696C6572
:10452000206469726563746F72792E0D0A00000051
:104530004552524F5221205365742074686520669D
:10454000696C65206469726563746F72792E0D0AF7
:104550000000000041542B5146545053495A453DE8
:10456000222573220D0A00002B5146545053495AFC
:10457000453A20302C00000046494E49534821203E
:1045800047657420746865206C656E677468206F79
:1045900066207468652066696C652E0D0A0000004F
:1045A0000D0A2B5146545053495A453A20252A6446
:1045B0002C257500A02100205468652066696C6573
:1045C00073697A652069733A2025750A0000000036
:1045D0004661696C656420746F2070617273652038
:1045E0007468652066696C6573697A652E0A0000D7
:1045F0004552524F52212047657420746865206CE3
:10460000656E677468206F66207468652066696CE3
:10461000652E0D0A0000000000100408141200208E
:104620007811002010B5174C94F8520010B194F88E
:10463000530000B910BD1448007820B101280CD0F7
:1046400002281BD113E000F025F810480078032859
:1046500002D101200C49087011E0FFF7C5FE0C489B
:104660000078052802D102200749087007E04FF4BE
:104670007A7007F08DFB02F0CDFD00E000BF00BFB7
:1046800000BFD7E7101000201D1200200C120020E0
:104690001C12002070B59AB000260024644D6421DD
:1046A00001A8FEF7E9F995F8280085F82800614887
:1046B000007820B101282BD0022871D194E05EA0AF
:1046C000FFF712FB5FA16148FFF7D6FA06461EB15D
:1046D0005FA005F017F904E0601CC4B262A005F009
:1046E00011F968A0FFF700FB56A15848FFF7C4FA7C
:1046F00006461EB16AA005F005F904E0601CC4B2CC
:104700006DA005F0FFF814B901204A4908708CE04B
:1047100005F114002B4670A26421009001A805F059
:1047200001F901A8FFF7E0FA46A14848FFF7A4FA0B
:1047300006461EB171A005F0E5F804E0601CC4B2A5
:1047400078A005F0DFF895F828307FA2642101A851
:1047500005F0E8F801A8FFF7C7FA3AA13B48FFF7D0
:104760008BFA06461EB165A005F0CCF804E0601C8B
:10477000C4B26CA005F0C6F895F8293079A264217E
:1047800001A805F0CFF801A8FFF7AEFA2DA12F4838
:10479000FFF772FA064626B179A005F0B3F805E0F6
:1047A00042E0601CC4B280A005F0ACF895F82A3055
:1047B00087A2642101A805F0B5F801A8FFF794FAD3
:1047C00020A12248FFF758FA06461EB14BA005F07B
:1047D00099F804E0601CC4B252A005F093F814B933
:1047E00002201449087020E0B5F8400005F12B03C1
:1047F0007FA26421009001A805F094F801A8FFF7BA
:1048000073FA81A0FFF7A2F90446012C04D1002419
:1048100081A005F077F802E088A005F073F814B9DC
:1048200003200449087000E000BF00BF1AB070BD4B
:10483000941100200C12002041542B514941435443
:104840003F0D0A004F4B0D0A00000000A021002080
:1048500050445020436F6E746578742053746174B3
:104860007573204F4B0D0A0050445020436F6E74F7
:1048700065787420537461747573206572726F72F9
:104880000D0A000041542B514654504346473D22E7
:10489000636F6E746578746964222C310D0A0000B0
:1048A0005365742050445020636F6E746578742093
:1048B000746F20312E0D0A004552524F5221205361
:1048C00065742050445020636F6E74657874207452
:1048D0006F20312E0D0A000041542B514654504395
:1048E00046473D226163636F756E74222C222573E7
:1048F000222C222573220D0A0000000046494E4951
:104900005348212053657420757365726E616D651F
:1049100020616E642070617373776F72642E0D0A6C
:10492000000000004552524F5221205365742075FB
:104930007365726E616D6520616E64207061737362
:10494000776F72642E0D0A0041542B514654504328
:1049500046473D2266696C6574797065222C256432
:104960000D0A000041542B514654504346473D2206
:104970007472616E736D6F6465222C25640D0A007C
:1049800046494E495348212053657420746F207066
:10499000617373697665207472616E7366657220E7
:1049A0006D6F64652E0D0A004552524F52212053FF
:1049B000657420746F2070617373697665207472FA
:1049C000616E73666572206D6F64652E0D0A00005E
:1049D00041542B514654504346473D2272737074E4
:1049E000696D656F7574222C25640D0A0000000046
:1049F00041542B514654504F50454E3D2225732271
:104A00002C25640D0A0000002B514654504F504590
:104A10004E3A20302C30000046494E495348212060
:104A20004C6F6720696E20746F207468652046544F
:104A300050207365727665722E0D0A004552524FF2
:104A40005221204C6F6720696E20746F2074686556
:104A500020465450207365727665722E0D0A000050
:104A60000146002000E0401C0A5C002AFBD1704790
:104A700070B5064610A13046FEF750F8044616E021
:104A80002046FEF72FF905460BA10020FEF746F859
:104A9000044640F6B8313046FDF7EEFF00200749E6
:104AA00008701F2D01DA012070BD0020FCE7002CEA
:104AB000E6D10020F8E700003A2C0000A01000200A
:104AC0002DE9FF4100260024002723A0FFF70CF961
:104AD00000F05CFD23A12548FDF7D9FF06461EB175
:104AE00023A004F00FFF06E025A004F00BFF012037
:104AF00004B0BDE8F081002511E0FDF791FF0068EA
:104B00002449495D405C202808D12248405D0DF8C9
:104B10000400641C0F2C01DB012705E06D1C1D48FF
:104B2000FDF7DDFFA842E8D800BF00200DF8040023
:104B30006FB16846FDF7D3FF05462A466946164819
:104B4000FDF781FF694615A004F0DCFE02E017A026
:104B500004F0D8FE0020CBE741542B43494D490DCA
:104B60000A0000004F4B0D0A00000000A0210020A9
:104B7000494D5349206973206765740D0A00000090
:104B8000494D5349206973206E6F74206765740D19
:104B90000A000000D820002080120020494D53490F
:104BA0002069733A2025730A000000004572726F75
:104BB000723A20556E61626C6520746F206578745E
:104BC0007261637420746865206E756D6265720A27
:104BD0000000000070B5002400256C48007808280B
:104BE00078D2DFE800F038516A849DB6041F68A0CF
:104BF000FFF77AF869A16B48FFF73EF805461DB14B
:104C000069A004F07FFE04E0601CC4B26DA004F053
:104C100079FE1CB907205D49087002E007205B4956
:104C20000870B0E071A0FFF75FF85CA15D48FFF786
:104C300023F805461DB170A004F064FE04E0601C7A
:104C4000C4B274A004F05EFE1CB908204F4908707D
:104C500000E0002497E078A0FFF746F84FA1514804
:104C6000FFF70AF805461DB17CA004F04BFE04E0F6
:104C7000601CC4B286A004F045FE1CB90120434963
:104C8000087000E000247EE08DA0FFF72DF843A11E
:104C90004448FEF7F1FF05461DB190A004F032FE36
:104CA00004E0601CC4B29AA004F02CFE1CB90220DF
:104CB0003649087000E0002465E0A5A0FFF714F86D
:104CC00036A13848FEF7D8FF054625B1A8A004F064
:104CD00019FE05E056E0601CC4B2B54804F012FEAF
:104CE0001CB903202949087000E000244BE0B1A062
:104CF000FEF7FAFF29A12B48FEF7BEFF05461DB1BE
:104D0000B34804F0FFFD04E0601CC4B2B14804F0F5
:104D1000F9FD1CB904201D49087000E0002432E0B0
:104D2000ADA0FEF7E1FF1DA11E48FEF7A5FF054659
:104D30001DB1B0A004F0E6FD04E0601CC4B2B4A054
:104D400004F0E0FD1CB905201049087000E00024C3
:104D500019E0B8A0FEF7C8FF10A11248FEF78CFFBB
:104D600005461DB1BAA004F0CDFD04E0601CC4B23C
:104D7000C1A004F0C7FD1CB906200449087000E07A
:104D8000002400E000BF00BF70BD00006C100020D8
:104D900041542B514750533D300D0A004F4B0D0AE3
:104DA00000000000A02100205475726E206F66661E
:104DB0002074686520474E5353206D6F64756C6591
:104DC0000D0A00004661696C656420746F2074757B
:104DD000726E206F66662074686520474E535320BC
:104DE0006D6F64756C650D0A0000000041542B5115
:104DF0004750533D310D0A005475726E206F6E207E
:104E000074686520474E5353206D6F64756C650D53
:104E10000A0000004661696C656420746F20747537
:104E2000726E206F6E2074686520474E5353206D5C
:104E30006F64756C650D0A0041542B514750534304
:104E400046473D226F7574706F7274222C22756113
:104E500072746465627567220D0A00004F75747084
:104E6000757474696E67204E4D45412053656E74AC
:104E7000656E636573207669612053657269616C44
:104E800020446562756767696E670D0A000000005F
:104E9000546865204E4D45412073656E74656E63A0
:104EA00065206F7574707574206973207365742044
:104EB000696E636F72726563746C790D0A0000002D
:104EC00041542B514750534346473D226E6D656117
:104ED000737263222C310D0A00000000456E61627E
:104EE0006C696E67204E4D45412073656E74656E2A
:104EF00063652072657472696576616C207669619C
:104F00002041542B51475053474E4D45410D0A0007
:104F10004661696C656420746F20656E61626C65C2
:104F20002072657472696576696E67204E4D4541E1
:104F30002073656E74656E636573207669612041C8
:104F4000542B51475053474E4D45410D0A00000028
:104F500041542B514750534346473D226770736E6F
:104F60006D656174797065222C36330D0A0000007E
:104F7000436F6E6669677572696E67207468652035
:104F80006F75747075742074797065206F66204E2B
:104F90004D45412073656E74656E63657320746F53
:104FA00020616C6C20666F726D6174730D0A000075
:104FB0002814010841542B514750534346473D2282
:104FC000676E7373636F6E666967222C310D0A001A
:104FD000C41401087014010841542B514750534325
:104FE00046473D226175746F677073222C300D0A3D
:104FF0000000000044697361626C6520474E5353A2
:10500000206175746F2D73746172740D0A00000055
:105010004661696C656420746F2064697361626CB9
:105020006520474E5353206175746F2D7374617200
:10503000740D0A0041542B514750534346473D22BB
:105040006170666C617368222C300D0A00000000EC
:1050500044697361626C652041502D466C617368D0
:1050600020717569636B2073746172742066756E4C
:105070006374696F6E0D0A004661696C6564207423
:105080006F2064697361626C652041502D466C61CC
:10509000736820717569636B207374617274206624
:1050A000756E6374696F6E0D0A000000F0B50446FA
:1050B000DDE90556881E011E01DC0C31641E6420EA
:1050C000B4FBF0F0C0EB94004FF4C877B4FBF7F7F3
:1050D000074440F26F1048434FF00C0CB0FBFCF05B
:1050E0003844871840F26D1000FB0470074FC01B56
:1050F00000EB400003EBC000C0EB001005EB8000AC
:10510000C0EB001006EB8000F0BD00008BFA0A0037
:1051100070B505460C46002616A1284605F0EEFFA0
:1051200004461CB916A004F0EDFB0EE01CA061695A
:1051300004F0E8FB6069012804D11DA004F0E2FB43
:10514000012602E027A004F0DDFB012E10D131A1E1
:10515000284605F0D3FF04461CB931A004F0D2FB69
:1051600006E037A0216904F0CDFB206907F046F97D
:1051700070BD0000726573756C74436F64650000E8
:105180004669656C642022726573756C74436F6444
:105190006522206E6F7420666F756E640A000000D1
:1051A000726573756C74436F64653A2025640A00F8
:1051B0005468652075706C6F6164206F6620737928
:1051C0006E6368726F6E697A6564206461746120D1
:1051D000776173207375636365737366756C2E0AEC
:1051E000000000005468652075706C6F6164206F6A
:1051F000662073796E6368726F6E697A6564206485
:1052000061746120686173206661696C65642E0A4F
:105210000000000073657276657254696D65000068
:105220004669656C64202273657276657254696D97
:105230006522206E6F7420666F756E640A00000030
:1052400073657276657254696D653A2025730A003C
:105250002DE9F04399B004460D4616466421684690
:10526000FDF70AFC4FF000080FF28C0900272348D5
:10527000007810B1012838D120E03346224620A121
:10528000684604F067FB6846FEF72EFD4946244851
:10529000FEF7F2FC8046B8F1000F08D04FF000088E
:1052A00020A004F02FFB01201449087005E024A081
:1052B00004F028FB00201149087000BF2846FEF7C3
:1052C00013FD25A0FEF742FC0746012F06D1002062
:1052D0000A49087025A004F015FB05E02EA004F093
:1052E00011FB00200549087000E000BF00BF3846F0
:1052F00019B0BDE8F08300003E00000070100020EF
:1053000041542B514D5450554245583D302C302C72
:10531000302C302C222573222C25640D0A0000002D
:10532000A021002054686520746F70696320686153
:1053300073206265656E206C696E6B65640D0A0092
:1053400054686520746F706963206C696E6B2066A9
:1053500061696C65640D0A002B514D5450554245EE
:10536000583A20302C302C30000000005468652062
:105370006D65737361676520686173206265656E32
:10538000207375636365737366756C6C7920706FD9
:10539000737465640D0A00004D6573736167652061
:1053A0007075626C69636174696F6E206661696CA7
:1053B00065640D0A000000003EB5002439A0FEF728
:1053C00093FC00F0E3F83DA13E48FDF760FB044686
:1053D0001CB13DA004F096FA03E047A004F092FA55
:1053E0003EBD38494EA004F08DFA3649534803F0CB
:1053F000AFFB534A082151487A300AF013F850485D
:1054000080794F4949794E4A1279CDE900210290BD
:105410004B48C378827801884AA004F073FA484860
:10542000807947494979464DCDE900102B79EA78D2
:10543000A9782888FFF73AFE4949C8600020494901
:10544000087040F6B8311F48FDF716FB3B4890F84E
:105450008A0000903948D0F8863090F88520D0F83E
:10546000811041A004F04EFA4FF0FF314648006829
:1054700006F0ECFCA0B93148D0F88100384948600A
:105480002E4890F8850088702C48D0F886008860F7
:105490002A4890F88A00C8703B48006806F07CFDF6
:1054A00000BF9DE741542B51475053474E4D454156
:1054B0003D22524D43220D0A000000004F4B0D0AC1
:1054C00000000000A02100204C6F636174696F6EC2
:1054D00020696E666F726D6174696F6E20726563AC
:1054E0006569766564207375636365737366756C4F
:1054F0006C790D0A000000004C6F636174696F6E77
:1055000020696E666F726D6174696F6E207265637B
:10551000657074696F6E206661696C65640D0A0060
:105520004C6F636174696F6E20696E666F726D6136
:1055300074696F6E3A25730D0A0000001E13002077
:105540006410002074696D65722D25642F25642F09
:1055500025642025643A25643A25640D0A0000007C
:1055600034120020A01000206C61746974756465A9
:105570003A256425642D2D6C6F6E676974756465BA
:105580003A256425640D0A009410002010B540F6F9
:10559000B8320A490A4802F05DFF09480068C0684D
:1055A00040F0100006490968C86002E0012006F0DA
:1055B000EFFB044800780028F8D010BDA02100209F
:1055C000582D0020A21000202DE9F04100250024D4
:1055D00000267B212B48FDF778FA07462FB92AA031
:1055E00004F090F90020BDE8F081384605F0A6FDF2
:1055F00005463DB92AA004F085F9284605F040FD8E
:105600000020F0E72DA1284605F078FD04461CB9DE
:105610002DA004F077F905E032A0616904F072F979
:10562000A08A86B2CA2E15D004DC662E08D06A2E57
:1056300021D10AE0A6F25A2088B103281BD114E038
:105640002146284607F094F816E021462846FFF741
:105650005FFD11E02146284600F054F80CE0264A90
:105660002146284600F0B2F806E0244A244928469C
:1056700006F080FF00E000BF00BF284605F000FDF7
:1056800030B2B0E7A02100204A534F4E206461742D
:1056900061206E6F7420666F756E640A00000000F2
:1056A0004661696C656420746F2070617273652057
:1056B0004A534F4E20646174610A0000636F6E7438
:1056C000726F6C436F6465004669656C6420226488
:1056D0006576496422206E6F7420666F756E640A69
:1056E00000000000636F6E74726F6C436F64653A04
:1056F0002025640A0000000094110020081A0020F0
:10570000C813002070B505460C460CA1284605F0CC
:10571000F5FC04461CB90CA004F0F4F80DE012A04E
:10572000616904F0EFF86069012803D112A004F068
:10573000E9F802E01AA004F0E5F870BD726573752F
:105740006C74436F646500004669656C6420227266
:105750006573756C74436F646522206E6F74206688
:105760006F756E640A000000726573756C74436F28
:1057700064653A2025640A0055706C6F6164656445
:10578000207265616C2D74696D652064617461209F
:105790007375636365737366756C6C790A000000DA
:1057A0005468652075706C6F6164206F6620726547
:1057B000616C2D74696D652064617461206861732A
:1057C000206661696C65640A000000002DE9F04103
:1057D00006460C46174614A1304605F08FFC0546D8
:1057E00025B914A004F08EF8BDE8F08119A128466F
:1057F00005F084FC04461CB919A004F083F810E0FD
:105800001EA0616904F07EF86069012806D11F4975
:1058100081F853001EA004F075F802E020A004F007
:1058200071F800BFE0E70000706172616D4C697350
:10583000740000004661696C656420746F207061BB
:1058400072736520706172616D4C6973742064615C
:1058500074610A0066756E6374696F6E0000000003
:105860004669656C64202275706461746522206EDF
:105870006F7420666F756E640A00000066756E6353
:1058800074696F6E3A2025640A0000001010002031
:1058900075706461746520626567696E0A00000056
:1058A0006E6F207570646174650A000070B59CB0FD
:1058B0000124924D642103A8FDF7DEF8904800789A
:1058C000092873D2DFE800F005151F39424B6973D0
:1058D0007A00FEF71BFA8B4800780C2805D10120CE
:1058E0008749087085F8520002E0002085F85200D0
:1058F00000E1FFF76FF984480078082802D1022000
:105900007F490870F6E08148D0F8D8007F49D1F887
:10591000D410CDE900107D4804227DA1D0F8D0300C
:1059200003A804F017F803A800F00AF90446012CB4
:1059300002D1032072490870DCE002F019FE04462F
:10594000012C02D108206E490870D3E009F0CAFB8F
:105950000446012C02D1082069490870CAE0FFF70B
:105960002BFD6A48406888B96848806870B96D48FE
:105970000078401C6B4908700846007804280BD159
:105980000020087006205E49087005E00020654987
:10599000087006205A490870ACE000F033F904465C
:1059A000012C02D1082056490870A3E0A1E000F0C4
:1059B000F5F904460820524908709BE040F6B832D9
:1059C00059495A4802F046FD58480068C06840F0FE
:1059D000100056490968C8605548007800284BD027
:1059E0005148FDF77CF886B24FF0FF3332464E49FE
:1059F000504802F047FDFFF7E7FD84B2662C0CD15A
:105A0000424890F8DC00012807D104203C49087086
:105A1000002400204849088026E0662C07D1032096
:105A20003749087000240020434908801CE040F2F8
:105A30005D20844207D105203149087000240020F0
:105A40003D49088010E06A2C07D107202C490870D6
:105A5000002400203849088006E040F25A208442A1
:105A600002D1FF202649087040F6B8312E48FDF7D4
:105A700003F800202E4908703048007801281BD117
:105A80002D4800880A2805DA2B480088401C2A493E
:105A900008802DE00020284908800520184908705A
:105AA000224802F0DDF921480068C06820F01000AB
:105AB0001E490968C8601BE01F480088B0F5967F42
:105AC00005DA1D480088401C1B49088010E00020B2
:105AD0001949088005200A490870144802F0C0F9E5
:105AE00012480068C06820F0100010490968C860BA
:105AF00000E000BF00BF1CB070BD0000101000200F
:105B00006D1000206B1000206C100020341200205B
:105B1000746F636C69656E742F25642F2578257802
:105B20002578000074100020A0210020582D0020AE
:105B3000A2100020A02D0020721000209011002043
:105B400030B599B0044664216846FCF795FF0025FE
:105B500022460EA1684603F0FDFE6846FEF7C4F833
:105B600010A0FDF7F3FF0546012D05D112A003F0AB
:105B7000C9FE012019B030BD022D04D118A003F0D8
:105B8000C1FE0020F6E70020F4E7000041542B514D
:105B90004D545355423D302C312C222573222C304C
:105BA0000D0A00002B514D545355423A20302C31F0
:105BB0002C302C30000000005375627363726970E2
:105BC00074696F6E20746F2074686520746F7069DB
:105BD00063207375636365737366756C0D0A0000EB
:105BE000537562736372697074696F6E20746F208D
:105BF00074686520746F706963206661696C6564A0
:105C00000D0A00002DE9F0438FB000250024002686
:105C1000342102A8FCF730FF05F01BFA05463AA034
:105C200005F020FA07463A4639A1284605F0DEF984
:105C3000394805F017FA07463A4638A1284605F0D4
:105C4000D5F938A005F00EFA07463A4637A128469E
:105C500005F0CCF938A005F005FA07463A4638A118
:105C6000284605F0C3F92C484C38D0F8D8000090ED
:105C700029484C38D0F8D43034A1D0F8D02002A82C
:105C800003F068FE02A805F0EDF907463A4631A197
:105C9000284605F0ABF931A005F0E4F907463A468D
:105CA00030A1284605F0A2F91B494C39C868FDF718
:105CB00095FA074605F0BBF981464A462DA12846CC
:105CC00005F094F900202D4905F0B1F907463A4650
:105CD0002BA1284605F08AF9284605F069FA044602
:105CE000284605F0CDF92046FCF7F9FE87B23A4682
:105CF000214625A0FFF7ACFA0646204605F0F4FC45
:105D000030460FB0BDE8F0836A736F6E000000008C
:105D10006D7367547970650080120020696D736936
:105D20000000000056312E300000000068617264EF
:105D300056657273696F6E00563130303100000065
:105D4000736F667456657273696F6E002578257877
:105D500025780000646576496400000056322E30D4
:105D60000000000070726F746F636F6C5665727321
:105D7000696F6E0074786E4E6F0000000000104076
:105D80006465765479706500746F536572766572D8
:105D90002F6D7174742F3130350000002DE9F04FF4
:105DA0008FB04FF00009002400250026A2463421C0
:105DB00002A8FCF761FE05F04CF9814698A005F0B9
:105DC00051F907463A4698A1484605F00FF9984818
:105DD00005F048F907463A4696A1484605F006F907
:105DE00096A005F03FF907463A4696A1484605F0C9
:105DF000FDF897A005F036F907463A4696A14846C1
:105E000005F0F4F88A484C38D0F8D800009088485B
:105E10004C38D0F8D43093A1D0F8D02002A803F0A9
:105E200099FD02A805F01EF907463A468FA148469B
:105E300005F0DCF88FA005F015F907463A468FA16A
:105E4000484605F0D3F87A494C39C868FDF7C6F9D9
:105E5000074605F0ECF883465A468CA1484605F003
:105E6000C5F800208B4905F0E2F807463A468AA1BA
:105E7000484605F0BBF805F0ECF806466C494C398D
:105E80004878FDF7ABF9074605F0D1F883465A4646
:105E900083A1304605F0AAF865494C39B1F8740081
:105EA000FDF79CF9074605F0C2F883465A467EA1E5
:105EB000304605F09BF85E494C39B1F87200FDF7A9
:105EC0008DF9074605F0B3F883465A4678A1304667
:105ED00005F08CF856486A3005F0C4F807463A4693
:105EE00075A1304605F082F851483C3805F0BAF803
:105EF00007463A4672A1304605F078F84C494C39CD
:105F00000878FDF76BF9074605F091F883465A4685
:105F10006DA1304605F06AF845494C39B1F860008A
:105F2000FDF75CF9074605F082F883465A4668A1FA
:105F3000304605F05BF83E494C39B1F86200FDF798
:105F40004DF9074605F073F883465A4662A130467C
:105F500005F04CF836494C39B1F86400FDF73EF9CC
:105F6000074605F064F883465A465DA1304605F0C1
:105F70003DF82F494C39B1F86800FDF72FF9074675
:105F800005F055F883465A4657A1304605F02EF8DD
:105F900027494C39B1F86C10254A4C3AB2F86A20BE
:105FA00001EB0240FDF709F9074605F040F883468A
:105FB0005A464FA1304605F019F81D494C39B1F841
:105FC0006E00FDF70BF9074605F031F883465A4697
:105FD00049A1304605F00AF805F020F8054631469B
:105FE000284604F0EEFF2A4645A1484604F0FEFF8D
:105FF000484605F0DDF80446484605F041F82046DD
:10600000FCF76DFD87B23A4621463FA0FFF720F925
:106010008246204605F068FB50460FB0BDE8F08F81
:106020006A736F6E000000006D73675479706500CD
:1060300080120020696D73690000000056312E3017
:10604000000000006861726456657273696F6E00CB
:106050005631303031000000736F667456657273CC
:10606000696F6E002578257825780000646576498B
:106070006400000056322E300000000070726F7411
:106080006F636F6C56657273696F6E0074786E4ED5
:106090006F00000000001040646576547970650060
:1060A00072743030330000007274303235000000FA
:1060B00072743032360000007274303237000000E3
:1060C00072743032380000007274303239000000CF
:1060D00072743033300000007274303331000000CD
:1060E00072743033320000007274303333000000B9
:1060F00072743033340000007274303335000000A5
:106100007274303030000000746F536572766572BF
:106110002F6D7174742F32303100000072B600BFE1
:10612000FEE770B586B004460D46012600200190BA
:1061300000F02CFD002002900494059501A902A80E
:1061400000F06AFC064600F0BFFC304606B070BDA9
:106150000021074AD1610749096941F00401054A54
:1061600011611146096941F0400111617047000059
:10617000002F0020002002400021074AD16107497A
:10618000096941F00201054A116111464861096936
:1061900041F0400111617047002F002000200240B3
:1061A0000022054BDA61054A126942F00102034BF5
:1061B0001A61018070470000002F0020002002407B
:1061C00000201E49C96801F0100139B11C49C96994
:1061D00041F002011A4AD16140F010001749C96824
:1061E00001F0040139B11649C96941F00101144AAD
:1061F000D16140F004001149C96901F0010169B1A0
:106200000F49C96941F004010D4AD16100BF0B4932
:10621000C96921F00101094AD16100BF00BF40F204
:106220000111884206D10549C96921F00101034ADB
:10623000D16101E00149C86000BF70470020024001
:10624000002F002070B5044600F070FE054609E0FE
:10625000601C38B124B100F069FE401BA04201D996
:10626000032070BD1248C06800F001000028EFD183
:106270000F48C06800F0200020B100BF20200C496A
:10628000C86000BF0A48C06800F0100048B908485C
:10629000C06900F0010020B90548C06800F00400A2
:1062A00018B1FFF78DFF0120DBE70020D9E70000E0
:1062B000002002402DE9F04104460E4617464FF0FB
:1062C000000809F095FD00F061FC002516E056F885
:1062D00025C0624600232146022000F0FFFB48B99A
:1062E00056F825102068884202D04FF0010807E0D8
:1062F000241D02E04FF0010802E06D1CBD42E6D310
:1063000000BF00F0E1FB0AF093FD4046BDE8F081DC
:1063100050B1002106E0054B03EB8102D2F8E827DB
:1063200004C0491C0329F6DB7047000000F0FF1F82
:106330000146002291F82100022808D00420886339
:1063400000BF002081F8200000BF012070470868CE
:10635000006820F00E000B6818600868006820F0E4
:1063600001000B68186091F8403001209840CB6B19
:106370005860012081F8210000BF002081F8200032
:1063800000BF1046E2E7000070B50446002594F80F
:106390002100022803D00420A0630125C1E0206869
:1063A000006820F00E00216808602068006820F076
:1063B0000100216808605C492068884252D95A4926
:1063C00078392068884201D1012047E05649643974
:1063D0002068884201D1102040E05349503920689C
:1063E000884201D1801539E04F493C392068884204
:1063F00001D1801432E04C4928392068884202D10A
:106400004FF480302AE0484914392068884202D18C
:106410004FF4801022E044492068884201D14004B2
:106420001CE042492068884201D1012016E03F4922
:1064300014312068884201D110200FE03B492831F7
:106440002068884201D1801508E038493C31206835
:10645000884201D1801401E04FF480303349091F94
:10646000086051E0304978392068884201D1012024
:1064700047E02D4964392068884201D1102040E06E
:10648000294950392068884201D1801539E02649D0
:106490003C392068884201D1801432E022492839F1
:1064A0002068884202D14FF480302AE01E49143916
:1064B0002068884202D14FF4801022E01A492068F7
:1064C000884201D140041CE018492068884201D16B
:1064D000012016E0154914312068884201D11020AE
:1064E0000FE0124928312068884201D1801508E068
:1064F0000E493C312068884201D1801401E04FF4FC
:106500008030094980394860012084F8210000BFAB
:10651000002084F8200000BF606B10B12046616B42
:106520008847284670BD00008000024008040240F1
:1065300070B50446E06B05682068066894F8401062
:10654000042088402840002875D006F00400002868
:10655000FAD02068006800F0200028B920680068A0
:1065600020F0040021680860D5492068884254D989
:10657000D34978392068884201D1042049E0D049C4
:1065800064392068884201D1402042E0CC4950392A
:106590002068884201D100153BE0C9493C39206898
:1065A000884202D14FF4804033E0C5492839206841
:1065B000884202D14FF480202BE0C1491439206871
:1065C000884202D14FF4800023E0BD492068884210
:1065D00001D1C0041DE0BB492068884201D10420DC
:1065E00017E0B84914312068884201D1402010E0FA
:1065F000B44928312068884201D1001509E0B14929
:106600003C312068884202D14FF4804001E04FF4D1
:106610008020AC49091F086054E0A94978392068F6
:10662000884201D104204AE0A549643920688842A3
:1066300002D1402043E04CE0A14950392068884213
:1066400001D100153BE09E493C392068884202D1C7
:106650004FF4804033E09A4928392068884202D1BB
:106660004FF480202BE0964914392068884202D1EB
:106670004FF4800023E092492068884201D1C00491
:106680001DE090492068884201D1042017E08D491F
:1066900014312068884201D1402010E08949283116
:1066A0002068884201D1001509E086493C31206804
:1066B000884202D14FF4804001E04FF480208049AD
:1066C00080394860E06A002802D02046E16A8847A5
:1066D000F4E094F84010022088402840002871D04F
:1066E00006F002000028FAD02068006800F02000C0
:1066F00040B92068006820F00A0021680860012085
:1067000084F821006E492068884254D96C49783950
:106710002068884201D1022049E069496439206833
:10672000884201D1202042E06549503920688842E2
:1067300001D140153BE062493C392068884202D1D2
:106740004FF4005033E05E4928392068884202D176
:106750004FF400302BE05A4914392068884202D1A6
:106760004FF4001023E056492068884201D180048C
:106770001DE054492068884201D1022017E05149A8
:1067800014312068884201D1202010E04D49283181
:106790002068884201D1401509E04A493C3120680F
:1067A000884202D14FF4005001E04FF400304549D7
:1067B000091F086054E0424978392068884202D1B4
:1067C00002204AE057E03E4964392068884201D1FE
:1067D000202042E03A4950392068884201D14015D2
:1067E0003BE037493C392068884202D14FF40050E1
:1067F00033E0334928392068884202D14FF4003011
:106800002BE02F4914392068884202D14FF4001040
:1068100023E02B492068884201D180041DE02949EA
:106820002068884201D1022017E0264914312068EF
:10683000884201D1202010E0224928312068884276
:1068400001D1401509E01F493C312068884202D13E
:106850004FF4005001E04FF400301949803948608E
:1068600000BF002084F8200000BFA06A30B320469B
:10687000A16A884722E094F8401008208840284008
:10688000E0B106F00800C8B12068006820F00E00F2
:106890002168086094F8401001208840E16B48604E
:1068A0000120A06384F8210000BF002084F82000AC
:1068B00000BF206B10B12046216B884770BD0000DF
:1068C00080000240080402400146002209B901206C
:1068D00070471E4B086898420BD21D4B0868C01ABF
:1068E0001423B0FBF3F08000086419480838C8632B
:1068F0000AE0164B0868C01A1423B0FBF3F08000BE
:10690000086412480838C863022081F8210008682A
:10691000026843F6F0708243D1E901031843CB6863
:1069200018430B6918434B6918438B691843CB69AB
:10693000184302430868026000208863012081F840
:106940002100002081F8200000BFC1E708040240B8
:10695000080002402DE9F04104460D4616461F4648
:106960004FF0000800BF94F82000012802D1022057
:10697000BDE8F081012084F8200000BF94F82100D8
:1069800001282CD1022084F821000020A063206877
:10699000006820F00100216808603B463246294625
:1069A0002046FDF739F9E06A30B12068006840F010
:1069B0000E00216808600BE02068006820F00400E9
:1069C000216808602068006840F00A0021680860BB
:1069D0002068006840F001002168086006E000BF00
:1069E000002084F8200000BF4FF002084046BFE7B7
:1069F00070B5044600F09AFA06462546681C10B1A8
:106A000004480078054400BF00F090FA801BA842BB
:106A1000FAD370BDAC1000202DE9F04104460E46BB
:106A20000127002500BF2648007E012802D1022050
:106A3000BDE8F08101202249087600BF20680228C5
:106A400013D14CF25030FFF7FDFB90BB0120FFF754
:106A50007FFB4CF25030FFF7F5FB07461948006901
:106A600020F004001749086123E04CF25030FFF792
:106A7000E9FBF0B94FF0FF303060A56812E028461E
:106A8000FFF77AFB4CF25030FFF7DCFB07460D486E
:106A9000006920F002000B4908610FB1356007E082
:106AA00005F50065D4E9021001EBC020A842E6D844
:106AB00000BF00BF00200249087600BF3846B7E794
:106AC000002F0020002002400348006940F08000B1
:106AD0000149086100207047002002402DE9FE4F67
:106AE00005468B4617469846012600240020029052
:106AF00000BF2448007E012802D10220BDE8FE8F9D
:106B000001202049087600BF4CF25030FFF79AFB75
:106B1000064686BB012D02D10120029006E0022D1F
:106B200002D10220029001E00420029000241EE025
:106B30002201B946C24648465146FBF761FF80B282
:106B40000190022000FB04B000900199FFF728FBA0
:106B50004CF25030FFF776FB06460B48006920F0F8
:106B600001000949086106B104E0601CC4B2029842
:106B70008442DDDB00BF00BF00200249087600BF71
:106B80003046BBE7002F00200020024000200849CB
:106B9000096901F0800151B10649054A5160064971
:106BA00051601146096901F0800101B1012070476F
:106BB0000020024023016745AB89EFCD2DE9F8475E
:106BC000024600239C467BE14FF0010808FA03F4DB
:106BD000D1F8008008EA0400A0427DD1DFF8F4A2D9
:106BE000D1F80480A8EB0A09D0453AD014DCB8F1FA
:106BF000030F50D009DCB8F1000F31D0B8F1010F0C
:106C00001CD0B8F1020F49D120E0B8F1110F18D013
:106C1000B8F1120F42D11EE0B9F5881F25D006DC6D
:106C2000B9F5803F20D0B9F5801F37D11AE0B9F50A
:106C3000001F18D0B9F5041F30D117E0D1F80CC0EF
:106C40002DE0D1F80C8008F1040C28E0D1F80C807C
:106C500008F1080C23E0D1F80C8008F10C0C1EE0C0
:106C600000BF00BF00BF00BF00BF00BFD1F8088059
:106C7000B8F1000F02D14FF0040C0BE0D1F80880FE
:106C8000B8F1010F03D14FF0080C146102E04FF08E
:106C9000080C546103E04FF0000C00E000BF00BF9F
:106CA000FF2801D8904601E002F104084646FF287B
:106CB00002D84FEA830803E0A3F108084FEA8808E6
:106CC0004746D6F800804FF00F0909FA07F928EA7D
:106CD00009080CFA07F900E07AE048EA0908C6F862
:106CE0000080D1F8048008F08058B8F1805F6FD13F
:106CF00000BFDFF8E481D8F8188048F00108DFF819
:106D0000D891C9F81880C846D8F8188008F001084A
:106D1000CDF8008000BF00BF4FEAB9384FEA9309B1
:106D200058F829504FEA83784FEA18794FF00F0846
:106D300008FA09F825EA0805DFF8A081424502D1E2
:106D40004FF0000824E0DFF89881424502D14FF06F
:106D500001081DE0DFF88C81424502D14FF00208A6
:106D600016E0DFF88481424502D14FF003080FE0BE
:106D7000DFF87881424502D14FF0040808E0DFF8DF
:106D80007081424502D14FF0050801E04FF006083E
:106D90004FEA83794FEA197908FA09F848EA0505B4
:106DA000DFF850814FEA930948F82950D1F8048060
:106DB00008F48018B8F5801F0BD1DFF83C81D8F8B3
:106DC000008048EA0008DFF83091C9F800800AE046
:106DD00075E0DFF82481D8F8008028EA0008DFF8A1
:106DE0001891C9F80080D1F8048008F40018B8F5AB
:106DF000001F0ED1DFF8008108F10408D8F80080E8
:106E000048EA0008DFF8F09009F10409C9F80080A9
:106E10000DE0DFF8E48008F10408D8F8008028EAE3
:106E20000008DFF8D49009F10409C9F80080D1F80E
:106E3000048008F40038B8F5003F0ED1DFF8B880C0
:106E4000A8F10408D8F8008048EA0008DFF8A89004
:106E5000A9F10409C9F800800DE0DFF89C80A8F1D1
:106E60000408D8F8008028EA0008DFF88C90A9F11F
:106E70000409C9F80080D1F8048008F48038B8F516
:106E8000803F0ED1DFF87080A8F10808D8F80080A4
:106E900048EA0008DFF86090A9F10809C9F8008005
:106EA0000DE0DFF85480A8F10808D8F8008028EA3F
:106EB0000008DFF84490A9F10809C9F800805B1CBC
:106EC000D1F8008028FA03F8B8F1000F7FF47CAE07
:106ED000BDE8F887000011100010024000080140D2
:106EE000000C014000100140001401400018014056
:106EF000001C01400800014008040140024693685C
:106F00000B400BB1012000E00020704710B5C268B3
:106F100021EA020302EA010443EA0443036110BDCB
:106F20000AB1016101E00B04036170470148006888
:106F300070470000A4100020034800680349097846
:106F40000844014908607047A4100020AC100020DC
:106F500010B50848006840F010000649086003209A
:106F600000F044F90F2000F007F800F055F8002079
:106F700010BD000000200240F0B587B00446002696
:106F80000027002500BF1F48806940F400601D49AC
:106F900088610846806900F40060009000BF00BF6F
:106FA00001A902A800F01EFA00F054FA064616489D
:106FB000B6FBF0F0471E15481549086040F2E7316E
:106FC0001348C1604760002101618160816100F068
:106FD0000BFD054695B90E4800F076FD05466DB9E6
:106FE000192000F06BF8102C07D20022214619203E
:106FF00000F0BEF80748046000E00125284607B00D
:10700000F0BD00000010024040420F00002C014083
:10701000B82E0020A810002008B500BF14488069D1
:1070200040F00100124988610846806900F00100C3
:10703000009000BF00BF00BF0846C06940F080500C
:10704000C8610846C06900F08050009000BF00BFD2
:1070500000220F21901E00F08BF800BF0549486800
:1070600020F0E06040F00070486000BF08BD000004
:10707000001002400000014010B5014608460028FB
:1070800017DB00F01F0301229A400B4B440943F821
:10709000242000BF00BF00BFBFF34F8F00BF00BF61
:1070A00000BF00BF00BF00BFBFF36F8F00BF00BFB6
:1070B00000BF00BF10BD000080E100E001460846AF
:1070C000002809DB00F01F0301229A4043099B00BE
:1070D00003F1E023C3F8002100BF70472DE9F0431E
:1070E00004462046002803DB1F4F3F5C3F0907E0B2
:1070F0001E4F00F00F0CACF1040C17F80C703F0998
:107100003D460E4606F00700C0F10708B8F1040F2F
:1071100002D94FF0040801E0C0F10708C44600F1AD
:107120000408B8F1070F02D24FF0000801E0A0F107
:107130000308474625FA07F84FF0010909FA0CF948
:10714000A9F1010908EA0908C2F800804FF0010816
:1071500008FA07F8A8F1010808EA0508C3F8008052
:1071600000BFBDE8F083000000E400E018ED00E09F
:107170002DE9F05F80460D461646002702F012FC0E
:10718000074639462A46334601F00700C0F1070A90
:10719000BAF1040F02D94FF0040A01E0C0F1070A66
:1071A000D14600F1040ABAF1070F02D24FF0000AEB
:1071B00001E0A0F1030AD4464FF0010A0AFA09FAE5
:1071C000AAF1010A0AEA020A0AFA0CFA4FF0010BC4
:1071D0000BFA0CFBABF1010B0BEA030B4AEA0B04B5
:1071E0002146404602F0E6FBBDE8F09F00BF00F0FC
:1071F0000702064B19684FF6FF031940044B0B4377
:1072000043EA0221014B196000BF70470CED00E01A
:107210000000FA0500BF00BF00BF00BF00BFBFF302
:107220004F8F00BF00BF00BF0948006800F4E06056
:1072300008490843001D0649086000BF00BF00BFA1
:10724000BFF34F8F00BF00BF00BF00BF00BFFDE70F
:107250000CED00E00000FA0570B504460D460CB9CF
:10726000012070BD5A48006800F00700A8420ED205
:107270005748006820F00700284355490860084631
:10728000006800F00700A84201D00120E9E720785B
:1072900000F0020002281DD1207800F0040004282C
:1072A00005D14C48406840F4E0604A494860207885
:1072B00000F00800082805D14648406840F46050B6
:1072C000444948604348406820F0F000A168084302
:1072D00040494860207800F0010078B360680128D8
:1072E00006D13C48006800F4003090B90120B8E7AE
:1072F0006068022806D13748006800F0007040B985
:107300000120AEE73348006800F0020008B9012010
:10731000A7E73048406820F00300616808432D4922
:107320004860FFF703FE064609E0FFF7FFFD801BFC
:1073300041F28831884202D9032092E707E02548CC
:10734000406800F00C006168B0EB810FEDD120487F
:10735000006800F00700A8420ED91D48006820F020
:10736000070028431A4908600846006800F0070033
:10737000A84201D0012074E7207800F0040004281E
:1073800007D11448406820F4E060E16808431149DF
:107390004860207800F00800082808D10D484068AF
:1073A00020F46050216940EAC1000A49486000F0B9
:1073B00061F808494968C1F30311074A515CC840A4
:1073C0000649086006480068FFF7D6FD002048E738
:1073D0000020024000100240BE110108B010002041
:1073E000A81000200F2202600D4A526802F003022A
:1073F00042600B4A526802F0F0028260084A52680A
:1074000002F4E062C260064A526802F46052D20896
:107410000261044A126802F007020A607047000025
:107420000010024000200240014800687047000040
:10743000B010002000B5FFF7F7FF04494968C1F319
:107440000221034A515CC84000BD00000010024008
:10745000CE11010800B5FFF7E7FF04494968C1F301
:10746000C221034A515CC84000BD00000010024028
:10747000CE11010870B50021002200240023002055
:10748000134D696801F00C05F5B1042D02D0082DEB
:1074900019D101E00F4819E00F4DC1F38346AB5DF0
:1074A00001F4803555B10A4D6D68C5F340450B4E6A
:1074B000725D084D5D43B5FBF2F402E0084D03FB3D
:1074C00005F4204602E000BF024800BF00BF70BDC7
:1074D0000010024000127A00AC110108BC11010832
:1074E00000093D00F8B504460CB90120F8BD20782C
:1074F00000F00100002878D0F848406800F00C0047
:1075000004280CD0F548406800F00C00082811D180
:10751000F248406800F48030B0F5803F0AD1EF486F
:10752000006800F4003000285FD0606800285CD15B
:107530000120DBE700BF6068B0F5803F06D1E74877
:10754000006840F48030E549086028E0606858B978
:10755000E248006820F48030E0490860084600688E
:1075600020F4802008601AE06068B0F5A02F0BD1ED
:10757000DA48006840F48020D8490860084600686E
:1075800040F4803008600AE0D448006820F480307D
:10759000D24908600846006820F48020086000BFD7
:1075A000606888B1FFF7C2FC054606E0FFF7BEFC45
:1075B000401B642801D9032098E7C848006800F4FC
:1075C00000300028F2D010E0FFF7B0FC054606E0DE
:1075D000FFF7ACFC401B642801D9032086E7BF48B5
:1075E000006800F400300028F2D1207800F002009A
:1075F000022857D1B948406800F00C0050B1B74894
:10760000406800F00C00082818D1B448406800F425
:10761000803098B9B148006800F0020020B12069BC
:10762000012801D0012061E7AC48006820F0F80093
:10763000616940EAC100A949086033E02069E8B106
:107640000120A7490860FFF771FC054606E0FFF737
:107650006DFC401B022801D9032047E79F480068C2
:1076600000F002000028F2D09C48006820F0F800EA
:10767000616940EAC1009949086013E00020984917
:107680000860FFF753FC054606E0FFF74FFC401B80
:10769000022801D9032029E79048006800F0020081
:1076A0000028F2D1207800F0080008282DD1A06928
:1076B000B8B101208B490860FFF738FC054606E0A9
:1076C000FFF734FC401B022801D903200EE7834852
:1076D000406A00F002000028F2D0012001F0CEFB49
:1076E00013E000207F490860FFF720FC054606E014
:1076F000FFF71CFC401B022801D90320F6E677485F
:10770000406A00F002000028F2D1207800F0040066
:10771000042873D100277148C06900F0805070B907
:1077200000BF6E48C06940F080506C49C86108468F
:10773000C06900F08050009000BF00BF01276A4878
:10774000006800F48070B0B96748006840F4807049
:1077500065490860FFF7EAFB054606E0FFF7E6FB30
:10776000401B642801D90320C0E65F48006800F48C
:1077700080700028F2D000BFE068012806D1574889
:10778000006A40F001005549086227E0E06858B9F6
:107790005248006A20F00100504908620846006A19
:1077A00020F00400086219E0E06805280BD14B487E
:1077B000006A40F00400494908620846006A40F047
:1077C000010008620AE04548006A20F001004349D0
:1077D00008620846006A20F00400086200BFE06802
:1077E000A0B1FFF7A3FB054609E0FFF79FFB401B95
:1077F00041F28831884202D9032077E622E03748F7
:10780000006A00F002000028EFD012E0FFF78EFBC4
:10781000054608E0FFF78AFB401B41F288318842A9
:1078200001D9032062E62D48006A00F0020000281A
:10783000F0D1012F05D12948C06920F08050274997
:10784000C86100BFE069C8B32448406800F00C007C
:10785000082860D0E069022848D100202049086645
:10786000FFF764FB054606E0FFF760FB401B0228BC
:1078700001D903203AE61948006800F0007000289A
:10788000F2D1206AB0F5803F07D11448406820F457
:107890000030A168084311494860D4E90801084351
:1078A0000E49496821F4741108430C4948600120CD
:1078B0000B490866FFF73AFB054607E03DE0FFF796
:1078C00035FB401B022801D903200FE6034800685E
:1078D00000F000700028F2D02FE0000000100240FD
:1078E00000004242800442420070004000201449DF
:1078F0000866FFF71BFB054606E0FFF717FB401B7A
:10790000022801D90320F1E50E48006800F000705C
:107910000028F2D111E0E069012800D1E6E509482C
:10792000466806F48031206A814204D106F4701161
:10793000606A814201D00120D8E50020D6E5000030
:1079400000004242001002407047704730B50246C6
:107950000B4600BF92F83C00012801D1022030BD47
:10796000012082F83C0000BF022082F83D00106830
:1079700044681068816824F0700418680443106833
:107980004460144D1068A84213D0134D1068A842EB
:107990000FD01068B0F1804F0BD0104D1068A84286
:1079A00007D00F4D1068A84203D00E4D1068A842B2
:1079B00005D121F0800158680143106881600120E1
:1079C00082F83D0000BF002082F83C0000BF00BFED
:1079D000C5E70000002C01400034014000040040D5
:1079E00000080040000C004010B504460CB901200E
:1079F00010BD94F83D0028B9002084F83C002046D2
:107A000000F026F8022084F83D00211D206801F0D6
:107A1000BFFA012084F8460000BF84F83E0001212F
:107A20003F200155402001554120015500BF00BFB6
:107A3000012084F84200432001554420015545208F
:107A4000015500BF012084F83D000020D0E7000070
:107A500038B504462068B0F1804F16D100BF1848F1
:107A6000C06940F001001649C8610846C06900F0CD
:107A70000100009000BF00BF002205211C20FFF77D
:107A800077FB1C20FFF71AFB19E00E49206888429B
:107A900015D100BF0A48C06940F004000849C86118
:107AA0000846C06900F00400009000BF00BF00223B
:107AB00005211E20FFF75CFB1E20FFF7FFFA38BDF3
:107AC0000010024000080040014691F83D000128E6
:107AD00001D001207047022081F83D000868C0688D
:107AE00040F001000B68D860164B0868984213D02C
:107AF000154B086898420FD00868B0F1804F0BD042
:107B0000124B0868984207D0114B0868984203D07E
:107B1000104B086898420CD10868806800F0070292
:107B2000062A0CD00868006840F001000B68186055
:107B300005E00868006840F001000B68186000204C
:107B4000C8E70000002C0140003401400004004060
:107B500000080040000C00402DE9F04104460D46AD
:107B6000002700BF94F83C00012802D10220BDE8A4
:107B7000F081012084F83C0000BF022084F83D0021
:107B80002068866826F0770626F47F46206886609F
:107B90002868502833D00CDC202850D004DC002882
:107BA0004BD0102851D149E0302849D040284CD141
:107BB00039E060282DD0702807D0B0F5805F03D061
:107BC000B0F5005F41D10DE041E0D5E902136A68EC
:107BD000206801F02BFA2068866846F07706206856
:107BE000866034E0D5E902136A68206801F01EFA65
:107BF0002068806840F480402168886027E0EA6857
:107C00006968206801F026FA5021206801F019FA0D
:107C10001DE0EA686968206801F02FFA6021206899
:107C200001F00FFA13E0EA686968206801F012FABF
:107C30004021206801F005FA09E000BF00BF00BF45
:107C40002968206801F0FDF901E0012700BF00BFAD
:107C5000012084F83D0000BF002084F83C0000BFF4
:107C6000384684E7704710B5044620680069C0F3C1
:107C70004000D8B12068C068C0F34000B0B16FF0D8
:107C8000020021680861012020772068806900F0E7
:107C9000030018B12046FFF7E5FF05E0204600F09D
:107CA000ADF8204600F0ABF800202077206800698E
:107CB000C0F38000D8B12068C068C0F38000B0B1C4
:107CC0006FF0040021680861022020772068806935
:107CD00000F4407018B12046FFF7C4FF05E02046CD
:107CE00000F08CF8204600F08AF800202077206809
:107CF0000069C0F3C000D8B12068C068C0F3C000FC
:107D0000B0B16FF008002168086104202077206876
:107D1000C06900F0030018B12046FFF7A3FF05E09B
:107D2000204600F06BF8204600F069F8002020772C
:107D300020680069C0F30010D8B12068C068C0F3A3
:107D40000010B0B16FF010002168086108202077A2
:107D50002068C06900F4407018B12046FFF782FF28
:107D600005E0204600F04AF8204600F048F80020E0
:107D700020772068006900F0010058B12068C068D1
:107D800000F0010030B16FF0010021680861204669
:107D900000F036F820680069C0F3C01058B12068C0
:107DA000C068C0F3C01030B16FF080002168086176
:107DB0002046FFF7C9FD20680069C0F3801058B164
:107DC0002068C068C0F3801030B16FF040002168B7
:107DD0000861204600F042F820680069C0F34010B6
:107DE00058B12068C068C0F3401030B16FF0200077
:107DF000216808612046FFF7A8FD10BD7047704755
:107E00001CB5044611492068884201D1FFF794F857
:107E10002068B0F1804F05D16B4601AA03211C20D8
:107E2000FFF75CF90A492068884205D16B4601AA30
:107E300003211D20FFF752F906492068884204D12A
:107E400005480068401C044908601CBD002C014026
:107E50000004004000080040781000207047704780
:107E600070B50446002520684069C0F3C01594F839
:107E70004100212817D1B5B100BF00BF21681431DE
:107E800051E8001F21F080002168143141E8000210
:107E9000002AF3D100BFA06B10B1A06BFEF748FA27
:107EA000204601F029FA20684069C0F3801594F853
:107EB0004200222817D1B5B100BF00BF216814319C
:107EC00051E8001F21F040002168143141E8000210
:107ED000002AF3D100BFE06B10B1E06BFEF728FA87
:107EE000204601F0C3F9002070BD70472DE9F84F1E
:107EF0000446206805682068C668206847694FF016
:107F00000009CA4605F00F09B9F1000F0AD105F0C2
:107F1000200038B106F0200020B1204601F0FFF922
:107F2000BDE8F88FB9F1000F7BD007F0010018B958
:107F300006F49070002874D005F0010030B106F40A
:107F4000807018B1606C40F00100606405F00400BE
:107F500030B107F0010018B1606C40F002006064BD
:107F600005F0020030B107F0010018B1606C40F07C
:107F70000400606405F0080048B106F0200010B964
:107F800007F0010018B1606C40F008006064606C9C
:107F9000002845D005F0200028B106F0200010B1DF
:107FA000204601F0BCF920684069C0F3801A606C7B
:107FB00000F0080010B9BAF1000F2CD0204601F0F3
:107FC00055F92068406900F0400000B300BF00BFD1
:107FD0002168143151E8001F21F04000216814315C
:107FE00041E80002002AF3D100BFE06B50B17748AE
:107FF000E16B4863E06BFEF7C7F988B1E06B416B5A
:1080000088470DE02046FFF770FF09E009E02046B1
:10801000FFF76BFF04E02046FFF767FF0020606476
:108020007EE7206B012877D105F01000002873D07F
:1080300006F010000028FAD000BF00200090206851
:108040000068009020684068009000BF00BF206872
:10805000406900F0400000285FD0E06B0068406895
:108060001FFA80F8B8F1000F55D0A08D404552DDC1
:10807000A4F82E80E06B8069202843D000BF00BFA9
:1080800021680C3151E8001F21F4807021680C3107
:1080900041E80002002AF3D100BF00BF00BF216801
:1080A000143151E8001F21F001002168143141E82A
:1080B0000002002AF3D100BF00BF00BF21681431C5
:1080C00051E8001F21F040002168143141E800020E
:1080D000002AF3D100BF202084F842000020206352
:1080E00000BF00BF21680C3151E8001F21F01000D3
:1080F00021680C3141E80002002AF3D100BFE06B97
:10810000FEF716F902206063A08DE28D801A81B21D
:108110002046FFF7A4FE03E742E0A08DE18D401A60
:108120001FFA80F8E08DD0B3B8F1000F37D000BF50
:1081300000BF21680C3151E8001F21F490702168C4
:108140000C3141E80002002AF3D100BF00BF00BF9C
:108150002168143151E8001F21F001002168143119
:1081600041E80002002AF3D100BF202084F8420039
:108170000020206300BF00BF21680C3151E8001FC0
:1081800021F0100021680C3141E80002002AF3D1EF
:1081900000BF0220606341462046FFF760FEBFE655
:1081A00005F0800030B106F0800018B1204601F0E3
:1081B00017FAB5E605F0400030B106F0400018B1FE
:1081C000204601F089F8ABE600BFA9E6319100082E
:1081D00010B504460CB9012010BDA06900B100E043
:1081E00000BF94F8410028B9002084F840002046E0
:1081F00000F02AF8242084F841002068C06820F4A8
:1082000000502168C860204601F008F92068006924
:1082100020F49040216808612068406920F02A001D
:10822000216848612068C06840F400502168C86037
:1082300000206064202084F8410084F8420000207F
:10824000606300BFC8E7000010B586B00446002098
:10825000029003900490059073492068884250D1A1
:1082600000BF7248C06940F400207049C8610846E8
:10827000C06900F40020019000BF00BF00BF0846A5
:10828000806940F0100088610846806900F01000A5
:10829000019000BF00BF0815029002200390032048
:1082A000059002A96248FEF789FC4FF40060029035
:1082B00000200390049002A95D48FEF77FFC5D4812
:1082C0005D4908600020486000215B488160802192
:1082D000C1600021016141618161C161FEF7F4FA71
:1082E00008B1FDF71BFF00BF5348E063446200BFC5
:1082F000002205213420FEF73BFF3420FEF7DEFE8E
:108300008FE04E492068884237D100BF47488069D6
:1083100040F48040454988610846806900F4804007
:10832000019000BF00BF00BF0846806940F0040014
:1083300088610846806900F00400019000BF00BF1A
:1083400048150290022003900320059002A93C48A2
:10835000FEF734FC4FF480600290002003900490FC
:1083600002A93748FEF72AFC002205212520FEF746
:10837000FFFE2520FEF7A2FE53E032492068884226
:108380004FD100BF2948C06940F480202749C86107
:108390000846C06900F48020019000BF00BF00BF04
:1083A0000846806940F0080088610846806900F04E
:1083B0000800019000BF00BF081502900220039042
:1083C0000320059002A92048FEF7F8FB4FF4006057
:1083D000029000200390049002A91B48FEF7EEFBD8
:1083E0001A481B4908600020486000211848816035
:1083F0008021C1600021016141618161C161FEF79D
:1084000063FA08B1FDF78AFE00BF1148E0634462D9
:1084100000BF002205212720FEF7AAFE2720FEF735
:108420004DFE06B010BD0000004C004000100240A0
:108430000010014030040240302E0020003801407E
:108440000008014000480040000C0140300002409C
:10845000742E002070B504460D46164694F842006E
:1084600020280BD105B10EB9012070BD002020637A
:1084700032462946204601F04FF8F6E70220F4E79D
:10848000704770472DE9F84F04460E461746994647
:108490004FF0000A94F8410020284AD106B117B9DC
:1084A0000120BDE8F88F00206064212084F841009D
:1084B000FEF73CFD8246A784E784A068B0F5805FA4
:1084C00004D1206910B90025B04602E035464FF0CE
:1084D00000081BE05346002280212046CDF8009082
:1084E00001F0AEF808B10320DBE745B9B8F80000A9
:1084F000C0F308002168486008F1020803E028780A
:10850000216848606D1CE08C401EE084E08C0028EF
:10851000E0D15346002240212046CDF8009001F0E2
:108520008FF808B10320BCE7202084F84100002028
:10853000B7E70220B5E7704700BFFEE710B520217E
:108540000948FEF7E3FC4FF480710848FEF7DEFCB3
:108550004FF400710548FEF7D9FC4FF480610348E1
:10856000FEF7D4FC10BD0000000C014000140140D7
:108570002DE9F0438FB0002500240026342102A805
:10858000FAF77AFA02F065FD05463AA002F06AFDB4
:1085900007463A4639A1284602F028FD394802F03C
:1085A00061FD07463A4638A1284602F01FFD38A073
:1085B00002F058FD07463A4637A1284602F016FD5C
:1085C00038A002F04FFD07463A4638A1284602F08F
:1085D0000DFD2C484C38D0F8D800009029484C3874
:1085E000D0F8D43034A1D0F8D02002A801F0B2F9EC
:1085F00002A802F037FD07463A4631A1284602F0AC
:10860000F5FC31A002F02EFD07463A4630A128467F
:1086100002F0ECFC0020324902F009FD07463A4620
:1086200030A1284602F0E2FC16494C39C868FAF736
:10863000D5FD074602F0FBFC81464A462BA12846A1
:1086400002F0D4FC284602F0B3FD0446284602F0AE
:1086500017FD2046FAF743FA87B23A46214625A08D
:10866000FCF7F6FD0646204603F03EF830460FB014
:10867000BDE8F0836A736F6E000000006D7367548D
:108680007970650080120020696D73690000000038
:1086900056312E30000000006861726456657273B6
:1086A000696F6E005631303031000000736F6674B0
:1086B00056657273696F6E002578257825780000FD
:1086C000646576496400000056322E3000000000D8
:1086D00070726F746F636F6C56657273696F6E0042
:1086E00000001040646576547970650074786E4EB1
:1086F0006F000000746F5365727665722F6D717430
:10870000742F31303100000008B500BF15484069B2
:1087100040F00100134948610846406900F001003B
:10872000009000BF00BF00BF0846406940F0020053
:1087300048610846406900F00200009000BF00BF99
:10874000002205210D20FEF713FD0D20FEF7B6FCDB
:10875000002205213A20FEF70BFD3A20FEF7AEFC81
:1087600008BD00000010024010B51D4803F0ACFB2E
:108770001C4908601C4803F0A7FB1C4908601C4802
:1087800003F0A2FB1B4908601B4A0121084603F0C5
:1087900037FC1A4908601A4A0121084603F030FCE8
:1087A00018490860184B00220121184803F00CFDFD
:1087B00017490860174A0021174803F097FC17492A
:1087C0000860174A0021174803F090FC164908601A
:1087D000164A0021164803F089FC1649086010BDAE
:1087E0005C1101088C1000206C1101089010002011
:1087F0007C110108941000208C11010898100020B1
:108800009C1101089C1000204C110108BF90000829
:1088100088100020E0100108B98E00087C100020AC
:1088200004110108B19000088010002028110108EF
:10883000A39000088410002000B585B000200190AE
:1088400002900390049000BF4648806940F04000C9
:10885000444988610846806900F04000009000BFEC
:1088600000BF00BF0846806940F0080088610846E4
:10887000806900F00800009000BF00BF00BF0846FC
:10888000806940F0200088610846806900F020007F
:10889000009000BF00BF00BF0846806940F00400A0
:1088A00088610846806900F00400009000BF00BFA6
:1088B00000BF0846806940F0100088610846806962
:1088C00000F01000009000BF00BF01224FF44041B3
:1088D0002548FEF725FB002240F201712348FEF7F0
:1088E0001FFB00224FF480712148FEF719FB012283
:1088F00020212048FEF714FB4FF440400190012056
:108900000290002003900320049001A91648FEF76E
:1089100055F940F20170019001200290002003906F
:108920000320049001A91148FEF748F94FF4807024
:10893000019001200290002003900320049001A9DF
:108940000B48FEF73BF92020019001200290002007
:1089500003900320049001A90648FEF72FF905B003
:1089600000BD00000010024000180140001401404A
:1089700000080140000C014000B587B000200390C2
:10898000049005900690019002904FF080401449A9
:10899000086041F61F40486000211148816042F2A2
:1089A0000F71C160002101618161FFF71DF808B1FD
:1089B000FDF7B4FB4FF48050039003A90848FFF77C
:1089C000CBF808B1FDF7AAFB00200190029001A9A5
:1089D0000348FEF7BBFF08B1FDF7A0FB07B000BDE1
:1089E0004820002000B587B0002003900490059037
:1089F000069001900290144814490860472048608E
:108A00000021124881600921C1600021016181615A
:108A1000FEF7EAFF08B1FDF781FB4FF480500390A9
:108A200003A90A48FFF798F808B1FDF777FB002083
:108A30000190029001A90548FEF788FF08B1FDF7F3
:108A40006DFB07B000BD0000000800409020002032
:108A500010B50F480F4908604FF4E130486000211D
:108A60000C488160C16001610C214161002181617C
:108A7000C161FFF7ADFB08B1FDF750FB0548006889
:108A8000C06840F0100003490968C86010BD0000CC
:108A9000004C0040582D002010B50B480B490860D1
:108AA0004FF4E1304860002108488160C1600161F5
:108AB0000C21416100218161C161FFF789FB08B18F
:108AC000FDF72CFB10BD000000380140A02D002058
:108AD00010B50F480F4908604FF4E130486000219D
:108AE0000C488160C16001610C21416100218161FC
:108AF000C161FFF76DFB08B1FDF710FB0548006889
:108B0000C06840F0100003490968C86010BD00004B
:108B100000480040E82D002000BFFEE70246134653
:108B200010E010782A2805D01078202802DB107871
:108B30007A2801DDFF20704710782C2801D1481ECB
:108B4000C1B2521C0029ECD1D01AC0B2F3E7000028
:108B50002DE9F04F85B00446884683A14046F9F7D9
:108B600096FF074601213846FFF7D8FF0546FF2D3F
:108B700023D0781904A900F008F982469DF8101056
:108B80000A2000F0F7F8BAFBF0F642F21070B6FBDC
:108B9000F0F0C1B27E2001556420B6FBF0F06421F4
:108BA000B0FBF1F201FB12017F2001556420B6FBFE
:108BB000F0F100FB11618020015503213846FFF7D9
:108BC000ADFF0546FF2D45D0781904A900F0DDF86A
:108BD00006469DF81000801CC1B20A2000F0CAF8B9
:108BE000B6FBF0F044F8810F9DF81000801CC1B274
:108BF0000A2000F0BFF8B6FBF0F100FB116A504606
:108C0000FAF7D6FA81469DF81000C0F10500C1B20E
:108C10000A2000F0AFF80090FAF7CAFA83464946F6
:108C2000FAF7C5F882465249FAF7F3F8052102909F
:108C30000A2000F09FF8216800FB01FA5046FAF77D
:108C4000B7FA01900299FAF75AF80390FAF7D3FAB3
:108C500044F8810904213846FFF760FF0546FF2DDF
:108C600002D0785D84F8850005213846FFF756FF6D
:108C70000546FF2D45D0781904A900F086F8064670
:108C80009DF81000801CC1B20A2000F073F8B6FBFA
:108C9000F0F044F8860F9DF81000801CC1B20A2045
:108CA00000F068F8B6FBF0F100FB116A5046FAF7E5
:108CB0007FFA81469DF81000C0F10500C1B20A207C
:108CC00000F058F80090FAF773FA83464946FAF72D
:108CD0006EF882462649FAF79CF8052102900A2090
:108CE00000F048F8216800FB01FA5046FAF760FAF4
:108CF00001900299FAF703F80390FAF77CFA44F826
:108D0000860906213846FFF709FF0546FF2D02D0E8
:108D1000785D84F88A0009213846FFF7FFFE054692
:108D2000FF2D1ED0781904A900F02FF8064642F254
:108D30001070B6FBF0F0C1B27D2001556420B6FB87
:108D4000F0F06421B0FBF1F201FB12017C2001552F
:108D50006420B6FBF0F100FB116000F5FA60A4F8A6
:108D60007A0005B0BDE8F08F24474E524D43000015
:108D70000000704210B50246012000E050430B1E77
:108D8000A1F10104E1B2F9D110BD2DE9F34F81B099
:108D900007463C46002000908346814600268046D8
:108DA00028E020782D2802D148F00208641C2078A1
:108DB0002C2802D020782A2800D11CE020782E28E8
:108DC00003D148F00108641C09E02078392802DC4E
:108DD0002078302803DA4FF0000900260BE008F075
:108DE000010010B1701CC6B203E009F1010000F0EF
:108DF000FF09641CD5E700BF08F0020000B17F1C2A
:108E000000250EE0A9F10100401BC1B20A20FFF7C6
:108E1000B1FF795D3039009A00FB01200090681C99
:108E2000C5B24D45EEDB052E00DD05260298067025
:108E300000250EE0701E401BC1B20A20FFF79AFF0A
:108E400009F101012944795C303900FB01BB681C40
:108E5000C5B2B542EEDB31460A20FFF78BFF009921
:108E600001FB00BA08F0020008B1CAF1000A50463E
:108E7000BDE8FE8F00BFFEE77047704708B50849A0
:108E80000968C9084FF47A72B1FBF2F141430091CD
:108E900000BF00BF00994A1E00920029F9D108BD09
:108EA000B010002072B602480249086062B67047EE
:108EB0000028000808ED00E000BF012002F068FF74
:108EC000FBE7000010B500BF502080F31188BFF30E
:108ED0004F8FBFF36F8F00BF07F016FE18B14FF032
:108EE00080500449086000BF002080F3118800BF53
:108EF00010BD000004ED00E000B58FB0282105A8EA
:108F0000F9F7BAFD14216846F9F7B6FD012005907E
:108F100000040690002007900120099002200C9088
:108F2000C1030D914FF4E0110E9105A8FEF7DAFA96
:108F300008B1FDF7F3F80F20009002200190002007
:108F400002904FF480600390002004900221684654
:108F5000FEF782F908B1FDF7E1F80FB000BD7047E8
:108F600010B50248FEF77FFE10BD0000B82E0020AD
:108F700010B50248FEF777FE10BD00004820002023
:108F800010B50248FEF76FFE10BD000090200020D3
:108F900010B50268204B98420ED0204B98420BD05F
:108FA000B0F1804F08D01E4B984205D01D4B98421F
:108FB00002D01D4B984203D122F070024B681A4335
:108FC000154B98420ED0154B98420BD0B0F1804F04
:108FD00008D0134B984205D0124B984202D0124B46
:108FE000984203D122F44072CB681A4322F08003E6
:108FF0004C6943EA040202608B68C3620B688362B7
:10900000054B984202D0054B984201D10B6903638E
:109010000123436110BD0000002C014000340140D9
:109020000004004000080040000C004030B50C4631
:10903000816821F47F4142EA032525432943816069
:1090400030BD0A46816821F0700142F007031943E0
:109050008160704730B50B461446026A056A25F0F8
:1090600001050562816921F0F00141EA041122F055
:109070000A021A438161026230BD30B50B461446C4
:10908000026A056A25F010050562816921F47041C4
:1090900041EA043122F0A00242EA03128161026235
:1090A00030BD00BF06F054F9012002F071FEF9E76F
:1090B00000BF06F06BF9012002F06AFEF9E7704785
:1090C00070B50546284605F0E5FF044614B1D4E91D
:1090D0000010884770BD000008B51248FEF706FF73
:1090E000104800680068C0F30010D0B10E48007846
:1090F000401C0D49087000BF00200090094800681E
:1091000000680090074800684068009000BF00BFFA
:109110000448FEF7A5FE40F6B83204490148FFF7BF
:1091200099F908BD582D0020A2100020A021002090
:1091300070B505466C6A0020E085E0842046FEF7A5
:10914000D4FE70BD70B506460025746A206840697B
:10915000C0F3C01594F84100212805D125B10020A5
:10916000E084204600F0C8F820684069C0F380150C
:1091700094F84200222805D125B10020E085204640
:1091800000F074F8606C40F0100060642046FEF758
:10919000ACFE70BD70B505466C6A2868006800F0CA
:1091A0002000002842D1E08500BF00BF21680C31BB
:1091B00051E8001F21F4807021680C3141E8000261
:1091C000002AF3D100BF00BF00BF2168143151E86D
:1091D000001F21F001002168143141E80002002A3B
:1091E000F3D100BF00BF00BF2168143151E8001F58
:1091F00021F040002168143141E80002002AF3D137
:1092000000BF202084F84200206B01280ED100BF4F
:1092100000BF21680C3151E8001F21F010002168C7
:109220000C3141E80002002AF3D100BF0020606346
:10923000206B012804D1A18D2046FEF710FE02E02C
:109240002046FFF71DF970BD70B505466C6A012018
:109250006063206B012805D1A08D41082046FEF7F0
:10926000FEFD02E02046FFF70CF970BD00BF00BF15
:1092700002680C3252E8002F22F4907102680C321E
:1092800042E80013002BF3D100BF00BF00BF02680B
:10929000143252E8002F22F001010268143242E831
:1092A0000013002BF3D100BF016B01290ED100BFC9
:1092B00000BF02680C3252E8002F22F01001026851
:1092C0000C3242E80013002BF3D100BF202180F8BC
:1092D000421000210163704710B504462068C06841
:1092E00020F040002168C860202084F8410020461A
:1092F000FFF721F9002010BD00BF00BF02680C324B
:1093000052E8002F22F0C00102680C3242E800133C
:10931000002BF3D100BF202180F841107047F8B531
:10932000044694F84200222875D1A068B0F5805F09
:109330000CD1206950B90025A66A20684068C0F3A6
:1093400008003080A06A801CA06215E0A56A002693
:10935000A068B0F5805F03D0A06828B9206918B96B
:1093600020684068287004E02068406800F07F00B2
:109370002870A06A401CA062E08D401E80B2E0858B
:10938000002846D12068C06820F020002168C8600D
:109390002068C06820F480702168C8602068406937
:1093A00020F0010021684861202084F8420000205C
:1093B0006063206B012826D10020206300BF00BF1E
:1093C00021680C3151E8001F21F0100021680C3198
:1093D00041E80002002AF3D100BF2068006800F0D5
:1093E000100010280AD100BF0020009020680068FB
:1093F000009020684068009000BF00BFA18D20460B
:10940000FEF72DFD02E02046FFF73AF80020F8BDF8
:1094100001E00020FBE70220F9E7000070B50446F8
:109420002168096921F44051E26811432268116101
:109430002269A1681143626941EA02052168C9688D
:1094400041F20C62914329432268D1602168496945
:1094500021F44071A2691143226851612D4A2168AB
:10946000914202D1FDF7F6FF01E0FDF7E3FF00EBCB
:10947000C00101EB001162689200B1FBF2F100EB58
:10948000C00202EB001263689B00B2FBF3F264239C
:10949000B2FBF3F202EBC20303EB0212A1EB820177
:1094A000322202EB01116422B1FBF2F101F0F00172
:1094B00000EBC00202EB001263689B00B2FBF3F208
:1094C0006423B2FBF3F201EB021200EBC00101EBEB
:1094D000001163689B00B1FBF3F100EBC00303EBE9
:1094E00000136668B600B3FBF6F36426B3FBF6F32D
:1094F00003EBC30606EB0313A1EB8301322303EB5B
:1095000001116423B1FBF3F101F00F011144226852
:10951000916070BD0038014077B581B004461546B2
:109520000298A062A58500206064222084F8420091
:109530002848E16B88622848E16BC8622748E16BE4
:1095400008630020E16B486302AE32682368191D8E
:109550002B46E06BFDF7FEF900BF0020009020686D
:109560000068009020684068009000BF00BF20693C
:1095700070B100BF00BF21680C3151E8001F41F4F9
:10958000807021680C3141E80002002AF3D100BF4D
:1095900000BF00BF2168143151E8001F41F00100F5
:1095A0002168143141E80002002AF3D100BF00BF56
:1095B00000BF2168143151E8001F41F040002168CC
:1095C000143141E80002002AF3D100BF002004B0AA
:1095D00070BD00009591000849920008459100086F
:1095E000014691F84100212828D18868B0F5805FB4
:1095F0000BD1086948B90A6A1088C0F308000B68E3
:109600005860086A801C086205E00B6A581C0862F2
:1096100018780B685860C88C401E80B2C88458B94E
:109620000868C06820F080000B68D8600868C068CF
:1096300040F040000B68D860002070470220FCE733
:109640002DE9F04104460D4617469846069E34E043
:10965000701C88B32EB1FDF769FCA0EB0800B04286
:109660002BD900BF00BF21680C3151E8001F21F445
:10967000D07021680C3141E80002002AF3D100BF0C
:1096800000BF00BF2168143151E8001F21F0010024
:109690002168143141E80002002AF3D100BF2020E4
:1096A00084F8410084F8420000BF002084F84000A4
:1096B00000BF0320BDE8F081FFE720680068284074
:1096C000A84201D1012000E00020B842C0D0002013
:1096D000F0E7000010B50248FEF708FC10BD0000DE
:1096E000A02D002038B51848FEF700FC1648006889
:1096F0000068C0F3001028B314480078401C1349D8
:10970000087000BF002000900F48006800680090BB
:109710000D4800684068009000BF00BF0A48FEF78F
:109720009FFB0B48C06B00684068C0F1C80084B262
:109730002146084802F036FEC82207490248FEF7D3
:1097400089FE00BF38BD0000E82D0020A0100020D9
:10975000582D0020A0210020D8200020F0B5ADF524
:10976000197D4D4C642180A8F9F786F94B49E06ECC
:109770000968884273D94949E06E0968471AB7F504
:10978000007F01D2384601E04FF40070054643489F
:10979000006820676567206F04F1560340A26421CA
:1097A000CDE9000580A800F0BDF880A8FAF79CFA82
:1097B0004FF4007342A2642180A800F0B3F880A89F
:1097C000FAF7C4F901284BD141026846F9F754F978
:1097D000FF224FF400716846F9F747F98022694685
:1097E000394801F0BBFE18B100200DF5197DF0BD20
:1097F00000262CE05DF82610344802680068401C02
:10980000324B1860324840F8221018460068B0F514
:10981000007F1BD12F484078401C2E4948702C49AE
:109820002D48006806F052FB08B90020DDE7FF2252
:109830004FF400612648F9F718F900202349086021
:109840002548006800F5006023490860761C802EDA
:10985000D0D31248006828441049086002E019E09B
:109860000020C2E70D49E06E0968884211D8174808
:10987000006860B117484078401C16494870144988
:109880001548006806F022FB08B90020ADE701206A
:10989000ABE700BF0020A8E79411002010120020C1
:1098A00041542B514654504745543D222573222C98
:1098B00022434F4D3A222C25752C25750D0A0000A8
:1098C0000D0A4F4B0D0A0000A021002018120020A5
:1098D0000C640020781100201412002000BFFEE765
:1098E00070B5064C012529462046FCF71AFC6A0291
:1098F00003492046FCF7DEFC70BD000000F00708BD
:10990000781100200FB4054B10B503A9044A029842
:1099100000F0C0F910BC5DF814FB0000CDB60008E3
:10992000241200200FB41CB50246002007AC002909
:109930000BD0491ECDE90021054B6A462146069809
:1099400000F0A8F9009A002111701CBC5DF814FB0E
:10995000C3A300080FB4084B10B504A902AA0398CA
:1099600000F098F9044602A9002000F035FD2046D9
:1099700010BC5DF814FB0000D9A30008490050EAB0
:10998000C12018BF04204A0D18BF40F0010040F26A
:10999000FF72B2EB515F08BF40F00200012808BF20
:1099A0000520704702480068C0F30220704700009D
:1099B0000CED00E010B5002804DB0A07130E054A81
:1099C000135406E00A07140E034A00F00F031B1F8E
:1099D000D45410BD00E400E018ED00E000487047EA
:1099E00030120020EFF311807047EFF305807047CD
:1099F000EFF3108070472DE9F0414F1E00EBC701D7
:109A00000446D1E9000115461E4637F006020DD086
:109A10002A463346F9F7E2FA7F1E04EBC703D3E97F
:109A20000023F9F734FA37F00602F1D1022F25D0DE
:109A3000042F13D0062F18BFBDE8F0812A46334605
:109A4000F9F7CCFAD4E90A23F9F721FA2A46334682
:109A5000F9F7C4FAD4E90823F9F719FA2A46334684
:109A6000F9F7BCFAD4E90623F9F711FA2A46334686
:109A7000F9F7B4FAD4E90423F9F709FA2A46334688
:109A8000F9F7ACFAD4E90223F9F701FA2A4633468A
:109A9000F9F7A4FAD4E90023BDE8F041F9F7F7B9E2
:109AA0000022134610460149F9F70ABB0000F03FB7
:109AB0000122F9F7A9BDF9F7EAB9002213461046C9
:109AC0001146F9F7FDBA40F2013200204FF0E041B3
:109AD000F9F79ABD024A00201107F9F795BD000079
:109AE00001FDFFFF02E008C8121F08C1002AFAD1D9
:109AF00070477047002001E001C1121F002AFBD10E
:109B000070470000014908607047000030120020D3
:109B10002DE9FF5F82B00021DDE90430020DDDF8A0
:109B200040B0034318D044F61050A2F2FF32424333
:109B30001514119801281FD0A5EB0B00401C5FEAFB
:109B4000000A4FF000064E4FDFF83891B0465046FD
:109B500015D5CAF1000413E0119801244AA3012885
:109B600001D16FEA0B010298119AC0E90031C0E9F6
:109B7000024206B0BDE8F09FCBF10000DFE70446EB
:109B80000021404A491842EB0450CDE9001012E090
:109B9000E00707D032463B4640464946F9F71EFAF1
:109BA0008046894632463B4610461946F9F716FA72
:109BB00006460F466410002CEAD1DDE90401DDE918
:109BC0000023BAF1000F06DAF9F708FA42464B46CD
:109BD000F9F704FA05E0F9F773FA42464B46F9F74C
:109BE0006FFA04460E460022284BF9F763FB03D8B0
:109BF0004FF0FF30014607E00022254B204631465A
:109C0000F9F745F9F9F768FD102409E0002C0ADBA3
:109C10000A220023F9F798FB039B30321A55641E81
:109C200050EA0102F2D1641C039AC4F111031444F6
:109C3000119A012A03D0012208430DD10AE00843FA
:109C400004D000204FF0110B119072E7A3EB0B052D
:109C50006D1E0DE05B4504DD4FF0000205F10105CE
:109C600004E003DA4FF00002A5F10105002AECD070
:109C700002981199C0E90231C0E9004579E7000076
:109C8000000014400000F03F300000000000F043EE
:109C90000000E03F2DE9FF4F95B09B468946064600
:109CA00000250FE2252877D100242746F84A012114
:109CB000059400E0044316F8013F203B01FA03F04D
:109CC0001042F7D130782A2811D06FF02F03307866
:109CD000A0F13002092A16D8059A44F0020402EBDA
:109CE000820203EB42021044761C0590EFE759F81C
:109CF000042B0592002A03DA504244F400540590E4
:109D000044F00204761C30782E2816D116F8010F84
:109D100044F004042A280DD06FF02F023078A0F10F
:109D20003003092B09D807EB870302EB4303C7185D
:109D3000761CF3E759F8047B761C30786C280FD03A
:109D400006DC4C2817D068280DD06A2814D104E00E
:109D5000742810D07A280FD10DE044F400140AE0E2
:109D600044F4801401E044F440147278824202D139
:109D700004F58014761C761C307866280BD013DC32
:109D8000582877D009DC002875D04528F6D0462819
:109D9000F4D047281AD19DE118E0632835D0642813
:109DA00079D0652812D195E1702873D008DC672836
:109DB000F1D069286FD06E280DD06F2806D1B5E09C
:109DC00073282CD0752875D0782874D05A461799E6
:109DD00090476D1C75E1C4F30250022809D0032896
:109DE0000DD0D9F8001004280DD00D6009F1040938
:109DF00067E1D9F80010EA17C1E90052F6E7D9F88F
:109E000000100D80F2E70D70F0E719F8041B8DF8D3
:109E1000001000208DF80100EA46012003E059F807
:109E200004AB4FF0FF3061074FF0000102D40DE0AA
:109E300008F101018846B9420FDA8045F8DB1AF8CB
:109E400008100029F4D108E008F101018846814298
:109E5000FADB1AF808100029F6D105985B46A0EB4A
:109E6000080721463846179A00F094FA284400EB78
:109E7000080507E04DE029E10DE01AF8010B5A460C
:109E800017999047B8F10108F7D25B46214638464A
:109E9000179A13E142E00A220092C4F302524FF0F3
:109EA000000A022A08D059F804CB032A4FEAEC71C1
:109EB0000AD00DE029E02AE009F1070121F00702AC
:109EC000F2E802C1914609E00FFA8CFC4FEAEC710E
:109ED000042A03D14FFA8CFC4FEAEC71002907DA0F
:109EE0000A460021DCF1000C61EB02012D2202E0A8
:109EF000220504D52B228DF80420012203E0E2077D
:109F000001D02022F7E7904659E00A2102E0102212
:109F10000DE010214FF0000A00910BE010224FF0ED
:109F2000000A44F004040827009203E008224FF0DE
:109F3000000A0092C4F30252022A05D059F804CB59
:109F40000021032A08D009E009F1070121F00702E6
:109F5000F2E802C1914605E01FFA8CFC042A01D107
:109F60000CF0FF0C4FF00008220728D5702806D00F
:109F7000009B83F0100353EA0A0305D00EE0402251
:109F80008DF80420012208E05CEA010206D03022AC
:109F90008DF804208DF8050002229046009B83F086
:109FA000080353EA0A030AD15CEA010201D16207FD
:109FB00005D530228DF804204FF001087F1E582867
:109FC00004D034A003900EA802900DE036A0F9E76B
:109FD00053466046009AF9F7B7F984460398825CC5
:109FE0000298401E029002705CEA0100F0D10298D3
:109FF00006A9081A00F1200A600702D524F480346B
:10A0000000E00127574502DDA7EB0A0000E0002031
:10A0100000EB0A01009005984144401A0590E003C6
:10A0200006D45B462146179A059800F0B3F905441B
:10A03000002706E001A85A46C05D179990476D1C9D
:10A040007F1C4745F6DBE0030CD55B462146179A9B
:10A05000059800F09FF9054404E030205A4617990E
:10A0600090476D1C0099481E00900029F5DC08E01F
:10A07000029802995A460078491C02911799904714
:10A080006D1CBAF10001AAF1010AF1DC65E10000E2
:10A0900009280100303132333435363738396162BE
:10A0A0006364656600000000303132333435363782
:10A0B00038394142434445460000000000F058F959
:10A0C0000544761C307800287FF4ECAD19B02846A2
:10A0D000BDE8F08F620700D4062709F1070222F0DD
:10A0E000070CFCE80223E14603F000485FEA080C95
:10A0F00002D00FF2702C0DE05FEA045C02D50FF283
:10A10000682C07E05FEAC47C02D00FF2602C01E00B
:10A11000AFF2700C4FF0FF3823F00043CDF850C081
:10A1200065280CD006DC452809D046281DD04728D4
:10A130003DD13DE0662818D067287ED138E0002167
:10A14000112F01DB112000E0781CCDE9000106A9E8
:10A150000EA8FFF7DDFCDDE90F010E9A0391002147
:10A16000009207F1010A04914DE04FF00040009782
:10A17000CDE9011006A90EA8FFF7CAFCDDE90F0220
:10A1800003920E9B11990022DDF80CA0009304921B
:10A1900011B9791C00EB010AB7EB0A0004D4C0F135
:10A1A000FF3007F1010A0490AAEB0700019044E098
:10A1B000012F00DA01270021112F01DD112000E01D
:10A1C0003846CDE9000106A90EA8FFF7A1FCDDE99C
:10A1D0000F010E9A0391002104910092BA462107C3
:10A1E0000CD40399514500DA8A46BAF1010F05DD16
:10A1F000009AAAF10101515C302908D0B84202DA74
:10A2000010F1040F06DA0121CDE9011015E0AAF1E1
:10A210000101E9E7002805DC049901440491AAEB57
:10A22000000102E0411C514500DD8A460499401AB4
:10A23000401C01904FF000400290200704D4019888
:10A24000504501DBCDF8048000208DF84F000298C6
:10A250000DF14F07B0F1004F25D02B200E90029842
:10A260004FF0020800280CDA404202902D200E9098
:10A2700007E00A210298F9F751F83031029007F807
:10A28000011DB8F10001A8F10108F2DC02980028D4
:10A29000EFD1791E0E980870307800F0200040F061
:10A2A000450007F8020D12A8C01B00F1070814981A
:10A2B000007800B1012000EB0A01019801EBE07188
:10A2C00005984144401A401E0590E00306D45B46C1
:10A2D0002146179A059800F05DF805441498007817
:10A2E00018B15A46179990476D1CE00324D55B4678
:10A2F0002146179A059800F04DF805441CE0049893
:10A30000002807DBDDE90301884203DD0098405C9B
:10A31000179901E0179930205A469047049805F1A3
:10A320000105401C04900198401E019004D12E208C
:10A330005A46179990476D1CBAF10001AAF1010A1B
:10A34000DDDC05E017F8010B5A46179990476D1CA4
:10A35000B8F10001A8F10108F4DC5B462146179A28
:10A360000598ABE62D0000002B0000002000000047
:10A370002DE9F041044600251E461746880404D402
:10A3800005E039462020B0476D1C641EF9D52846EB
:10A39000BDE8F0812DE9F041044600251E469046B7
:10A3A000C80301D5302700E02027880404D505E044
:10A3B00041463846B0476D1C641EF9D52846BDE8B5
:10A3C000F0814A68002A06D00A68531C0B6010709E
:10A3D0004868401E486070470A68531C0B60107044
:10A3E000704700002DE9F04D8D4F21F0004A86B0F6
:10A3F00005460C46BA452ADBAAEB070028430AD0DB
:10A400008848824501DC1AD1CDB106B02846BDE8A6
:10A41000F04DFFF74DBB844A844B2846F8F7DEFD2C
:10A4200007460E46824A834B28462146F8F7D6FD5A
:10A4300006B03A463346BDE8F04DF8F728BD012096
:10A44000FFF760FB06B0BDE8F04DFFF736BB7A487A
:10A45000824542DABAF1795F0BDA2846FFF78EFAC5
:10A46000042808BFFFF736FB284606B02146BDE8A2
:10A47000F08D2A460B461046F8F7B0FD834602469B
:10A480006E480E460B4606217844FFF7B4FA5A464A
:10A490003346F8F7A3FD804669488A465A46334654
:10A4A00004217844FFF7A7FA5A463346F8F796FD99
:10A4B00000223B46F8F7EBFC02460B46404651466D
:10A4C000F8F7FEFD2A462346F8F788FD06B02A462F
:10A4D0002346BDE8F04DF8F7DABC284624F00041E9
:10A4E00000223D463B46F8F776FD4FF0FF32F9F784
:10A4F0008BF80646024653480F460B460621784421
:10A50000FFF779FA32463B46F8F768FDCDE90001DE
:10A510004D4832463B4604217844FFF76CFA3246F8
:10A520003B46F8F75BFD00222B46F8F7B0FC83466C
:10A5300002913046394604F0E2FE804643480D461B
:10A54000504517DCDDE900015A46029BF8F7B8FDDB
:10A5500042462B46F8F742FD42462B46F8F797FC59
:10A560000122F9F751F8304A304BF8F731FD304A03
:10A57000304B4CE04FF0000A52460B464046F8F78D
:10A5800086FCCDE9031052462B4610461946F8F7D3
:10A5900025FD32463B46F8F71EFDDDE90332F8F7AC
:10A5A0008FFD06460F46DDE900015A46029BF8F78B
:10A5B00087FD83460091012230463946F9F724F899
:10A5C000194A1A4BF8F707FD06460F460122404686
:10A5D0002946F9F719F85A46009BF8F7FFFC32466E
:10A5E0003B46F8F7F5FC06460F4601225046294641
:10A5F000F9F70AF80E4DDFF858802A464346F8F777
:10A60000EAFC32463B46F8F7E6FC2A464346F8F7B2
:10A61000E2FC002CD8BF81F0004106B0BDE8F08D0F
:10A620000000F03F0000F07F075C143326A6913C49
:10A63000182D4454FB21F93F0000E03F9C6D0000C1
:10A64000B26D0000266D00003C6D00003333EF3F1B
:10A65000FB21E93F2DE9F84F04460D4621F000406B
:10A6600000917349814211DC7249884201DC06D1B4
:10A670002CB120462946BDE8F84FFFF719BA6E48BD
:10A68000002DCCBF6D496E49BDE8F88F6D49814200
:10A6900011DD6D498142D8BF4FF0FF366DDD204698
:10A6A0002946FFF76BF9042808BFFFF713FA204685
:10A6B0002946BDE8F88F6549654F25F00045814280
:10A6C00033DD6449814219DD002632464FF0804374
:10A6D00020462946F8F7DBFB80468A4601222046C1
:10A6E0002946F8F791FF00223B46F8F771FC4246F5
:10A6F0005346F8F7E5FC04460D463EE001260022ED
:10A70000BA463B4620462946F8F7C1FB80460F462D
:10A710000022534620462946F8F75AFC42463B465B
:10A72000F8F7CEFC04460D4627E04B4981421BDD7D
:10A73000DFF828A102260022534620462946F8F7D2
:10A740004DFC00223B46F8F7A2FB80460F46002254
:10A75000534620462946F8F73BFC42463B46F8F76D
:10A76000AFFC04460D4608E0032622462B46002097
:10A770003B49F8F7A5FC04460D4622462B461046F9
:10A780001946F8F72BFC8B46824602460B46F8F733
:10A7900025FC07460246334888460B460621784486
:10A7A000FFF729F952465B46F8F718FC82462E4817
:10A7B0008B463A46434605217844FFF71CF93A4652
:10A7C0004346F8F70BFC02460B46002E504659460E
:10A7D0000CDAF8F75CFB22462B46F8F7FFFB01B0DA
:10A7E00022462B46BDE8F04FF8F7F5BBF8F74FFBD4
:10A7F00022462B46F8F7F2FB1C4A7A4402EBC603CA
:10A80000D3E90023F8F7E4FB22462B46F8F7E0FBF8
:10A81000174A7A4402EBC603D3E90023F8F7DBFBBF
:10A82000009A002AB8BF81F00041BDE8F88F00000F
:10A83000000010440000F07F182D4454FB21F93F24
:10A84000FB21F9BF0000DC3F0000203E0000F33F89
:10A850000000F03F0000E63F008003400000F83FAA
:10A860000000F0BF4E6C00000C6C0000AA6B0000F2
:10A87000726B00002DE9F04D9446CCF1000423F0FA
:10A8800000464CEA0404524F46EAD4749A4688467D
:10A8900021F00042BC4206D8454240EA050442EAA3
:10A8A000D474BC4204D9BDE8F04D6246FFF703B949
:10A8B000AAF14055A5F17F6555EA0C040BD002249E
:10A8C00004EAAA74434DDFF810E144EAD87452EA6E
:10A8D000000B04D00CE0BDE8F04DFFF7BBBE002C30
:10A8E00014BF012CBDE8F08D022C30D0032C32D0E7
:10A8F00056EA0C0B0AD0BE4220D1BA4209D126F04A
:10A90000804622F080423346114617E000291ADBC8
:10A9100025E0DFF8C8B0FB44002C04BFDBE90001F0
:10A92000BDE8F08D012C02BFDBE9000181F00041A0
:10A93000BDE8F08D022C0AD0032C0CD0BA4212D103
:10A94000B8F1000F0BDA23482549BDE8F08D284601
:10A950002449BDE8F08D28467146BDE8F08D1D48BC
:10A960002149BDE8F08D921B12153C2AC4BF19483D
:10A970001D490EDCBAF1000FBEBF12F13C0F0020E2
:10A98000014606DB6246F8F79BFB21F00041FFF72A
:10A9900061FE002C08BFBDE8F08D012C04BF81F0E2
:10A9A0000041BDE8F08D114A114B022C07D0F8F799
:10A9B0000FFB2A46BDE8F04D0A4BF8F709BBF8F744
:10A9C00007FB2A46BDE8F04D064BF8F704BB000034
:10A9D0000000F07F182D4454FB2109C0066B0000D5
:10A9E000FB21F9BFFB210940FB21F93F075C143330
:10A9F00026A6A13C2DE9F04F99B004460D46164617
:10AA00000027B846B946BA4612A814A913AB0EAA35
:10AA1000CDE9001015A917A800F064FC18B10120B9
:10AA200019B0BDE8F08FBDF8500000F48070002828
:10AA30007ED00E98F8F7B3FB83464FF09D41F8F7B0
:10AA4000E8F907460F98F8F7AAFB83464FF09D41B7
:10AA5000F8F7DFF980461098F8F7A1FB83464FF02E
:10AA60009D41F8F7D6F981461198F8F798FB83468F
:10AA70004FF09D41F8F7CDF9824639464FF08040BE
:10AA8000F8F795F949460590F8F791F9414607908E
:10AA90004FF04040F8F78BF951460590F8F787F9E9
:10AAA00006900799F8F72BF98346F8F7D7FBCDE91D
:10AAB0000801FFF797FC4FF06632544BCDE90A01CD
:10AAC000F8F78CFACDE90C01F8F70CFC2060494648
:10AAD0004FF08040F8F76BF949460290F8F767F9B4
:10AAE000414604904FF04040F8F761F9414602902A
:10AAF000F8F75DF903900499F8F753F983464FF09E
:10AB00007E51F8F7FCF80590F8F7A8FBCDE90801AD
:10AB100039464FF08040F8F74AF941460390F8F77C
:10AB200046F9494604904FF08040F8F740F900E0BC
:10AB300068E051460390F8F73AF983460499F8F72C
:10AB4000DEF80590F8F78AFBCDE90601DDE9082378
:10AB5000FFF790FE4FF066322C4BCDE90A01F8F773
:10AB60003DFACDE90C01F8F7BDFB2860514650468F
:10AB7000F8F71DF9494604904846F8F718F9414698
:10AB800003904046F8F713F9394601903846F8F734
:10AB90000EF900900199F8F7B2F802900399F8F7CE
:10ABA00000F983460499F8F7FCF80590F8F756FB8E
:10ABB000CDE9080151463846F8F7F9F849460490BE
:10ABC0004046F8F7F4F803900499F8F798F84FF036
:10ABD00080410590F8F7EBF88346F8F73FFBCDE9A5
:10ABE0000601DDE90823FFF745FE4FF06632074B0B
:10ABF000CDE90A01F8F7F2F9CDE90C01F8F772FB9B
:10AC0000306001E001200BE7002009E766A64C4018
:10AC100010B504460CB9012010BDFCF787F920607F
:10AC20000020F9E72DE9FC4104460D4616466B4627
:10AC300006224321682000F047F90746BFB99DF876
:10AC400001009DF8001040EA012000B220809DF82C
:10AC500003009DF8021040EA012000B228809DF810
:10AC600005009DF8041040EA012000B2308038460B
:10AC7000BDE8FC8110B500BF002280211048FCF720
:10AC80004FF900BF00F01EF800BF012240210C4820
:10AC9000FCF746F900BF00F015F800BF0022402184
:10ACA0000748FCF73DF900BF00F00CF800BF012297
:10ACB00080210348FCF734F900BF00F003F810BD11
:10ACC000000C014000B50220F8F7BCFF00BD0000F9
:10ACD00010B500BF012280210C48FCF721F900BF0C
:10ACE000FFF7F0FF00BF012240210848FCF718F9E8
:10ACF00000BFFFF7E7FF00BF002240210348FCF739
:10AD00000FF900BFFFF7DEFF10BD0000000C01408F
:10AD100070B50546002400261CE06006040E00BF46
:10AD2000012240211048FCF7FBF800BFFFF7CAFFE3
:10AD300080210D48FCF7E2F808B1601CC4B200BFE6
:10AD4000002240210848FCF7EBF800BFFFF7BAFFEC
:10AD5000701CC6B2082EE0DB15B9FFF7B9FF01E0A1
:10AD6000FFF788FF204670BD000C014070B5044617
:10AD7000002524E000BFE00928B101228021154808
:10AD8000FCF7CEF804E0002280211248FCF7C8F856
:10AD900000BFFFF797FF00BF012240210D48FCF7DD
:10ADA000BFF800BFFFF78EFF00BF00224021094817
:10ADB000FCF7B6F800BF6006040E681CC5B2082D8B
:10ADC000D8DB00BF012280210248FCF7A9F800BFB0
:10ADD00070BD0000000C014010B500BF01228021B1
:10ADE0000F48FCF79DF800BF00BF012240210C482E
:10ADF000FCF796F800BFFFF765FF00BF0022802137
:10AE00000748FCF78DF800BFFFF75CFF00BF00228A
:10AE100040210348FCF784F800BFFFF753FF10BD43
:10AE2000000C014010B500BF002280210C48FCF747
:10AE300077F800BFFFF746FF00BF01224021084816
:10AE4000FCF76EF800BFFFF73DFF00BF0122802135
:10AE50000348FCF765F800BFFFF734FF10BD0000A2
:10AE6000000C014070B50024002500BF01228021A4
:10AE70001448FCF755F800BFFFF724FF00BF01227C
:10AE800040211048FCF74CF800BFFFF71BFF07E01C
:10AE9000601CC4B2FA2C03DDFFF7C4FF012505E0F6
:10AEA00080210848FCF72AF80028F1D100BF00BF34
:10AEB000002240210348FCF733F800BFFFF702FFF0
:10AEC000284670BD000C01402DE9F04105460F46B3
:10AED00014461E46FFF780FF002141EA4501C8B233
:10AEE000FFF744FFFFF7BEFF012804D1FFF79AFFE9
:10AEF0000220BDE8F0813846FFF738FFFFF7B2FFC8
:10AF0000012803D1FFF78EFF0220F2E7FFF764FF6D
:10AF1000012101EB4501C8B2FFF728FFFFF7A2FFAF
:10AF2000012803D1FFF77EFF0220E2E70BE0012CAE
:10AF300001DD012100E000210846FFF7E9FE307045
:10AF4000601EC4B2761C002CF1D1FFF76BFF00200D
:10AF5000CFE72DE9F04105460E4617469846FFF724
:10AF60003BFF002141EA4501C8B2FFF7FFFEFFF7B2
:10AF700079FF012804D1FFF755FF0220BDE8F081D9
:10AF80003046FFF7F3FEFFF76DFF012803D1FFF70F
:10AF900049FF0220F2E700240DE018F80400FFF753
:10AFA000E5FEFFF75FFF012803D1FFF73BFF02201B
:10AFB000E4E7601CC4B2BC42EFDBFFF733FF0020C4
:10AFC000DCE770B505460E46AC6806B970BD0CB935
:10AFD000AE6009E000E0246814B120680028FAD1CE
:10AFE0003146204604F0B1F900BFEFE770B50646E0
:10AFF0000D46144604B970BD206A18B10649206A8E
:10B0000009688847284600F003F920622146304647
:10B01000FFF7D7FF00BFEEE70C10002010B500F0DF
:10B020007DF804460CB10520E060204610BD70B5E7
:10B0300005460E4600F072F8044644B10320E06075
:10B04000C4E9065628463146F8F7E9F8606120461B
:10B0500070BD10B500F062F804460CB10620E06047
:10B06000204610BD70B5054600F058F804462CB1D6
:10B070000420E060284600F0CBF82061204670BD37
:10B0800070B5044622E02568A08900F4807020B9DC
:10B09000A06810B1A068FFF7F3FFA08900F48070EA
:10B0A00028B9206918B10B49206909688847A08927
:10B0B00000F4007028B9206A18B10649206A0968AE
:10B0C000884720460349096888472C46002CDAD176
:10B0D00070BD00000C1000200246906801E0491E7F
:10B0E000006808B10029FADC704701468A68002030
:10B0F00001E0401C1268002AFBD1704770B505467C
:10B100000E46AC6800E024682CB13146206A00F09D
:10B1100058F80028F7D1204670BD000010B528204F
:10B1200005490968884704461CB128212046F7F7DD
:10B13000A3FC204610BD00000810002010B50446F6
:10B1400000221146204600F001F810BD2DE9F0471D
:10B1500080460D4616460024FFF7E0FF0746002014
:10B16000124908600FB9BDE8F087404604F0BEF808
:10B1700081464946384601F089FE044624B93846DE
:10B18000FFF77EFF0020EEE766B1204604F0AEF840
:10B190000446207830B13846FFF772FF0348046058
:10B1A0000020E0E705B12C603846DCE70410002001
:10B1B00010B50446002301221946204603F0B0F8DA
:10B1C00010BD70B504460D462CB9AC4201D001202B
:10B1D00070BD0020FCE70DB90120F9E705E02078FB
:10B1E00008B90020F4E7641C6D1C2078F7F725FCF3
:10B1F00006462878F7F721FC8642F0D02078F7F74A
:10B200001CFC06462878F7F718FC301AE0E7000027
:10B2100070B504462046F7F762FC451C28460649EF
:10B2200009688847061E00D170BD2A46214630466F
:10B23000F7F709FC3046F7E708100020F0B505469F
:10B240000C46042C02DA4FF0FF30F0BDA01E295C42
:10B25000601E285C41EA0027A11E284600F038FC49
:10B260000646B74201D10020EFE74FF0FF30ECE790
:10B2700010B50248FCF728FC10BD0000902000200B
:10B280002DE9F0410446E07800F0C006E07800F0D7
:10B290003F05607800F0010098B1EF102846E917EB
:10B2A00005EB5171C910A5EBC101491C01F0FF0864
:10B2B0000B48006820B10A4841460268384690476A
:10B2C00000BF607800F0080030B10548406818B150
:10B2D000B011034A516888470020BDE8F0810000A2
:10B2E000FC6300202DE9F04F8DB0074688461546D7
:10B2F0009946DDE9166B0024002030806B49887B7D
:10B300005A4605A900F000FC18B1601E0DB0BDE85A
:10B31000F08F6648807A00F01400002867D09DF80E
:10B32000140000069DF8151040EA01409DF8161023
:10B3300040EA01209DF81710084328609DF8180086
:10B3400000069DF8191040EA01409DF81A1040EAE5
:10B3500001209DF81B10084368609DF81C00000642
:10B360009DF81D1040EA01409DF81E1040EA0120A2
:10B370009DF81F100843A8609DF8200000069DF866
:10B38000211040EA01409DF8221040EA01209DF87A
:10B3900023100843E86004F11000C4B228680014C8
:10B3A0000190686800140290A86800140390E8688F
:10B3B0000014049001984043029901FB0100039995
:10B3C00001FB0100049901FB010ABAF1706F02DB75
:10B3D000BAF1885F05DD00F0F7FB00203080401EE9
:10B3E00094E7B6F9000040F48070308000BF2F4829
:10B3F000807A00F0400020B305A9601C085C095D5C
:10B4000040EA012000B2A8F8000005A9E01C095C90
:10B4100005AAA01C105C41EA002000B2A8F80200B6
:10B4200005A9601D095C201D105C41EA002000B2E6
:10B43000A8F80400A01DC4B2B6F9000040F008004E
:10B4400030801A48408900F4C07008B305A9601C18
:10B45000085C095D40EA012000B2388005A9E01CC3
:10B46000095C05AAA01C105C41EA002000B27880AB
:10B4700005A9601D095C201D105C41EA002000B296
:10B48000B880A01DC4B2B6F9000040F07000308052
:10B490000648807A00F0030018B105A90819FFF7E3
:10B4A000EFFE4846FFF7B4FB00202FE7FC630020C7
:10B4B00001210120094A12680AB100200CE0084A63
:10B4C00012680AB1002007E0064A1368064A1268AB
:10B4D000521E934200D1022070470000E833002042
:10B4E000D810002010340020C41000202DE9F041B5
:10B4F00004460E460CB1206810B90020BDE8F0816A
:10B50000A06806446068B04203DBA1682068084474
:10B51000F4E7304602F004FA074638460D49096858
:10B52000884705463DB90C492068096888470020CE
:10B5300060602060E2E725B12846D4E90012F7F701
:10B5400082FA054920680968884767602560A06815
:10B550002844D3E7081000200C1000202DE9FC5FE0
:10B560000646894692460FF2740B1FA00190594679
:10B570003046F7F78CFA044624B15846F7F7AFFA8D
:10B58000044400E034460198F7F7A9FA0090A01BA4
:10B5900040F6B832111A2046DDE9003203F080FE91
:10B5A000054615B90120BDE8FC9F2F1B07F00300DD
:10B5B00008B10120F7E74FEA9708D04501D90120EB
:10B5C000F1E74FEA880221464846F7F73CFA40F691
:10B5D000B8313046F7F750FA0020E4E70D0A434F40
:10B5E0004E4E4543540D0A000D0A4F4B0D0A000004
:10B5F0002DE9F041C1F30A52A2F2FF362F4A304B37
:10B600000D460446142E2FDA002E12DAF7F73FFC0F
:10B6100000221346F7F74EFE4CD2002DA4BF0024A3
:10B62000254647DA25F00040204318BF254D41D07C
:10B6300018E0DFF894C02CFA06F705EA070C5CEA7C
:10B64000040C08BFBDE8F081F7F721FC0022134687
:10B65000F7F730FE2ED2002D03DA4FF48010F040C1
:10B660000544BD43002425E0332EC8BFBDE8F0816A
:10B67000A6F1140C4FF0FF3727FA0CF73C4208BF35
:10B68000BDE8F081F7F7A7FC00221346F7F712FE9A
:10B6900010D2002D0DDA142E08BF6D1C09D0C6F192
:10B6A0003400012101FA00F02044A04238BF6D1C93
:10B6B0000446BC4329462046BDE8F0819C750088BD
:10B6C0003CE4377E0000F0BFFFFF0F0013B50C46CF
:10B6D0004FF47A73012269460248FCF7D3FE0098C2
:10B6E0001CBD0000A02D002010B5002821D0114B5A
:10B6F0000022001F196803E0814203D80A46496806
:10B700000029F9D152B11368841A9C4204D100680F
:10B7100018441060104602E0506000E0186039B133
:10B7200002680B1A934203D10B681A4402604968FD
:10B73000416010BD281200202DE9F04F89B0002093
:10B740000790089008AA911E07A8FFF76BFABDF9A9
:10B750002000F7F732FD044600224FF0804301F04D
:10B76000F3FB82468B46BDF91E00F7F726FD064621
:10B7700000224FF0804301F0E7FB04460D46BDF97F
:10B780001C00F7F71AFD064600224FF0804301F037
:10B79000DBFB804622462B46F7F779FB52465B4699
:10B7A000CDE90001F7F773FBCDE9020103F0A7FD36
:10B7B000CDE90401F7F796FD0690069809B0BDE8BB
:10B7C000F08F0000014800687047000078100020EA
:10B7D0002DE9FE4F002002900190009000BF6A46C4
:10B7E00002A901A8FFF706F90028F8D10198F7F798
:10B7F00035FD07463A460B4654A0FEF783F80298FB
:10B80000F7F72CFD07463A460B4653A0FEF77AF8A9
:10B810000098F7F723FD07463A460B4651A0FEF77E
:10B8200071F8FFF789FF044651480199006800F05C
:10B83000CDF801904F480299006800F0C7F80290D7
:10B840004D480099006800F0C1F8009021464B482F
:10B85000006800F0BBF80446454801680198F7F716
:10B86000A0FA8246F7F7FAFC21F000410746F7F705
:10B8700039FD05463F4801680298F7F792FA82467B
:10B88000F7F7ECFC21F000410746F7F72BFD0646E1
:10B89000394801680098F7F784FA8246F7F7DEFC2A
:10B8A00021F000410746F7F71DFD81462846F7F7CE
:10B8B000D5FC07463A460B4631A0FEF723F8304642
:10B8C000F7F7CCFC07463A460B4633A0FEF71AF8CA
:10B8D0004846F7F7C3FC07463A460B4634A0FEF746
:10B8E00011F82846F7F7BAFC07460022354BF7F760
:10B8F000E1FC11D33046F7F7B1FC07460022314B8B
:10B90000F7F7D8FC08D34846F7F7A8FC074600220B
:10B910002C4BF7F7CFFC03D201202B49087002E033
:10B9200000202949087012490198086011490298BD
:10B9300008601149009808601048046022480078A7
:10B94000012801D1BDE8FE8F0020FBE77069746318
:10B95000683A252E31660A00726F6C6C3A252E31DA
:10B96000660A00007961773A252E31660A000000E8
:10B970008011002084110020881100208C110020EB
:10B9800070697463684368616E6765526174653A93
:10B99000252E31660A000000726F6C6C4368616E80
:10B9A0006765526174653A252E31660A0000000011
:10B9B0007961774368616E6765526174653A252ED7
:10B9C00031660A000000F03F901100202DE9FC5F75
:10B9D00083460C462046F7F741FC07460C4A0D4BC0
:10B9E000F7F7FCFA81468A465846F7F737FC0746D0
:10B9F000094A0A4BF7F7F2FA4A465346CDE90001E5
:10BA0000F7F745FA0546F7F76DFCBDE8FC9F000027
:10BA1000989999999999B93FCDCCCCCCCCCCEC3FA5
:10BA2000FBF796FAFDF768FAFDF73CFAFCF704FF1E
:10BA3000FCF76AFEFCF7A0FFFCF7D4FFFDF72CF83B
:10BA4000FDF746F8FDF704F80548FAF761FC00F049
:10BA5000BBF9FCF789FE00F0D7F900BFFEE7000054
:10BA600004130020F0B50B30154D20F00701002421
:10BA7000144A0FE003688B420BD38B4205D95E1A40
:10BA800043184768C3E9006700E04368136002C0D9
:10BA900004E0021D10680028ECD12046002802D1E5
:10BAA000286808B10020F0BD064A07481060074A20
:10BAB000121A22F00702C0E9002401202860D7E70B
:10BAC0002C12002028120020846C0020807C002092
:10BAD00030B502460B464FF6FF70002110E0545C73
:10BAE0006040082409E000F0010525B140104AF249
:10BAF0000105684000E04010641E002CF3D1491C91
:10BB00009942ECDB30BD0000F8B504460F461646FE
:10BB10002C4890F8240010B94FF0FF30F8BD2948A8
:10BB2000807A10B94FF0FF30F8E7264A1268917A10
:10BB3000244A526810786B460222FFF7C5F910B10B
:10BB40004FF0FF30EAE79DF801009DF8001040EA51
:10BB50000125A54203DA00203070401EDEE71948B7
:10BB600040684088B5EB600F17DD164A1268517CBB
:10BB7000144A526810786B460122FFF7A5F910B1FC
:10BB80004FF0FF30CAE79DF8000000F0100020B130
:10BB900000F01AF86FF00100C0E7E2B2094B1B6831
:10BBA000D97A084B5B6818783B46FFF78DF910B1DE
:10BBB0004FF0FF30B2E795FBF4F0401E30700020EC
:10BBC000ACE700004011002008B57048807A10B939
:10BBD0004FF0FF3008BD002000906C4A1268D17B06
:10BBE0006A4A526810786B460122FFF7B2F910B129
:10BBF0004FF0FF30EEE7654A12685179634A5268A8
:10BC000010786B460122FFF7A4F910B14FF0FF3016
:10BC1000E0E75E4A126811795C4A526810786B4618
:10BC20000122FFF796F910B14FF0FF30D2E75748E5
:10BC300090F82400002853D00C200090534A12683A
:10BC40001179524A526810786B460122FFF781F948
:10BC500010B14FF0FF30BDE73220FAF7C9FEC02027
:10BC600000904A48807A00F0010020B19DF8000061
:10BC700040F020000090454A12681179434A52680A
:10BC800010786B460122FFF764F910B14FF0FF30D6
:10BC9000A0E73E48407C10B10220009001E0002067
:10BCA00000903A4A1268D17B384A526810786B4645
:10BCB0000122FFF74EF910B14FF0FF308AE7002064
:10BCC0000090324A12685179304A526810786B46B7
:10BCD0000122FFF73EF9002855D04FF0FF3079E7F9
:10BCE00004200090294A12681179284A5268107875
:10BCF0006B460122FFF72DF910B14FF0FF3069E7D5
:10BD00002248807C20B92148807A00F0010010B9D7
:10BD10004020009001E0602000901C4A12681179D8
:10BD20001A4A526810786B460122FFF712F910B1D7
:10BD30004FF0FF304EE73220FAF75AFE1348407CAE
:10BD400010B10120009001E0002000900F4A12681D
:10BD5000D17B0E4A526810786B460122FFF7F9F842
:10BD600010B14FF0FF3035E7084A12685179074AA1
:10BD700052681078054B10330122FFF7EAF810B132
:10BD80004FF0FF3026E7002024E70000401100209C
:10BD900070B50546FDF729FE48B9FDF729FE30B913
:10BDA00008480068022805D1FDF71CFE10B16FF0AD
:10BDB000050404E0002415B1284603F053FE204694
:10BDC00070BD00000C11002010B5FDF70EFE48B943
:10BDD000FDF70EFE30B90B480068022805D1FDF7CB
:10BDE00001FE10B16FF0050409E00648006820B9B3
:10BDF000012004490860002401E04FF0FF34204690
:10BE000010BD00000C11002010B5FDF7EEFD48B983
:10BE1000FDF7EEFD30B90C480068022805D1FDF7AA
:10BE2000E1FD10B16FF005040CE00748006801283F
:10BE300006D102200449086003F0F8FE002401E066
:10BE40004FF0FF34204610BD0C1100202DE9F041C9
:10BE500004460D4624F0010604F001080027FDF712
:10BE6000C4FD48B9FDF7C4FD30B916480068022882
:10BE700005D1FDF7B7FD10B16FF005071FE016B94A
:10BE80006FF003071BE0B8F1000F0CD029463046D5
:10BE900004F022FD012812D015B16FF001070EE069
:10BEA0006FF002070BE02946304604F039FC012808
:10BEB00005D015B16FF0010701E06FF002073846B9
:10BEC000BDE8F0810C1100202DE9F0470446002662
:10BED000FDF78BFD002859D1FDF78AFD002855D1CB
:10BEE0002C480068022803D1FDF77CFD00284DD1C5
:10BEF0000CB1676800E0002707F0010008B10125D8
:10BF000000E0002507F0080008283FD04FF0FF3878
:10BF100074B1A06828B1E068502802D34FF001083E
:10BF200008E0A06830B9E06820B94FF0000801E0EF
:10BF30004FF00008B8F1010F0CD12DB10420A16819
:10BF400004F0C7F8064612E00120A16804F0C1F829
:10BF500006460CE0B8F1000F09D125B1042004F029
:10BF6000A7F8064603E0012004F0A2F806464EB109
:10BF700014B1D4F8009001E04FF000094946304672
:10BF800003F002FD16B10DB146F001063046BDE8E2
:10BF9000F08700000C1100202DE9F041044624F048
:10BFA000010504F001070026FDF71FFD48B9FDF764
:10BFB0001FFD30B911480068022805D1FDF712FDB8
:10BFC00010B16FF0050616E015B96FF0030612E028
:10BFD0003FB1284604F0CCFA01280CD06FF00206DD
:10BFE00009E000231A461946284604F071F9012891
:10BFF00001D06FF002063046BDE8F0810C11002040
:10C000002DE9F84305460F4614464FF00008FDF7AA
:10C01000ECFC002864D1FDF7EBFC002860D132482D
:10C020000068022803D1FDF7DDFC002858D1002D5F
:10C0300056D0AF4254D84FF0FF3664B1A06820B15B
:10C04000E068502801D3012606E0A06820B9E06826
:10C0500010B9002600E00026701C70B3012D23D11A
:10C06000012E09D103200090002211460120A3686F
:10C0700004F073F8804605E003220021012004F05B
:10C080003DF88046B8F1000F1DD0E7B100231A46F5
:10C090001946404604F01CF9012814D0404603F02C
:10C0A00089FC4FF000080EE0012E07D139462846E2
:10C0B000A26803F0CBFF804605E011E03946284630
:10C0C00003F096FF8046B8F1000F09D014B1D4F800
:10C0D000009001E04FF000094946404603F054FC4F
:10C0E0004046BDE8F88300000C1100202DE9F04720
:10C0F00086B080468946144600200490FDF775FC02
:10C1000000285DD1FDF774FC002859D12D48006846
:10C11000022803D1FDF766FC002851D1B8F1000FC9
:10C120004ED080261825002005900DF1140A471ED8
:10C1300044B3206808B1D4F800A0A06900B1A56993
:10C140002DB1382D03D8207900F0010018B100205E
:10C1500006B0BDE8F087606908B160698608A0682C
:10C1600040B1E068602805D3206918B1606908B162
:10C17000012708E0A06830B9E06820B9206910B94B
:10C18000002700E00027012F0CD12169A0684B4651
:10C190003246CDE9005102905146404604F03CFC45
:10C1A00004900DE067B904A8B2B24B465146CDE900
:10C1B0000050404604F0FEFB012801D0002004900E
:10C1C0000498C5E70C1100202DE9FE4F064689466C
:10C1D00092461C4600200290FDF707FC002851D132
:10C1E000FDF706FC00284DD128480068022803D13D
:10C1F000FDF7F8FB002845D1002E43D0082002F0BF
:10C200009BFE0546002D3DD02E60C5F804A0B9F177
:10C21000000F01D1002700E001274FF0FF384FF059
:10C22000000B94B1206808B1D4F800B0A06828B120
:10C23000E068302802D34FF0010808E0A06830B968
:10C24000E06820B94FF0000801E04FF00008B8F1B5
:10C25000010F0BD10E49A0682B463A46CDE90010DC
:10C260000121584604F081FE02900BE0B8F1000F66
:10C2700008D107482B463A4601210090584604F061
:10C2800059FE02900298BDE8FE8F00000C110020BC
:10C29000C190000870B504460D46094E052D02DB1D
:10C2A0006078032805D007A0FDF72CFB4FF0FF3086
:10C2B00070BD2079E17840EA012030800020F7E766
:10C2C0000C6C0020526573706F6E736520746F6F15
:10C2D0002073686F7274206F722066756E63746964
:10C2E0006F6E20636F6465206D69736D6174636840
:10C2F000210A00002DE9F04104460F46082F02D123
:10C300006078102806D00BA0FDF7FCFA4FF0FF3044
:10C31000BDE8F081E078A17840EA012560792179D3
:10C3200040EA01263246294610A0FDF7EBFA00202C
:10C33000EEE70000526573706F6E7365206C656E7A
:10C34000677468206D69736D61746368206F722013
:10C3500066756E6374696F6E20636F6465206D69C6
:10C36000736D61746368210A00000000577269747C
:10C3700074656E20746F20737461727420616464DC
:10C38000726573733A2025642C206E756D62657238
:10C39000206F66207265676973746572733A202531
:10C3A000640A000070B504460D4600262946204662
:10C3B000FEF744FF20B10CA0FDF7A4FA701E70BD7B
:10C3C0006678032E02D0102E0AD104E029462046BA
:10C3D000FFF760FF05E029462046FFF78BFF00E0EE
:10C3E00000BF00BF0020EAE7435243206368656353
:10C3F0006B206661696C6564210A000030B589B004
:10C4000004460422214607A8F6F753FB00208DF8C6
:10C4100020000222211D06A8F6F74BFB00208DF814
:10C420001A000222A11D05A8F6F743FB00208DF893
:10C430001600022204F1080104A8F6F73AFB0020D6
:10C440008DF81200022204F10A0103A8F6F731FB6D
:10C4500000208DF80E00022204F10C0102A8F6F76C
:10C4600028FB00208DF80A0007A8F6F73BFC2449BA
:10C47000488006A8F6F736FC2149087105A8F6F7AA
:10C4800031FC1F49487104A8F6F72CFC1C4988713F
:10C4900003A8F6F727FC1A49C87102A8F6F722FC90
:10C4A000174908720846007AC979154DCDE9001080
:10C4B000AB796A7929796888F8F7F8FD1149C8607D
:10C4C0002846418810A0FDF71DFA2846017912A0E0
:10C4D000FDF718FA2846417914A0FDF713FA28460B
:10C4E000817916A0FDF70EFA2846C17917A0FDF74D
:10C4F00009FA2846017A1AA0FDF704FA09B030BDFE
:10C500001413002034120020596561722028696ECE
:10C5100074293A2025640A004D6F6E7468202869DA
:10C520006E74293A2025640A0000000044617920D5
:10C5300028696E74293A2025640A0000486F7572D4
:10C540002028696E74293A2025640A004D696E75A9
:10C5500074652028696E74293A2025640A00000059
:10C560005365636F6E642028696E74293A202564D0
:10C570000A0000002DE9F74F81468A46B9F1000F05
:10C5800005D137A0FDF7BEF90020BDE8FE8F3AA126
:10C590004846FEF7B3FD044614B1E068052804D010
:10C5A00038A0FDF7AFF90020EFE741A14846FEF7BC
:10C5B000A5FD8046B8F1000F02D0E068052804D040
:10C5C0003EA0FDF79FF90020DFE72046FEF78DFD36
:10C5D00005464046FEF789FD0646B54201D1C82D05
:10C5E00004DD41A0FDF78EF90020CEE7002716E01C
:10C5F00039462046FEF770FD8346BBF1000F03D09D
:10C60000DBF80C00032804D045A0FDF77BF90020DF
:10C61000BBE70AEBC702DBE9060103C27F1CAF429E
:10C62000E6DB002718E039464046FEF755FD834615
:10C63000BBF1000F03D0DBF80C00032804D042A0AC
:10C64000FDF760F90020A0E7DBE90621029800EB86
:10C65000C700C0E900217F1CB742E4DB012094E75A
:10C66000526F6F74206F626A656374206973204E25
:10C67000554C4C0A00000000706F6C79676F6E4C6F
:10C6800061740000706F6C79676F6E4C6174206923
:10C6900073206E6F7420616E206172726179206FF9
:10C6A00072206973206D697373696E670A000000F8
:10C6B000706F6C79676F6E4C6F6E0000706F6C7985
:10C6C000676F6E4C6E67206973206E6F7420616EA9
:10C6D000206172726179206F72206973206D6973B5
:10C6E00073696E670A000000417272617920736994
:10C6F0007A6573206D69736D61746368206F722051
:10C70000657863656564206D6178696D756D20611C
:10C710006C6C6F7765642073697A650A00000000AD
:10C720004C6174206974656D206973206E6F74208C
:10C7300061206E756D626572206F72206973206D65
:10C74000697373696E670A004C6E67206974656D62
:10C75000206973206E6F742061206E756D62657242
:10C76000206F72206973206D697373696E670A00A8
:10C7700070B505460C460EA12846FEF7BFFC0446E0
:10C780001CB90EA0FDF7BEF810E014A06169FDF71A
:10C79000B9F86069012806D1144981F8DC0014A0B9
:10C7A000FDF7B0F802E01BA0FDF7ACF870BD00008B
:10C7B000726573756C74436F646500004669656CDF
:10C7C000642022726573756C74436F646522206EF9
:10C7D0006F7420666F756E640A0000007265737571
:10C7E0006C74436F64653A2025640A00341200209B
:10C7F0004C6F67696E20726573706F6E736520642D
:10C80000617461207375636365737366756C6C79AD
:10C810000A0000004C6F67696E20726573706F6E5E
:10C82000736520686173206661696C65640A000045
:10C830002DE9F04705460C4620785B2804D02648B1
:10C8400004600020BDE8F0870520E860601C02F06D
:10C850004DFD044620785D2801D1601CF2E7FEF70B
:10C860005DFC0646A860A86808B90020EAE72046F3
:10C8700002F03CFD80464146304600F007FB07468B
:10C8800002F034FD04460CB90020DBE717E0FEF7A8
:10C8900045FC071E00D1D5E737607E603E46601C30
:10C8A00002F024FD81464946304600F0EFFA80460A
:10C8B00002F01CFD04460CB90020C3E700BF20783D
:10C8C0002C28E4D020785D2801D1601CBAE702480A
:10C8D00004600020B6E7000004100020014600229A
:10C8E0000878302806DB0878392803DC08783038E7
:10C8F000024415E00878412806DB0878462803DC66
:10C900000878373802440BE00878612806DB08789D
:10C91000662803DC08785738024401E0002070479D
:10C920001201491C0878302806DB0878392803DC16
:10C9300008783038024415E00878412806DB08788A
:10C94000462803DC0878373802440BE00878612871
:10C9500006DB0878662803DC08785738024401E0D3
:10C960000020DCE71201491C0878302806DB087833
:10C97000392803DC08783038024415E0087841286B
:10C9800006DB0878462803DC0878373802440BE0D9
:10C990000878612806DB0878662803DC08785738B1
:10C9A000024401E00020BAE71201491C087830284F
:10C9B00006DB0878392803DC08783038024415E0B3
:10C9C0000878412806DB0878462803DC08783738E1
:10C9D00002440BE00878612806DB0878662803DC4F
:10C9E00008785738024401E0002098E7104696E79F
:10C9F0002DE9F04F8BB083468A4600200446054659
:10CA00000026674F0021884689460990012008903A
:10CA10009AF800002D2802D1624F0AF1010A9AF813
:10CA20000000302801D10AF1010A9AF800003128EB
:10CA300022DB9AF8000039281EDC00BF1AF8011B1F
:10CA4000A1F13000F6F7B9FB0022574BCDE9060102
:10CA500020462946F6F7C2FACDE90401DDE90623AE
:10CA6000F6F715FA04460D469AF80000302803DB65
:10CA70009AF800003928E1DD9AF800002E2830D11C
:10CA80009AF8010030282CDB9AF80100392828DCBC
:10CA90000AF1010A00BF1AF8011BA1F13000F6F7F4
:10CAA0008CFB0022404BCDE9060120462946F6F7D3
:10CAB00095FACDE90401DDE90623F6F7E8F9044625
:10CAC0000D460022364B40464946F6F781FA80462D
:10CAD00089469AF80000302803DB9AF800003928CC
:10CAE000D9DD9AF80000652803D09AF8000045289F
:10CAF00023D10AF1010A9AF800002B2802D10AF189
:10CB0000010A08E09AF800002D2804D14FF0FF3008
:10CB100008900AF1010A08E01AF8010B3038099967
:10CB200001EB810100EB410009909AF800003028E8
:10CB300003DB9AF800003928EEDDDDE9082101FB6E
:10CB400002F0F6F73AFB42464B46CDE90001F6F714
:10CB50009EF902460B46CDE902010020124900F081
:10CB6000F3F922462B46CDE9060130463946F6F761
:10CB700035FACDE90401DDE90623F6F72FFA04467C
:10CB80000D46CBE9064520462946F6F748FBCBF88B
:10CB900014000320CBF80C0050460BB0BDE8F08F1A
:10CBA0000000F03F0000F0BF000024402DE9F047F6
:10CBB00006460C4620787B2804D0404804600020BC
:10CBC000BDE8F0870620F060601C02F08FFB044691
:10CBD00020787D2801D1601CF2E7FEF79FFA054618
:10CBE000B060B06808B90020EAE7204602F07EFB9A
:10CBF00080464146284600F063F8074602F076FB7F
:10CC000004460CB90020DBE728692862002028616F
:10CC100020783A2803D0294804600020D0E7601C1F
:10CC200002F064FB80464146284600F02FF9074693
:10CC300002F05CFB04460CB90020C1E731E0FEF7CE
:10CC40006DFA071E00D1BBE72F607D603D46601C7A
:10CC500002F04CFB81464946284600F031F88046F8
:10CC600002F044FB04460CB90020A9E728692862B9
:10CC70000020286120783A2803D010480460002062
:10CC80009EE7601C02F032FB81464946284600F0D0
:10CC9000FDF8804602F02AFB04460CB900208FE71D
:10CCA00000BF20782C28CAD020787D2801D1601CB4
:10CCB00086E702480460002082E70000041000209C
:10CCC0002DE9F05F8346884608F10104002798F8B3
:10CCD0000000222805D06A48C0F800800020BDE886
:10CCE000F09F04E014F8011B5C2900D1641C20783B
:10CCF000222804D0207810B1781C071EF2D1781CAD
:10CD00006049096888478146B9F1000F01D10020C8
:10CD1000E5E708F101044D469EE020785C2804D048
:10CD200014F8010B05F8010B96E0641C20787228BA
:10CD300018D006DC622809D066280BD06E287DD179
:10CD40000CE0742812D07528F9D113E0082005F8FA
:10CD5000010B7FE00C2005F8010B7BE00A2005F8B1
:10CD6000010B77E00D2005F8010B73E0092005F8B1
:10CD7000010B6FE0601CFFF7B1FD0646241DB6F500
:10CD80005C4F02D3B6F5604F00D306B962E0B6F54A
:10CD9000584F1CD3B6F55C4F19D260785C2802D18D
:10CDA000A078752800D055E0E01CFFF797FD82467B
:10CDB000A41DBAF55C4F02D3BAF5604F00D349E029
:10CDC000C6F30901504661F39F2000F58036042721
:10CDD000802E01D2012708E0B6F5006F01D20227AC
:10CDE00003E0B6F5803F00D203273D44012F20D059
:10CDF000022F15D0032F0AD0042F24D106F0BF0034
:10CE000040F08001681E05460170B60900BF06F0BB
:10CE1000BF0040F08001681E05460170B60900BFE2
:10CE200006F0BF0040F08001681E05460170B6099B
:10CE300000BF1548C05D3043C1B200E006E0681E87
:10CE40000546017000BF00BF3D4403E0207805F8AF
:10CE5000010B00BF00BF641C2078222803D020787B
:10CE600000287FF45AAF002028702078222800D1B3
:10CE7000641CCBF810900420CBF80C0020462EE761
:10CE80000410002008100020D810010870B50546D5
:10CE90000C460CB9002070BD042224A12046F5F7F1
:10CEA0002EFE18B90220E860201DF4E7052221A11A
:10CEB0002046F5F724FE18B90020E860601DEAE777
:10CEC00004221EA12046F5F71AFE20B90120E860D1
:10CED0006861201DDFE72078222804D121462846FA
:10CEE000FFF7EEFED7E720782D2805D020783028F0
:10CEF00007DB2078392804DC21462846FFF778FD37
:10CF0000C9E720785B2804D121462846FFF790FC2A
:10CF1000C1E720787B2804D121462846FFF746FE4A
:10CF2000B9E7084804600020B5E700006E756C6C36
:10CF30000000000066616C73650000007472756526
:10CF400000000000041000202DE9F04D1D460C46A5
:10CF500098B0174621F0004123F00043002814BF89
:10CF60004FF0010C4FF0000C0CEB440CFE4A0CEBA4
:10CF700002064FEA620C66452BD33E0018BF01261D
:10CF800006EB45061644F94A964222D3F84A53EA7C
:10CF9000070C02D0944205D148B918B000201146C0
:10CFA000BDE8F08D002808BF4FF0000C01D04FF015
:10CFB000010C0CEB440212F5001F0AD8002F14BF1D
:10CFC0004FF0010C4FF0000C0CEB450212F5001F66
:10CFD00007D918B03A462B462146BDE8F04DFCF77C
:10CFE0006ABD0022DFF88CA3002CB8BF534526DAB7
:10CFF000DFF884C36345A8BF022220DADFF870C3DC
:10D000009C451CDCDFF874C30CEB235CBCF1140FF3
:10D0100008DDCCF1340627FA06FC0CFA06F6BE420F
:10D020000DD108E05FB9CCF1140623FA06FC0CFA26
:10D0300006F69E4203D10CF00102C2F1020251EA4F
:10D04000000C19D1002D17DA002C18BF022A01D0CC
:10D05000012A07D00220FCF755FD18B0BDE8F04DBD
:10D06000FCF71EBD0220FCF74DFDFCF719FD18B0C2
:10D0700081F00041BDE8F08DB7F1000C6CD1534553
:10D0800025D104F1804212F5801201BF0028002052
:10D09000B74918B008BFBDE8F08DB548884207DC35
:10D0A000002DA1BF6046294618B0BDE8F08D07E00D
:10D0B000281E05DA80F0004118B06046BDE8F08D0A
:10D0C000AF497944D1E9000118B0BDE8F08DDFF82F
:10D0D000A0C2634525D1002D1FDA19B1514512D1E7
:10D0E000D8B909E0002840F0EC82A24A214618B0E5
:10D0F00062F31E01BDE8F08D0020214618B060F3F8
:10D100001E01BDE8F08D08DA18B02346BDE8F04DE9
:10D11000024600206146F5F7D3BF18B02146BDE8AE
:10D12000F08D514518DAB5F1804F0DD0A5F1005CB6
:10D13000BCF1FF5C10D1B4F1000C0DDB18B06146FE
:10D14000BDE8F04D02F0DBB8234618B00246BDE85A
:10D15000F04D1946F5F742BF060024F0004C3BD1D4
:10D16000D9B1514533D1002C06DD002DA1BF0020DF
:10D17000514618B0BDE8F08D002C01DD002D1BDB01
:10D18000002C13DA002D11DB012A4FF0000014BF30
:10D1900078497C4918B0BDE8F08D022A18BF002CF0
:10D1A0000AD0012A08D1002C06DA0AE0002CB8BF08
:10D1B000002D11DA012A04D0002018B00146BDE884
:10D1C000F08D18B000204FF00041BDE8F08DA1F1C6
:10D1D0004050B0F17F601AD0012000EBE47050EABB
:10D1E000020421D0624C521E4FF0000B104304BFCA
:10D1F0004FF0000B644C654883427CDD644A65480F
:10D2000093421FDD884217DB002D25DB37E0002C21
:10D2100000DA4AB1022A0CBF01204FF0FF3018B0EB
:10D22000BDE8F04DF5F7C9BF0120FCF76BFC18B065
:10D23000BDE8F04DFCF741BC4D4A8A4202DC002DAE
:10D240000ADC1CE0814202DA002D18DA04E0484BC7
:10D25000994220DD002D12DD0220FCF753FCFCF783
:10D2600032FC05460E460022534658462146F5F745
:10D27000B5FE18B066F31E012846BDE8F08D022009
:10D28000FCF740FCFCF726FC0A46214618B062F386
:10D290001E01BDE8F08D002230466146F5F798FE8C
:10D2A00080460E466FF00102F6F7AEF94FF05532A8
:10D2B000394BF5F790FE42463346F5F78FFE0022D4
:10D2C000364BF5F788FE82464246334604911046B7
:10D2D0001946F5F783FE5246049BF5F77FFE8A4612
:10D2E00000904FF0C0422E4B40463146F5F776FE97
:10D2F0002C4A2B4B00E027E0CDE90601514600986F
:10D30000F5F76CFE82460191274A284B404631468C
:10D31000F5F764FE5246019BF5F75AFE82460B462E
:10D3200002460591DDE90601F5F7B1FDDDE90623C9
:10D33000002688463046F5F74BFE5246059BF5F72A
:10D340004AFE024600F07EB90020B1F5801F07DAE0
:10D35000352230466146F6F757F906466FF034003D
:10D3600000EB215024E00000FFFF1F00FFFF0F0033
:10D370000000F03F0000F07F0000404301FCFFFF91
:10D380005A4300000000F0FF0000F0BF0000E04141
:10D390000000F043FFFFEF3F5555D53F0000E03F51
:10D3A0004715F73FFE822B6544DF5DF80BAE543E18
:10D3B000A0F2FF300190C1F3130040F07F6141F013
:10D3C00040510291FE498842D8BF002004DDFD494A
:10D3D0008142C8BF012001DD0D9008E000200D90C2
:10D3E0000198401C01900298A0F5801002900299CB
:10D3F000F54878440B910D9900EBC100D0E900236A
:10D400000F9330460A920B99F5F7E2FDCDE906013C
:10D41000DDE90A2130460F9BF5F739FD02460B4640
:10D420000020EA49F5F74CFE059102460B460090B4
:10D43000DDE90601F5F7D2FD1490E5488A464FF084
:10D44000000878440299006812904FF0005040EABA
:10D4500061010D980F9B01EB804000F500210991BF
:10D460000A9A1298F5F7B4FD32460B9BF5F7B3FD17
:10D4700042465346F5F7B2FD0646029140465146F4
:10D48000099B129AF5F7AAFDDDE90623F5F7A3FD3E
:10D490003246029BF5F79CFD059B009AF5F79EFD31
:10D4A0000091149A0490534610461946F5F796FDDC
:10D4B00006460246C7480B46029106217844FCF70F
:10D4C0009AFACDE90510029B324610461946F5F747
:10D4D00085FDDDE90532F5F781FD059106465346E8
:10D4E00040461946149AF5F7D2FC009B049AF5F7CA
:10D4F00075FD3246059BF5F7CAFCCDE9051042469D
:10D50000534610461946F5F769FD0022B24B0291C9
:10D510000A90F5F7BCFCDDE90532F5F7B8FC0E46DC
:10D520004246AD4B4046F5F753FD029B0A9AF5F78C
:10D530004FFDDDE90532F5F74EFD424602910A90B6
:10D54000334610465146F5F749FDCDE906015346ED
:10D55000149A02990A98F5F741FD8A4602903346DB
:10D56000424600990498F5F739FD5346029AF5F7BB
:10D570008EFC82460B4602460591DDE90601F5F771
:10D5800086FCDDE90623002088460646F5F720FDE7
:10D590005246059BF5F71FFD824609914FF0604208
:10D5A0008E4B30464146F5F719FD049006918C4AA2
:10D5B0008A4B50460999F5F711FD82460291894A36
:10D5C000894B30464146F5F709FD5246029BF5F777
:10D5D0005EFC864B7B440D9A03EBC203D3E9002328
:10D5E000F5F755FC0E9007910198F5F7E6FD0591CA
:10D5F000DDE9061382460E9A0498F5F748FC7C4A4A
:10D600007A440D9B02EBC303D3E9002300930292FB
:10D61000F5F73DFC5246059BF5F739FC0026884698
:10D6200052463046059BF5F7D3FC009B029AF5F76E
:10D63000CFFC069B049AF5F7CBFC079B0E9AF5F7F7
:10D64000CAFC024600200B46029038462946F5F7F0
:10D65000C5FC824601912B4638461946029AF5F7D9
:10D66000B7FC32464346F5F7B9FC5246019BF5F745
:10D670000EFC07468A463246434629460298F5F78D
:10D68000ADFC05460E463A465346F5F700FC594AAE
:10D690008846914221DBA8EB020353EA000210D135
:10D6A0002A463346F5F794FCCDE90401524A534B20
:10D6B00038465146F5F7EBFBDDE90423F5F7FAFDB3
:10D6C00021D20220FCF71EFAFCF7FDF90A4621469A
:10D6D00018B062F31E01BDE8F08D494B28F00042FE
:10D6E0009A4210D3474A08EB020353EA00027FF440
:10D6F000C6AD2A463346F5F76BFC3A465346F5F776
:10D70000D9FD7FF6BCAD0022019228F000403E49D1
:10D710003E4A01EB2051824223DA481C4FF480112B
:10D7200021FA00F040443A4AC0F30A517A44394B96
:10D73000A1F2FF31CB4020EA0303C0F3130040F411
:10D740008010C1F11401C84012680190B8F1000FB7
:10D75000BCBF4042019028463146F5F739FC0546EA
:10D760000E462A46334638465146F5F790FB4FF0B1
:10D7700000084246284B40460591F5F72FFCCDE9BD
:10D780000601264A264B40460599F5F727FC0091ED
:10D7900002902A46334640460599F5F719FC3A4669
:10D7A0005346F5F718FC1F4A1F4BF5F717FC009B73
:10D7B000029AF5F76CFB0746884602460B4635E0B1
:10D7C0008E9803007AB60B00823E00000000F03F06
:10D7D000DA3F0000E83D00000000084009C7EE3FC6
:10D7E000FD033ADCF5015B14E02F3EBEC03C0000B7
:10D7F000843C000000009040FE822B654715973C5A
:10D8000000CC904000346F3F01FCFFFF0000E03F80
:10D81000F03C0000FFFF0F00432EE63F396CA80CE0
:10D82000615C20BEEF39FAFE422EE63FDDE90601DB
:10D83000F5F72DFBDDE9062305460E46F5F7C8FB97
:10D840003A464346F5F7C7FB0F462A463346009053
:10D8500010461946F5F7C2FB824602462E48884616
:10D860000B4605217844FCF7C6F852464346F5F7C7
:10D87000B5FB2A463346F5F7AEFB80468A463B4663
:10D8800028463146009AF5F7A9FB3B46009AF5F782
:10D89000FEFA0691009000224FF080434046514628
:10D8A000F5F796FB0F460C90424653462846314604
:10D8B000F5F794FB3B460C9AF5F702FC069B009AA1
:10D8C000F5F786FB2A463346F5F782FB0022134B19
:10D8D000F5F781FB054601980E4601EB005108154E
:10D8E000002810DC28463146019AF5F78DFEFCF73A
:10D8F00045F8042808BFFCF7EDF828463146019AA0
:10D90000F5F782FE05460B4618B02A4658462146D2
:10D91000BDE8F04DF5F762BB703A00000000F03F43
:10D920000146491E41EA610141EAA10141EA211192
:10D9300041EA212141EA2141481C70472DE9FF4F6E
:10D9400085B092461E464FF0000B052003900598C7
:10D95000D0F80880D946002500200290019003E00D
:10D9600009F10109D8F80080B8F1000FF8D1B9F138
:10D97000000F16D12EB103213046FDF7B7FD8346C7
:10D9800004E003207E49096888478346BBF1000F05
:10D9900003D07CA15846F5F7A9F8584609B0BDE870
:10D9A000F08F002E57D0B56801213046FDF79EFD5F
:10D9B00004460CB90020F1E75B202070B068401CE1
:10D9C000B0600598D0F808802EE03346524606999C
:10D9D000491C404600F0A4FC304601F013FDB06045
:10D9E000D8F80000F0B1BAF1000F01D0022000E039
:10D9F000012003900399491C3046FDF777FD04464A
:10DA00000CB90020CAE72C2004F8010BBAF1000F72
:10DA100002D0202004F8010B00202070B168039888
:10DA20000844B060D8F80080B8F1000F02D0029826
:10DA30000028CAD002213046FDF758FD04460CB933
:10DA40000020ABE75D2004F8010B00202070306857
:10DA500000EB050B91E04FEA8900494909688847C6
:10DA600007460FB9002099E74FEA89013846F5F7D4
:10DA700003F80598D0F8088021E000235246069963
:10DA8000491C404600F04CFC049029466D1C04984B
:10DA900047F82100049870B10498F5F720F8801C2D
:10DAA000BAF1000F01D0012100E0002101440398E8
:10DAB0000844039001E001200290D8F80080B8F1FA
:10DAC000000F02D002980028D7D0029820B92C4924
:10DAD0000398096888478346BBF1000F01D10120F4
:10DAE0000290029890B1002508E057F8250020B177
:10DAF00057F825002449096888476D1C4D45F4DB1B
:10DB00003846214909688847002047E75B208BF8A1
:10DB100000000BF1010400202070002521E057F8DF
:10DB20002500F4F7DCFF019057F825102046019AF4
:10DB3000F4F789FF01980444A9F10100A8420AD032
:10DB40002C2004F8010BBAF1000F02D0202004F8B9
:10DB5000010B0020207057F825000B490968884701
:10DB60006D1C4D45DBDB38460749096888475D2059
:10DB700004F8010B002004F8010B58460EE70000E2
:10DB8000081000205B5D00000C1000202DE9FC4710
:10DB900082460E464FF00009DAE906450022134698
:10DBA00020462946F5F76EFB13D12EB102213046EF
:10DBB000FDF79CFC814604E002204A490968884739
:10DBC0008146B9F1000F03D047A00088A9F80000F2
:10DBD00084E0DAF81400F5F7F0FA074622462B46FF
:10DBE000F5F7F6F921F000410022404BCDE90001A4
:10DBF000F5F748FB23D83E4A3E4B20462946F5F729
:10DC000041FB1CD800223C4B20462946F5F752FB2D
:10DC100015D82EB115213046FDF768FC814604E089
:10DC200015203049096888478146B9F1000F55D061
:10DC300032A14846DAF81420FBF78CFE4EE02EB1F4
:10DC400040213046FDF752FC814604E04020254942
:10DC5000096888478146B9F1000F3FD02046294620
:10DC6000FDF7C6FC074622462B46F5F7B1F921F031
:10DC7000004100221D4BCDE90001F5F703FB0FD851
:10DC800025F0004127461E4A1E4B3846F5F7FAFAA2
:10DC900006D222462B461CA14846FBF75BFE1DE040
:10DCA00025F0004127461A4A1A4B3846F5F7EAFA9A
:10DCB00007D325F000410022174B3846F5F7FAFA52
:10DCC00006D222462B4615A14846FBF743FE05E047
:10DCD00022462B4612A14846FBF73CFE4846BDE8CB
:10DCE000FC87000008100020300000000000B03C5D
:10DCF0000000C0FFFFFFDF410000E0C1256400001D
:10DD000044F3C2E4E4E9634C252E306600000000D1
:10DD10008DEDB5A0F7C6B03E65CDCD4125650000BF
:10DD2000256600002DE9FF4F89B0884616461F463C
:10DD300000200890079006904FF0070A00250998E8
:10DD4000D0F80890002002900190009004E0029822
:10DD5000401C0290D9F80090B9F1000FF7D1029859
:10DD6000002835D157B116B108F1040000E00320B6
:10DD700001463846FDF7BAFB069009E016B108F1F6
:10DD8000040100E003210846EA4909688847069033
:10DD9000069818B900200DB0BDE8F08F069C7B20D6
:10DDA00004F8010B66B10A2004F8010B002503E01A
:10DDB000092004F8010B6D1CA8F10100A842F7DC52
:10DDC0007D2004F8010B002004F8010B0698E2E71F
:10DDD000002F77D0BD680EB1022000E001208246FE
:10DDE0000AF101013846FDF781FB04460CB9002019
:10DDF000D1E77B2004F8010B16B10A2004F8010BCF
:10DE000000202070B8685044B8600998D0F8089095
:10DE100008F1010868E0B6B141463846FDF766FBF7
:10DE200004460CB90020B6E70020039005E0092065
:10DE300004F8010B0398401C039003984045F6DB5F
:10DE4000B8684044B8603946D9F8200000F07EF93F
:10DE5000384601F0D7FAB8600EB1022000E0012088
:10DE6000824651463846FDF741FB04460CB9002076
:10DE700091E73A2004F8010B16B1092004F8010BD0
:10DE8000B8685044B8603B4632464146484600F0C8
:10DE900047FA384601F0B6FAB8600EB1012000E04A
:10DEA0000020D9F8001009B1012100E0002100EBA9
:10DEB000010A0AF101013846FDF718FB044614B9BE
:10DEC000002068E734E0D9F8000010B12C2004F8F5
:10DED000010B16B10A2004F8010B00202070B8686D
:10DEE0005044B860D9F80090B9F1000F93D116B141
:10DEF00008F1010000E0022001463846FDF7F6FA7D
:10DF000004460CB9002046E74EB1002503E0092085
:10DF100004F8010B6D1CA8F10100A842F7DC7D207C
:10DF200004F8010B00202070386828440690FEE0B9
:10DF3000029988007F49096888470890089808B9BD
:10DF4000002028E7029988007A49096888470790E5
:10DF5000079828B9784908980968884700201AE77F
:10DF6000029881000898F4F787FD029881000798CD
:10DF7000F4F782FD0998D0F8089008F1010806B17D
:10DF8000C2442EE00021D9F8200000F0DFF8049010
:10DF9000079941F82500002332464146484600F0E3
:10DFA000BFF929466D1C0590089A42F82100049893
:10DFB00098B1059888B10598F4F791FD83460498C7
:10DFC000F4F78DFD0BEB0001891C16B108F102007E
:10DFD00000E000200844824401E001200190D9F8CB
:10DFE0000090B9F1000FCDD1019820B950465149A8
:10DFF000096888470690069808B9012001900198A1
:10E0000018B3002514E0079850F8250028B10799A7
:10E0100051F82500484909688847089850F82500B4
:10E0200028B1089951F825004349096888476D1CB3
:10E0300002988542E7DB40490798096888473E49CE
:10E040000898096888470020A5E67B21069801709A
:10E050000698441C16B10A2004F8010B0020207019
:10E06000002548E05EB10020039005E0092004F897
:10E07000010B0398401C039003984045F6DB079979
:10E0800051F82500F4F72BFD0090079850F8251063
:10E090002046009AF4F7D7FC009804443A2004F88C
:10E0A000010B16B1092004F8010B089850F825104F
:10E0B0002046F4F71BFD089951F82500F4F70FFDF1
:10E0C00004440298401EA84202D02C2004F8010B00
:10E0D00016B10A2004F8010B00202070079951F8AE
:10E0E0002500154909688847089951F82500124903
:10E0F000096888476D1C02988542B3DB0E49079872
:10E10000096888470C490898096888474EB1002576
:10E1100003E0092004F8010B6D1CA8F10100A842DE
:10E12000F7DC7D2004F8010B002004F8010B0698B1
:10E1300031E60000081000200C10002070B50446E5
:10E140000D462946206900F001F870BD2DE9F05F09
:10E15000804689460027BB46454611E028780028BE
:10E1600002DD2878202805DB2878222802D02878AC
:10E170005C2801D1012000E0002040EA0B0B6D1C5F
:10E1800028780028EAD1BBF1000F22D1A5EB0807BF
:10E19000B9F1000F05D0F91C4846FDF7A7F906466E
:10E1A00004E0F81C584909688847064616B900205B
:10E1B000BDE8F09F3446222004F8010B414620467A
:10E1C000F4F794FC2220E0550021781C21543046BD
:10E1D000EEE7B8F1000F16D1B9F1000F05D0032119
:10E1E0004846FDF783F9064604E0032046490968DE
:10E1F000884706460EB90020DAE744A13046F4F716
:10E2000075FC3046D4E745460BE0514640A0F4F794
:10E210005CFC08B17F1C03E0BAF1200F00DA7F1D1F
:10E220006D1C95F800A0BAF1000F02D0781C071EF3
:10E23000EBD1B9F1000F05D0F91C4846FDF756F9AE
:10E24000064604E0F81C30490968884706460EB9BE
:10E250000020ADE734464546222004F8010B47E094
:10E2600028781F280ADD2878222807D028785C28FB
:10E2700004D015F8010B04F8010B39E05C2004F818
:10E28000010B15F8011B8A460C2919D006DC082958
:10E2900012D0092920D00A2922D115E00D2917D042
:10E2A000222905D05C291BD15C2004F8010B1EE05B
:10E2B000222004F8010B1AE0622004F8010B16E09A
:10E2C000662004F8010B12E06E2004F8010B0EE04A
:10E2D000722004F8010B0AE0742004F8010B06E038
:10E2E00052460DA12046FBF735FB641D00BF00BF61
:10E2F00028780028B4D1222004F8010B002004F86B
:10E30000010B304654E700000810002022220000D4
:10E31000225C080C0A0D09007525303478000000D5
:10E320002DE9F04104460F4690461D46002614B9DB
:10E330000020BDE8F081002D46D0207B072842D286
:10E34000DFE800F00F1A04252B313900052128469B
:10E35000FDF7CCF806461EB137A13046F4F7C6FBF0
:10E3600031E006212846FDF7C1F806461EB134A16A
:10E370003046F4F7BBFB26E005212846FDF7B6F84A
:10E3800006461EB130A13046F4F7B0FB1BE029462B
:10E390002046FFF7FBFB064615E029462046FFF71F
:10E3A000CDFE06460FE02B46424639462046FFF793
:10E3B000C5FA064607E02B46424639462046FFF797
:10E3C000B1FC064600BF34E0207B072830D2DFE8EE
:10E3D00000F0090E0413191F270017A0FCF718FFFF
:10E3E000064625E016A0FCF713FF064620E016A01F
:10E3F000FCF70EFF06461BE000212046FFF7C6FB98
:10E40000064615E000212046FFF798FE06460FE07D
:10E410000023424639462046FFF790FA064607E0B9
:10E420000023424639462046FFF77CFC064600BFE3
:10E4300000BF30467DE700006E756C6C0000000088
:10E4400066616C7365000000747275650000000001
:10E450002DE9F04105460E46164807681648006843
:10E46000001D01F07CF8681C38B936B1124801680B
:10E47000091D124801F0CAF81AE07C190E4800681C
:10E480004460BC4207D20C480168091D0C48006872
:10E4900001F0A2F80CE008480168091D094800686D
:10E4A00001F09AF808480068844201D206480460E6
:10E4B000BDE8F081C8100020B41000201034002006
:10E4C000BC100020B8100020E410002010B5044655
:10E4D00001F0A8F824480068401C2349086023483C
:10E4E000006840B9214804600846006801280DD141
:10E4F00000F086FA0AE01E48006838B91B48006838
:10E50000C06AE16A884201D8184804601948006866
:10E51000401C184908600846006860641649E06AB3
:10E520000968884202D91449E06A0860E16A01EB8F
:10E530008101124A02EB8100211D01F067F801F010
:10E540009BF80B48006868B108480068C06AE16A37
:10E55000884207D24FF0805009490860BFF34F8FBF
:10E56000BFF36F8F10BD0000C4100020B410002056
:10E57000D0100020E0100020CC100020602F0020E0
:10E5800004ED00E008B501F04DF812480068E8B964
:10E59000114801F011F8114801F00EF80E48104929
:10E5A00008600E480F49086000200F4B0F4A1021E9
:10E5B00000900A2001F0D1FD064908600846006875
:10E5C00020B10BA10348006801F0DEF901F054F816
:10E5D00008BD000000110020243400203834002041
:10E5E000F8100020FC1000204C3400209C34002047
:10E5F000546D72510000000010B516E001F012F8E1
:10E600000C48C068C468201D00F0A9FF0A480068D3
:10E61000401E0949086009480068401E0749086013
:10E6200001F02AF8204600F05EF80448006800284F
:10E63000E4D110BDFC330020C4100020C010002025
:10E6400070B504460D46206C70B1216CE06808443A
:10E65000E0606168E068884201D32068E060284695
:10E66000226CE168F4F7EFF970BD2DE9F041044642
:10E670000F4615464FF00008A66B206C40B9206885
:10E6800060BB606802F0E2FA80460020606025E02E
:10E690007DB93946226CA068F4F7D5F9216CA068E1
:10E6A0000844A060D4E90110884217D32068A06014
:10E6B00014E03946226CE068F4F7C5F9216CE06893
:10E6C000401AE0602168E068884203D2216C6068EB
:10E6D000401AE060022D01D106B1761E701CA063C5
:10E6E0004046BDE8F08110B5044694F85D0030B9AD
:10E6F000206B00F0DFFF204600F0DCFF1AE094F80A
:10E700005D00012803D1204600F0D4FF12E094F808
:10E710005D00022801D1012000E0002050B900BFB7
:10E72000502080F31188BFF34F8FBFF36F8F00BF6E
:10E7300000BFFEE710BD01464A6A22B10A6B1268AB
:10E74000C2F1380000E000207047000000210C4AB0
:10E75000126802B101210B4A1268D26A0AB1002084
:10E760000DE0094A1268012A01D9002007E009B129
:10E77000002004E0054A1268054B1B68D01A704758
:10E78000CC100020B4100020602F0020E4100020E6
:10E79000C81000200146084A126812680AB901220E
:10E7A00000E000220A600A6822B9034A1268D268AF
:10E7B000106800E000207047F810002030B54FF4DA
:10E7C0002053174800F007042CB1C01D20F00700AB
:10E7D000134C041B1B1B0246124C22600024114DDB
:10E7E0006C60D018083820F007000F4C206000241F
:10E7F0000D4D2D686C600C4D2D682C601146441A2F
:10E800004C60094C24680C60084D4C682C60084D25
:10E810004C682C604FF00044064D2C6030BD000069
:10E82000FC3B0020101100201811002020110020B6
:10E830001C1100202411002000BFFFF7DDFE194845
:10E840000068012807D94FF0805017490860BFF3CE
:10E850004F8FBFF36F8FFFF779FF0446022C20D351
:10E8600001F0C6FA1148006811490968884201D3CD
:10E87000012000E0002050B900BF502080F3118833
:10E88000BFF34F8FBFF36F8F00BF00BFFEE7FFF7EF
:10E890005DFF0446022C02D3204600F089FF02F0FF
:10E8A000C7FACAE7602F002004ED00E0E410002062
:10E8B000C810002010B504464CB1002060602060F4
:10E8C000E06000231A461946204601F001FD10BD04
:10E8D0002DE9F04106460D4617469846069C0DB9AF
:10E8E000246000E02760E66325640121204601F0F2
:10E8F000A3FC84F84C80BDE8F0812DE9F05F8246EE
:10E900000F4690469B460A9E0C9C4FEA8801A52222
:10E91000206BF4F7AAF8A8F10100216B01EB800944
:10E9200029F0070909F0070008B9012000E00020DC
:10E9300050B900BF502080F31188BFF34F8FBFF351
:10E940006F8F00BF00BFFEE7002507E0795D04F18F
:10E9500034004155785D00B902E06D1C102DF5D3EF
:10E9600000BF002143200155382E00D33726E66230
:10E97000E66400202065201D00F02BFE04F1180045
:10E9800000F027FE2461C6F13800A0616462002017
:10E990006065A06584F85C005A465146484600F020
:10E9A0008FFB20600B9808B10B980460BDE8F09FC6
:10E9B0002DE9F04706460D4617469846DDE90894CE
:10E9C0000DB1012000E0002050B900BF502080F3BD
:10E9D0001188BFF34F8FBFF36F8F00BF00BFFEE7FB
:10E9E0005CB1FFF7CFFD2660A561E761C4F8208028
:10E9F000C4F82490201D00F0ECFDBDE8F087000075
:10EA000010B5002407E004EB84010F4A02EB8100FB
:10EA100000F0D2FD641C382CF5D30C4800F0CCFD7E
:10EA20000B4800F0C9FD0B4800F0C6FD0A4800F095
:10EA3000C3FD0A4800F0C0FD0448094908600448C5
:10EA40000849086010BD0000602F0020C03300207E
:10EA5000D4330020E8330020FC33002010340020A1
:10EA6000B8100020BC10002010B50146164800E088
:10EA7000006803688B42FBD30246436813448B4211
:10EA800004D143684C682344436001460A464B68FE
:10EA900013440468A34211D10C4C03682468A342B8
:10EAA00008D04B680468646823444B6003681B68A3
:10EAB0000B6005E0054B1B680B6001E003680B6011
:10EAC000884200D0016010BD1011002018110020F4
:10EAD0002DE9F04104460D4616461F464FF000084A
:10EAE00065602461B5420CD8F01BA169884202D34D
:10EAF0004FF0010811E0211D0948006800F06CFD8D
:10EB00000BE0BE4204D2BD4202D34FF0010804E044
:10EB1000211D0448006800F05FFD4046BDE8F0811B
:10EB2000FC100020F810002070B5054600F07AFDBA
:10EB3000A86B08B9012400E0002400F09DFD2046E8
:10EB400070BD70B5054600F06DFDA86BE96B88429D
:10EB500001D1012400E0002400F08EFD204670BDAC
:10EB6000F8B505460F4616480068C068C468201D01
:10EB700000F0F5FCE06901281DD1A06941192B4680
:10EB80003A462046FFF7A4FFA8B1002003462A46D4
:10EB900001460090204602F05DFA064656B900BFD5
:10EBA000502080F31188BFF34F8FBFF36F8F00BFEA
:10EBB00000BFFEE700BF2046616A8847F8BD00003D
:10EBC000F8100020F0B587B082E00398002811DA31
:10EBD00004AE56B900BF502080F31188BFF34F8FA9
:10EBE000BFF36F8F00BF00BFFEE7D6E90020B1681A
:10EBF000904700BF039800286ADB059C606908B94C
:10EC0000012000E0002010B9201D00F0A8FC02A89F
:10EC100000F0C0F8054603980A2857D2DFE800F054
:10EC200009050731334F0608323400BF00BF00BF6B
:10EC300000BF0498A269811803462A462046FFF7C0
:10EC400047FFE8B12046616A8847E069012817D18B
:10EC5000002000900498A16942180023194620461C
:10EC600002F0F8F9074657B900BF502080F3118829
:10EC7000BFF34F8FBFF36F8F00BF00BFFEE700BF32
:10EC800025E000BF23E000BF0498A061A06908B19F
:10EC9000012000E0002050B900BF502080F311880F
:10ECA000BFF34F8FBFF36F8F00BF00BFFEE7A069B8
:10ECB00041192B462A462046FFF70AFF07E094F841
:10ECC0002C0010B9204600F0F5FC00E000BF00BFAA
:10ECD000002203A90448006801F06EFC00287FF4BC
:10ECE00074AF07B0F0BD000000110020F8B5054674
:10ECF0000C4601F07DF8684600F04CF80646009896
:10ED000020BB44B9B54206D802F092F831462846F5
:10ED1000FFF726FF1CE03CB10E480068006808B908
:10ED2000012000E000200446A91B22460A48006892
:10ED300000F072FE02F07CF850B94FF080500749A5
:10ED40000860BFF34F8FBFF36F8F01E002F070F8E0
:10ED5000F8BD0000FC1000200011002004ED00E0D0
:10ED60000A490968096809B9012100E0002121B1B7
:10ED70004FF0FF31064A116006E004490968C9688E
:10ED8000C868034A4168116070470000B81000204D
:10ED9000E410002070B5044601F0B0FE05460748B7
:10EDA0000068854204D200F00BF80120206001E0E9
:10EDB0000020206001480560284670BD0811002031
:10EDC0002DE9F84332E024480068C068056822480D
:10EDD0000068C068C468201D00F0C1FB2046616A5D
:10EDE0008847E069012821D1A0694619AE4207D9B8
:10EDF00066602461211D1848006800F0EDFB15E0F5
:10EE0000002003462A4601460090204602F022F9DF
:10EE1000074657B900BF502080F31188BFF34F8FCA
:10EE2000BFF36F8F00BF00BFFEE700BF0A48006856
:10EE3000006808B9012000E000200028C3D006487F
:10EE4000D0F8008005480068034908600348C0F80E
:10EE50000080BDE8F8830000F8100020FC100020BE
:10EE60000E480068401C08B9012000E0002050B99D
:10EE700000BF502080F31188BFF34F8FBFF36F8F17
:10EE800000BF00BFFEE700BF502080F31188BFF332
:10EE90004F8FBFF36F8F00BF00BFFEE72811002028
:10EEA00008B500BF6846FFF775FC04462046009988
:10EEB000FFF71CFFFFF786FEF4E770B5044600F08D
:10EEC000B1FB94F9455010E0606A08B9012000E0F8
:10EED000002038B904F1240001F05CFF18B100F003
:10EEE000FBFD00E003E0681E45B2002DECDC00BF36
:10EEF000FF2084F8450000F0BFFB00F093FB94F97D
:10EF0000445010E0206908B9012000E0002048B911
:10EF100004F1100001F03EFF08B100F0DDFD681EB5
:10EF200045B200E001E0002DECDC00BFFF2084F8DA
:10EF3000440000F0A1FB70BD2DE9F04104464FF004
:10EF4000000800F055FF4648006808B9FFF736FC96
:10EF500044480068204000286BD1D4B1083404F044
:10EF60000700B0B104F00700C0F10800044404F049
:10EF7000070008B9012000E0002050B900BF502070
:10EF800080F31188BFF34F8FBFF36F8F00BF00BFB7
:10EF9000FEE7002C4DD034480068844249D8334EF7
:10EFA0003046056801E02E462D686868A04202D20E
:10EFB00028680028F7D12A480068854239D030688F
:10EFC00000F10808286830606868001B102819D90B
:10EFD0002F1907F0070008B9012000E0002050B900
:10EFE00000BF502080F31188BFF34F8FBFF36F8FA6
:10EFF00000BF00BFFEE76868001B78606C603846A1
:10F00000FFF732FD184968680968081A1649086050
:10F010000846006816490968884203D21248006809
:10F02000134908600F496868096808436860002050
:10F03000286001F0FDFE08F0070008B9012000E09B
:10F04000002050B900BF502080F31188BFF34F8FCC
:10F05000BFF36F8F00BF00BFFEE74046BDE8F08101
:10F0600018110020241100201C1100201011002074
:10F07000201100200648006830B10549096801F1F7
:10F080005000096D491C016001480068704700008C
:10F09000B410002070B50446254654B900BF502076
:10F0A00080F31188BFF34F8FBFF36F8F00BF00BF96
:10F0B000FEE700F0B7FA2E6A00F0DEFA304670BDC7
:10F0C000001F4FF080730360001F21F001030360F5
:10F0D000001F034B036014380260203870470000A3
:10F0E00061EE00082DE9F0438FB0002500240026D2
:10F0F000342102A8F3F7C0FCFBF7ABFF05463FA0A5
:10F10000FBF7B0FF07463A463EA12846FBF76EFFE5
:10F110003E48FBF7A7FF07463A463DA12846FBF7C6
:10F1200065FF3DA0FBF79EFF07463A463CA12846F7
:10F13000FBF75CFF3DA0FBF795FF07463A463DA174
:10F140002846FBF753FF31484C38D0F8D8000090E0
:10F150002E484C38D0F8D43039A1D0F8D02002A8AD
:10F16000FAF7F8FB02A8FBF77DFF07463A4636A1FF
:10F170002846FBF73BFF36A0FBF774FF07463A46ED
:10F1800036A12846FBF732FF35A0FBF76BFF074699
:10F190003A4635A12846FBF729FF1C494C39C86877
:10F1A000F4F71CF80746FBF742FF81464A4632A1B6
:10F1B0002846FBF71BFF00203149FBF738FF0746C5
:10F1C0003A4630A12846FBF711FF2846FBF7F0FF2F
:10F1D00004462846FBF754FF2046F3F780FC87B22D
:10F1E0003A46214629A0F6F733F806462046FCF7B2
:10F1F0007BFA30460FB0BDE8F08300006A736F6E93
:10F20000000000006D736754797065008012002063
:10F21000696D73690000000056312E300000000057
:10F220006861726456657273696F6E005631303072
:10F2300031000000736F667456657273696F6E00FB
:10F2400025782578257800006465764964000000FB
:10F25000355874324171384A62394C0076696E0013
:10F2600056322E300000000070726F746F636F6C46
:10F2700056657273696F6E0074786E4E6F00000091
:10F28000000010406465765479706500746F5365B2
:10F29000727665722F6D7174742F363034000000F1
:10F2A0002DE9F04105460C4616462F46B4460BB1F3
:10F2B0009C4202D20020BDE8F081002211E0002132
:10F2C00007E05018385C1CF80180404500D002E08F
:10F2D000491C9942F5D300BF994201D1B818EAE719
:10F2E000521CE01A9042EAD20020E4E700E0401C01
:10F2F00020B1017811B101782029F8DD70472DE99E
:10F30000F04106460F46F4F796F9041E0D4618BF65
:10F310000120284320F00040C0F17F6000F1E04070
:10F32000C00F0ED0301C18BF0120384320F0004021
:10F33000C0F17F6000F1E040C00F04BF0120FAF788
:10F34000E1FB20462946BDE8F08101604860704736
:10F3500010B50024F9F7F2F8F5F764F9094890F8C8
:10F36000530050B12720F7F787FE0748006800F0E8
:10F37000DBFCC820FCF70CFD03E04FF47A70FCF7CF
:10F3800007FD10BD101000208010002070B50D4C3E
:10F390000025F6F78BFA0C48007801280ED10B48AF
:10F3A00090F85300012809D0FCF712FA18B108A010
:10F3B000FAF7A8FA02E00DA0FAF7A4FA6420FCF725
:10F3C000E7FC70BD34120020001000201010002057
:10F3D0005468652076656869636C6520697320747C
:10F3E00075726E696E672E0D0A00000056656869B9
:10F3F000636C65206E6F74207475726E696E672E13
:10F400000D0A000070B504460CB1206808B9002050
:10F4100070BDA168206845182846F3F760FBA16815
:10F420000844F5E72DE9F04703460F464FF0000C7E
:10F43000E04619889878DC781E79F51901280BD0F8
:10F44000032809D0052807D0072805D0082803D0AD
:10F450000A2801D00C282ED14FF01F0C4FF01E08A7
:10F46000032821D14FF4C87991FBF9FA09FB1A1945
:10F47000B9F1000F13D04FEAE17901EB99794FEA26
:10F48000A909A1EB8909B9F1000F0BD14FF064096B
:10F4900091FBF9FA09FB1A19B9F1000F02D04FF0EC
:10F4A0001D0801E04FF01C08082801D0012833D1C5
:10F4B0004FF01F0830E0042805D0062803D00928A3
:10F4C00001D00B2804D14FF01E0C4FF01F0823E091
:10F4D0004FF01F084FF4C87991FBF9FA09FB1A198C
:10F4E000B9F1000F13D04FEAE17901EB99794FEAB6
:10F4F000A909A1EB8909B9F1000F0BD14FF06409FB
:10F5000091FBF9FA09FB1A19B9F1000F02D04FF07B
:10F510001D0C01E04FF01C0C182D0ADB183D641C7B
:10F52000644506DDA4EB0C04401C0C2801DD0C38FE
:10F53000491C002D09DA1835641E012C05DA4446F1
:10F54000401E012801DA0C20491E11809070D470F1
:10F5500015715E7956719E799671BDE8F087014606
:10F560000A69D1E901309860D1E901035860506817
:10F57000884201D188685060002008611068401EF0
:10F580001060106870470000034B0360034B0B6072
:10F5900080231360704700003C3500209C3500201C
:10F5A000034B0360034B0B604FF480731360704791
:10F5B0009C370020FC37002000F1080141604FF02B
:10F5C000FF31816000F10801C1600161002101602B
:10F5D000704700210161704710B502460B685C1C42
:10F5E0000CB9106907E002F1080000E040684468C7
:10F5F00024689C42FAD944684C604C68A1608860D9
:10F6000041600A611468641C146010BD42684A605D
:10F6100093688B60936859609160086103685B1C14
:10F620000360704700BF502080F31188BFF34F8FF5
:10F63000BFF36F8F00BF0E480068401C0C49086084
:10F6400008460068012812D10A480068C0B208B90B
:10F65000012000E0002050B900BF502080F3118845
:10F66000BFF34F8FBFF36F8F00BF00BFFEE7704740
:10F670002811002004ED00E00D48006850B900BFDB
:10F68000502080F31188BFF34F8FBFF36F8F00BFFF
:10F6900000BFFEE706480068401E054908600846AE
:10F6A000006820B9002080F3118800BF00BF7047B8
:10F6B0002811002070B506463546002E3FD0083D83
:10F6C0002C461F4960680968084008B1012000E025
:10F6D000002050B900BF502080F31188BFF34F8F36
:10F6E000BFF36F8F00BF00BFFEE7206808B901209D
:10F6F00000E0002050B900BF502080F31188BFF314
:10F700004F8FBFF36F8F00BF00BFFEE70C496068EB
:10F710000968084098B1206888B909496068096893
:10F720008843606000F064FB06496068096808442B
:10F73000044908602046FFF797F901F079FB70BD96
:10F74000241100201C110020154800684FF47A7124
:10F75000B0FBF1F013490860084600686FF07F4184
:10F76000B1FBF0F0104908600D480068B0FBF0F004
:10F770002D21B1FBF0F00D49086000204FF0E02191
:10F7800008618861064800684FF47A71B0FBF1F0B7
:10F79000401E4FF0E02148610720086170470000DB
:10F7A000B01000202C110020301100203411002056
:10F7B00071B581B0534901980968884202D951480E
:10F7C000006801904FF0E020006920F001004FF048
:10F7D000E0210861084681690198401E4A4A126882
:10F7E00002FB001449480068844202D94748006877
:10F7F000241A72B6BFF34F8FBFF36F8FFBF758FE1B
:10F8000080B94FF0E02080694FF0E0214861084660
:10F81000006940F0010008613B480068401E4861F3
:10F8200062B66DE04FF0E020446100204FF0E0212F
:10F8300088610846006940F0010008610198009065
:10F840006846F9F71AFB009820B1BFF34F8F30BF1D
:10F85000BFF36F8F01A8F9F70FFB62B6BFF34F8FAD
:10F86000BFF36F8F72B6BFF34F8FBFF36F8F06205A
:10F870004FF0E02108610846006900F48030C0B113
:10F8800021490968491E4FF0E0229269A21A881A9C
:10F890001E490968884203D31B490968884202D976
:10F8A00019490968481E4FF0E021486101994D1E31
:10F8B00013E015490198096848434FF0E021896930
:10F8C000461A11480068B6FBF0F5681C0E49096835
:10F8D0004843801B4FF0E021486100204FF0E021B9
:10F8E00088610846006940F001000861284600F080
:10F8F000FBF905480068401E4FF0E021486162B600
:10F900007CBD0000301100202C110020341100209B
:10F9100070B5F3F75FF80446102C16D304F1E0201D
:10F9200090F8F05315480078854201DB012000E093
:10F93000002050B900BF502080F31188BFF34F8FD3
:10F94000BFF36F8F00BF00BFFEE70D48006800F4F3
:10F95000E0600C490968884201D8012000E00020DD
:10F9600050B900BF502080F31188BFF34F8FBFF311
:10F970006F8F00BF00BFFEE770BD00003811002090
:10F980000CED00E03C110020024600200BE0084B8B
:10F9900053F8303033B9064B43F8301003EBC00353
:10F9A0005A6002E0401C0828F1D300BF70470000F5
:10F9B000202F002070B50446254655B900BF5020C1
:10F9C00080F31188BFF34F8FBFF36F8F00BF00BF6D
:10F9D000FEE7284600F008F895F8460010B92846DA
:10F9E000FFF768FE70BD0000014600200EE0094AE6
:10F9F00002EBC00252688A4207D10022054B43F84D
:10FA0000302003EBC0035A6002E0401C0828EED30C
:10FA100000BF7047202F00202DE9F04105460E461B
:10FA200017462C46FFF7FEFD94F94400401C10B920
:10FA3000002084F8440094F94500401C10B90020CF
:10FA400084F84500FFF718FEA06B28B93A46314606
:10FA500004F1240000F062F82046FFF72EFABDE81A
:10FA6000F081000070B504460025D4B1124800684A
:10FA700008B9012000E0002050B900BF502080F3F9
:10FA80001188BFF34F8FBFF36F8F00BF00BFFEE73A
:10FA900000F0AEF900212046FEF7DAFC01F0C8F9CB
:10FAA00005463DB94FF0805004490860BFF34F8FC1
:10FAB000BFF36F8F70BD0000EC10002004ED00E07C
:10FAC0000349096801600349096841607047000003
:10FAD000DC100020C8100020012001490860704798
:10FAE000D810002070B504460D4654B900BF502010
:10FAF00080F31188BFF34F8FBFF36F8F00BF00BF3C
:10FB0000FEE70548016818312046FFF765FD012131
:10FB10002846FEF79DFC70BDB410002070B5054668
:10FB20000E46144655B900BF502080F31188BFF32C
:10FB30004F8FBFF36F8F00BF00BFFEE7064801681D
:10FB400018312846FFF762FD0CB14FF0FF36214611
:10FB50003046FEF77DFC70BDB41000202DE9F04763
:10FB600006460F4634464FF00109002E55D0206D51
:10FB700050B900BF502080F31188BFF34F8FBFF3FF
:10FB80006F8F00BF00BFFEE7E06CB84201D23D4678
:10FB900000E0E56CE06AA8423FD0206D01283CD12E
:10FBA0001F480068844201D0012000E0002050B9C5
:10FBB00000BF502080F31188BFF34F8FBFF36F8FCA
:10FBC00000BF00BFFEE7D4F82C80E562A06900F01A
:10FBD000004010B9C5F13800A06108EB8801114A56
:10FBE00002EB81016069884201D1012000E0002020
:10FBF00098B1201DFFF7B3FC0B49E06A0968884201
:10FC000002D90949E06A0860E16A01EB8101054A0D
:10FC100002EB8100211DFFF7F9FCBDE8F087000031
:10FC2000B4100020602F0020CC10002010B586B04A
:10FC300000200590049003AA04A905A8FFF7A4FCDE
:10FC40000022DDE904101346CDE9002102901FA136
:10FC50002048039A00F0E0FE1F490860084600684B
:10FC600008B1012400E00024012C02D101F0B6F912
:10FC70000446012C17D100BF502080F31188BFF338
:10FC80004F8FBFF36F8F00BF4FF0FF3013490860F5
:10FC9000012013490860002012490860FBF7E8FAC8
:10FCA00000F02AF910E0601C08B1012000E00020FB
:10FCB00050B900BF502080F31188BFF34F8FBFF3BE
:10FCC0006F8F00BF00BFFEE706B010BD49444C4532
:10FCD0000000000039E80008E8100020E4100020CF
:10FCE000D0100020C81000200D49096801440D4AB9
:10FCF0001268914201D8012100E0002151B900BFF2
:10FD0000502181F31188BFF34F8FBFF36F8F00BF76
:10FD100000BFFEE7024909680144014A11607047CB
:10FD2000C8100020E410002070B50546FFF77AFCEB
:10FD300015B92948006800E028460446201DFFF751
:10FD40000EFCA06A18B104F11800FFF708FC211D91
:10FD50002248FFF75BFC94F85C00012802D10020E8
:10FD600084F85C00FFF788FC1D48006828B1FFF7A5
:10FD700059FCFEF7F5FFFFF77FFC17480068844247
:10FD800029D117480068D0B11648006808B9012089
:10FD900000E0002050B900BF502080F31188BFF36D
:10FDA0004F8FBFF36F8F00BF00BFFEE74FF0805053
:10FDB0000D490860BFF34F8FBFF36F8F0BE007480B
:10FDC00000680A490968884203D100200249086096
:10FDD00001E000F015F870BDB410002010340020D0
:10FDE000D0100020EC10002004ED00E0C410002032
:10FDF00002480068401C014908607047EC10002070
:10FE000010B52B48006818B101202A4908604EE05F
:10FE1000002028490860FBF7D5FC27490860084600
:10FE200000682649096888420BD92549096801F10B
:10FE30005400496D204A1268204B1B68D21A1144A5
:10FE400001601D4800681D4908601E4801680CE0FB
:10FE500051B900BF502080F31188BFF34F8FBFF31B
:10FE60006F8F00BF00BFFEE7491E01EB8100164AFD
:10FE700052F8200008B9012000E000200028E7D156
:10FE800001EB8102104B03EB820042685268426032
:10FE900000F108024368934202D14268526842600E
:10FEA0004268D268064B1A600648016000BF10BD68
:10FEB000EC100020D8100020F4100020F0100020DA
:10FEC000B4100020CC100020602F002070B5044634
:10FED0000D4601212046F6F724F908B1002070BD37
:10FEE0004FF4007229462046F6F7E4F908B10020E5
:10FEF000F5E70120F3E700001CB538490846007813
:10FF00000190FF200A4610700846007800909DF886
:10FF1000000000F0F0009DF80020904201D1012087
:10FF200000E0002050B900BF502080F31188BFF3DB
:10FF30004F8FBFF36F8F00BF00BFFEE79DF800003B
:10FF400000F05000264A10700720264A106009E091
:10FF500024480068401E234A10609DF800004006B7
:10FF6000000E00909DF8000000F080008028EFD087
:10FF70001C480068C0F10700042801D1012000E0FE
:10FF8000002050B900BF502080F31188BFF34F8F7D
:10FF9000BFF36F8F00BF00BFFEE71248006800028A
:10FFA000104A10601046008800F4E06010600B4AB0
:10FFB000019810700C48006840F470000A4908600D
:10FFC0000846006840F070400860FFF7BDFB002065
:10FFD00006490860F2F7C8FC00201CBD00E400E000
:10FFE000381100203C11002020ED00E028110020F5
:10FFF00070B505460E460DB1012000E0002050B955
:020000040801F1
:1000000000BF502080F31188BFF34F8FBFF36F8F75
:1000100000BF00BFFEE7AE4201D8012000E0002093
:1000200050B900BF502080F31188BFF34F8FBFF34A
:100030006F8F00BF00BFFEE702220021284600F0BC
:100040005DF8044604B1A663204670BDF8B50546C8
:100050000E4617460DB1012000E0002050B900BF48
:10006000502080F31188BFF34F8FBFF36F8F00BF15
:1000700000BFFEE7AE4201D8012000E0002050B9E9
:1000800000BF502080F31188BFF34F8FBFF36F8FF5
:1000900000BF00BFFEE702203B4600221146009051
:1000A000284600F05AF8044604B1A6632046F8BD7D
:1000B0002DE9F041044601260027224600210120B7
:1000C00000F01CF805462846FEF7F4FB2846BDE87C
:1000D000F0812DE9F84304460D4601274FF0000852
:1000E0002B46002211460120009400F036F8064607
:1000F0003046FEF7DFFB3046BDE8F8832DE9F843D4
:1001000005460E4690460DB1012000E0002050B992
:1001100000BF502080F31188BFF34F8FBFF36F8F64
:1001200000BF00BFFEE70EB9002701E005FB06F7A0
:1001300007F15000FEF700FF04465CB104F15009DE
:10014000002084F8460043464A463146284600943B
:10015000FEF7BEFB2046BDE8F8832DE9F843804654
:100160000E4617461D46DDF82090B8F1000F01D06D
:10017000012000E0002050B900BF502080F311881A
:10018000BFF34F8FBFF36F8F00BF00BFFEE70DB10E
:10019000012000E0002050B900BF502080F31188FA
:1001A000BFF34F8FBFF36F8F00BF00BFFEE707B1F4
:1001B0000EB1012000E0002050B900BF502080F3B4
:1001C0001188BFF34F8FBFF36F8F00BF00BFFEE7F3
:1001D00007B90EB9012000E0002050B900BF50203F
:1001E00080F31188BFF34F8FBFF36F8F00BF00BF45
:1001F000FEE7502000900098502801D1012000E037
:10020000002050B900BF502080F31188BFF34F8FFA
:10021000BFF36F8F00BF00BFFEE72C464CB101203B
:1002200084F846004B463A46314640460094FEF775
:100230004FFB2046BDE8F88370B505460E462C46B8
:1002400054B900BF502080F31188BFF34F8FBFF324
:100250006F8F00BF00BFFEE7FFF7E4F9D4E90F128C
:10026000206801FB020060600020A0632068A0609D
:10027000E06B401E226C216800FB0210E060FF2052
:1002800084F8440084F845009EB9206908B901202B
:1002900000E00020A8B904F1100000F07BFD80B15F
:1002A0004FF0805009490860BFF34F8FBFF36F8F45
:1002B00007E004F11000FFF77FF904F12400FFF7D5
:1002C0007BF9FFF7D9F9012070BD000004ED00E0D3
:1002D0002DE9FF4383B0064688461D464FF00009CE
:1002E000344654B900BF502080F31188BFF34F8FBC
:1002F000BFF36F8F00BF00BFFEE7B8F1000F01D161
:10030000206C08B9012000E0002050B900BF502047
:1003100080F31188BFF34F8FBFF36F8F00BF00BF13
:10032000FEE7022D02D1E06B012801D1012000E09F
:10033000002050B900BF502080F31188BFF34F8FC9
:10034000BFF36F8F00BF00BFFEE700F0C7FB08B927
:10035000059808B9012000E0002050B900BF5020E6
:1003600080F31188BFF34F8FBFF36F8F00BF00BFC3
:10037000FEE700BFFFF756F9A06BE16B884201D39F
:10038000022D28D12A4641462046FEF76EF907463F
:10039000606A08B9012000E0002068B904F1240077
:1003A00000F0F8FC88B14FF0805032490860BFF38C
:1003B0004F8FBFF36F8F08E03FB14FF080502D4952
:1003C0000860BFF34F8FBFF36F8FFFF755F9012020
:1003D00007B0BDE8F083059818B9FFF74DF9002084
:1003E000F6E7B9F1000F04D101A8FFF769FB4FF060
:1003F0000109FFF741F9FFF7FBFCFFF713F994F947
:100400004400401C10B9002084F8440094F94500D1
:10041000401C10B9002084F84500FFF72DF905A90C
:1004200001A800F081FAF0B92046FEF78AFBA0B1DE
:1004300004F110000599FFF755FB2046FEF73DFD3E
:1004400000F0F6FC002895D14FF080500949086073
:10045000BFF34F8FBFF36F8F8CE72046FEF72DFD64
:1004600000F0E6FC86E72046FEF727FD00F0E0FC02
:100470000020ADE704ED00E02DE9F05F07468A4675
:1004800090461E463C4654B900BF502080F3118868
:10049000BFF34F8FBFF36F8F00BF00BFFEE7BAF10E
:1004A000000F01D1206C08B9012000E0002050B9F4
:1004B00000BF502080F31188BFF34F8FBFF36F8FC1
:1004C00000BF00BFFEE7022E02D1E06B012801D180
:1004D000012000E0002050B900BF502080F31188B7
:1004E000BFF34F8FBFF36F8F00BF00BFFEE7FFF773
:1004F0000FFA00BF5021EFF3118081F31188BFF391
:100500004F8FBFF36F8F00BF0546A06BE16B884232
:1005100001D3022E23D194F945B0324651462046EC
:10052000FEF7A3F80BF1010088B9606A08B9012051
:1005300000E0002080B904F1240000F02BFC58B149
:10054000B8F1000F08D00120C8F8000004E00BF15A
:10055000010040B284F845004FF0010901E04FF07E
:10056000000900BF85F3118800BF4846BDE8F09F31
:1005700070B505462C4654B900BF502080F3118851
:10058000BFF34F8FBFF36F8F00BF00BFFEE700F0D8
:100590009FFA616888420CD1E068401EE060E06824
:1005A00028B900231A4619462046FFF791FE012676
:1005B00000E00026304670BD2DE9F74183B00546C6
:1005C0000E464FF000082C4654B900BF502080F36F
:1005D0001188BFF34F8FBFF36F8F00BF00BFFEE7DF
:1005E0000EB9206C08B9012000E0002050B900BF0E
:1005F000502080F31188BFF34F8FBFF36F8F00BF80
:1006000000BFFEE700F06AFA08B9059808B90120B2
:1006100000E0002050B900BF502080F31188BFF3E4
:100620004F8FBFF36F8F00BF00BFFEE700BFFEF725
:10063000F9FFA76BF7B131462046FEF701F8781EA7
:10064000A063206908B9012000E0002060B904F12E
:10065000100000F09FFB38B14FF080502F49086028
:10066000BFF34F8FBFF36F8FFFF706F8012006B07F
:10067000BDE8F081059818B9FEF7FEFF0020F6E707
:10068000B8F1000F04D101A8FFF71AFA4FF00108E2
:10069000FEF7F2FFFFF7ACFBFEF7C4FF94F944004E
:1006A000401C10B9002084F8440094F94500401C17
:1006B00010B9002084F84500FEF7DEFF05A901A867
:1006C00000F032F9F0B92046FEF72EFAA0B104F19D
:1006D00024000599FFF706FA2046FEF7EEFB00F02E
:1006E000A7FB0028A3D14FF080500C490860BFF34E
:1006F0004F8FBFF36F8F9AE72046FEF7DEFB00F0C7
:1007000097FB94E72046FEF7D8FB00F091FB2046CC
:10071000FEF70AFA00288AD00020A8E704ED00E0DE
:100720002DE9F34182B005464FF000082C46002623
:1007300054B900BF502080F31188BFF34F8FBFF32F
:100740006F8F00BF00BFFEE7206C08B9012000E0FA
:10075000002050B900BF502080F31188BFF34F8FA5
:10076000BFF36F8F00BF00BFFEE700F0B7F908B915
:10077000039808B9012000E0002050B900BF5020C4
:1007800080F31188BFF34F8FBFF36F8F00BF00BF9F
:10079000FEE700BFFEF746FFA76BFFB1781EA06320
:1007A000206810B9FEF766FC6060206908B9012076
:1007B00000E0002060B904F1100000F0EBFA38B15D
:1007C0004FF0805043490860BFF34F8FBFF36F8FE6
:1007D000FEF752FF012004B0BDE8F081039898B9FC
:1007E0000EB9012000E0002050B900BF502080F376
:1007F0001188BFF34F8FBFF36F8F00BF00BFFEE7BD
:10080000FEF73AFF0020E6E7B8F1000F04D1684692
:10081000FFF756F94FF00108FEF72EFFFFF7E8FA51
:10082000FEF700FF94F94400401C10B9002084F842
:10083000440094F94500401C10B9002084F845009C
:10084000FEF71AFF03A9684600F06EF840BB204689
:10085000FEF76AF9F0B1206838B9FEF7E3FE606888
:1008600000F046FA0646FEF707FF04F1240003995C
:10087000FFF738F92046FEF720FB00F0D9FA0028F0
:1008800088D14FF0805013490860BFF34F8FBFF3FA
:100890006F8F7FE72046FEF710FB00F0C9FA79E77B
:1008A0002046FEF70AFB00F0C3FA2046FEF73CF9AB
:1008B0000028EED05EB1FEF7B5FE2046FDF73BFF07
:1008C000074639466068FFF749F9FEF7D5FE002074
:1008D00081E7000004ED00E02DE9F04106460F46F7
:1008E000344654B900BF502080F31188BFF34F8FB6
:1008F000BFF36F8F00BF00BFFEE700F0E9F861684B
:10090000884204D1E068401CE060012508E03946D7
:100910002046FFF705FF054615B1E068401CE06082
:100920002846BDE8F081000070B505460C4655B973
:1009300000BF502080F31188BFF34F8FBFF36F8F3C
:1009400000BF00BFFEE754B900BF502080F31188FC
:10095000BFF34F8FBFF36F8F00BF00BFFEE7FEF7FF
:1009600061FE124802686868131A2068401C08B9C2
:10097000002617E00E4928680968884204D0686894
:10098000904201D801260DE02068984207D92068DE
:10099000C01A20602846FFF793F8002602E00020E6
:1009A00020600126FEF768FE304670BDC8100020AA
:1009B000DC1000202DE9FF4F85B0804689461746A0
:1009C000DDE912ABB800FEF7B7FA064656B1602073
:1009D000FEF7B2FA04460CB1266304E03046FEF797
:1009E00069FE00E000248CB1002084F85D00CDE9B0
:1009F00000ABCDE902403A4649464046089BFDF728
:100A00007CFF2046FDF762FD012501E04FF0FF3538
:100A1000284609B0BDE8F08F2DE9F04F85B00746B4
:100A2000884691469A46DDE90EB6109C0EB101202B
:100A300000E0002050B900BF502080F31188BFF3C0
:100A40004F8FBFF36F8F00BF00BFFEE70CB10120D7
:100A500000E0002050B900BF502080F31188BFF3A0
:100A60004F8FBFF36F8F00BF00BFFEE76020039082
:100A70000398602801D1012000E0002050B900BF98
:100A8000502080F31188BFF34F8FBFF36F8F00BFEB
:100A900000BFFEE7B4B1AEB125462C462E6302205E
:100AA00085F85D00002004A953464A46CDE900B10F
:100AB000CDE9025041463846FDF71FFF2846FDF7B5
:100AC00005FD01E000200490049805B0BDE8F08F1A
:100AD0000149086870470000B41000200549096802
:100AE00009B9012005E00449096809B9022000E0BC
:100AF00000207047D0100020EC1000200149086849
:100B000070470000C81000202DE9F0414FF00008A8
:100B100043480068002876D142480068451C414897
:100B2000056015BB40480068006808B9012000E076
:100B3000002050B900BF502080F31188BFF34F8FC1
:100B4000BFF36F8F00BF00BFFEE737480768374825
:100B50000068354908603548076035480068401C22
:100B600033490860FEF7FCF800BF32480068854250
:100B70003BD300BF2C480068006808B9012000E0A2
:100B8000002020B14FF0FF302A4908602CE02648B1
:100B90000068C068C4686668B54202D2254806602D
:100BA00022E0201DFEF7DBFCA06A18B104F118005A
:100BB000FEF7D5FC2049E06A0968884202D91E493F
:100BC000E06A0860E16A01EB81011C4A02EB8100E6
:100BD000211DFEF71BFD1A49E06A0968C96A8842AF
:100BE000C8D34FF00108C5E700BF15480068C06AC8
:100BF00000EB8000114951F82000012801D94FF085
:100C0000010805E0FFE70F480068401C0D49086037
:100C10000D48006808B14FF001084046BDE8F0817A
:100C2000EC100020C8100020B8100020BC100020DC
:100C3000DC100020E4100020CC100020602F0020E9
:100C4000B4100020D4100020D810002070B5054644
:100C50002C460026002D43D022480068844201D152
:100C6000012000E0002050B900BF502080F311881F
:100C7000BFF34F8FBFF36F8F00BF00BFFEE7206D44
:100C800050B900BF502080F31188BFF34F8FBFF3DE
:100C90006F8F00BF00BFFEE7206D401E2065E16C36
:100CA000E06A88421CD0206DD0B9201DFEF757FCA9
:100CB000E06CE062E06AC0F13800A0610A49E06AD5
:100CC0000968884202D90849E06A0860E16A01EBD4
:100CD0008101064A02EB8100211DFEF797FC0126E7
:100CE000304670BDB4100020CC100020602F0020D2
:100CF00070B505462C460026002D42D02249E06AF8
:100D00000968C96A884235D2A06900F0004028B954
:100D10001D480068C06AC0F13800A061E16A01EBBB
:100D200081011A4A02EB81016069884201D10120E8
:100D300000E00020C0B1201DFEF711FC1248006841
:100D4000C06AE0621249E06A0968884202D9104923
:100D5000E06A0860E16A01EB81010C4A02EB810064
:100D6000211DFEF753FC03E007480068C06AE062FB
:100D7000012606E00449E06C0968C96A884200D28D
:100D80000126304670BD0000B4100020602F002006
:100D9000CC10002070B50646F068C46854B900BF96
:100DA000502080F31188BFF34F8FBFF36F8F00BFC8
:100DB00000BFFEE704F11800FEF7D1FB16480068FB
:100DC000A0B9201DFEF7CBFB1449E06A09688842F0
:100DD00002D91249E06A0860E16A01EB8101104A18
:100DE00002EB8100211DFEF711FC04E004F1180163
:100DF0000C48FEF70BFC0C49E06A0968C96A884296
:100E000004D9012501200949086000E00025FDF70B
:100E1000A7FF284670BD0000EC100020CC10002079
:100E2000602F0020E8330020B4100020D8100020EC
:100E300070B5002400263648006850B900BF502025
:100E400080F31188BFF34F8FBFF36F8F00BF00BFD8
:100E5000FEE7FEF7E7FB2E480068401E2C490860BD
:100E60000846006800284ED12A48006800284AD069
:100E700023E02948C068C46804F11800FEF76FFB3E
:100E8000201DFEF76CFB2549E06A0968884202D9FB
:100E90002249E06A0860E16A01EB8101204A02EB25
:100EA0008100211DFEF7B2FB1E49E06A0968C96A8C
:100EB000884202D301201C4908601748006808B91D
:100EC000012000E000200028D3D00CB1FDF748FF3E
:100ED0001648056865B100BFFFF716FE10B1012086
:100EE000114908606D1E002DF6D100200F490860E1
:100EF0000D48006838B1012630070D490860BFF37E
:100F00004F8FBFF36F8FFEF7B7FB304670BD000009
:100F1000EC100020C4100020E8330020CC1000208A
:100F2000602F0020B4100020D8100020D410002022
:100F300004ED00E02DE9FC4705460E4617469846AD
:100F4000DDF828903020FDF7F7FF044654B1434602
:100F50003A4631462846CDE90094FDF729FD0020A8
:100F600084F82C002046BDE8FC872DE9FC470646A6
:100F70000F4690469946DDE90AA530200190019878
:100F8000302801D1012000E0002050B900BF5020DE
:100F900080F31188BFF34F8FBFF36F8F00BF00BF87
:100FA000FEE755B900BF502080F31188BFF34F8F83
:100FB000BFF36F8F00BF00BFFEE72C4654B14B4616
:100FC000424639463046CDE900A4FDF7F1FC012048
:100FD00084F82C002046BDE8FC87000010B586B0E0
:100FE0000024FDF7CFFA16480068D0B10020059024
:100FF000049003AA04A905A8FEF7D2FA0222DDE9AB
:1010000004100023CDE9002102900EA10F48039A9D
:10101000FFF702FD0E4908600846006800B1012490
:1010200000BF54B900BF502080F31188BFF34F8F29
:10103000BFF36F8F00BF00BFFEE7204606B010BDB4
:1010400000110020546D722053766300A1EE000859
:10105000041100202DE9FF4704460D4616461F46A1
:10106000DDF830804FF0000954B900BF502080F304
:101070001188BFF34F8FBFF36F8F00BF00BFFEE734
:101080001448006810B3009501960294062D15DAF5
:10109000FFF724FD022808D10023424669460D4887
:1010A0000068FFF715F9814610E000231A466946EB
:1010B00008480068FFF70CF9814607E000233A462C
:1010C000694604480068FFF7D7F98146484604B0EE
:1010D000BDE8F087001100200000C0E0F0F8FC003F
:1010E000681501080000000000000000000000007A
:1010F00000000000000200001800000000000000D6
:10110000000000003415010800000000000000008D
:1011100000000000000000000004000010000000BB
:10112000000000000000000074150108000000002D
:1011300000000000000000000000000000040000AB
:101140001100000000000000000000001015010860
:10115000000000000000000000000000541501081D
:10116000000000000000000000000000441501081D
:1011700000000000000000000000000084150108CD
:101180000000000000000000000000002815010819
:101190000000000000000000000000001815010819
:1011A0000000000000000000000000000203040531
:1011B000060708090A0B0C0D0E0F101001020000A3
:1011C00000000000000001020304060708090000F7
:1011D000000001020304000075191A0C6A231B1C8D
:1011E0001F207274433B4138393A6B6C376F0624C9
:1011F0006D6E70006800000476005401F7FD000178
:101200008300000000080000000100183200050003
:10121000000020410000D242295C0F3E9A99993E7D
:101220003333733F295C0F3E555555555555C53FD2
:101230007D6FEB0312D6D4BF5544880E55C1C93F0C
:101240003B8F68B52882A4BF88B20175E0EF493FA3
:1012500009F7FD0DE13D023F4B2D8A1C273A03C0E3
:10126000C88A599CE52A004059018D1B6C06E6BFCF
:1012700082922EB1C5B8B33F000000000000F03FDD
:10128000000000000000F83F000000000000000027
:101290000000004003B8E23F000000000000000032
:1012A00006D0CF43EBFD4C3E033333333333E33FC0
:1012B000FFAB6FDBB66DDB3F4D268F515555D53FEC
:1012C00001411DA96074D13F65DBC9934A86CD3FBA
:1012D000EF4E454A287ECA3F3E5555555555C53FA8
:1012E00093BDBE166CC166BF2CDE25AF6A56113F9A
:1012F000F16BD2C541BDBBBED0A4BE726937663E9C
:101300000040404040404040404041414141414018
:1013100040404040404040404040404040404040CD
:10132000400502020202020202020202020202025C
:101330000220202020202020202020020202020261
:1013400002029090909090901010101010101010B9
:1013500010101010101010101010101002020202C5
:101360000202888888888888080808080808080809
:101370000808080808080808080808080202020205
:1013800040000000011301084FBB610567ACDD3F61
:10139000182D4454FB21E93F9BF681D20B73EF3F9C
:1013A000182D4454FB21F93FE2652F227F2B7A3C14
:1013B000075C143326A6813CBDCBF07A8807703CCD
:1013C000075C143326A6913CC4EB98999999C9BF40
:1013D000711623FEC671BCBF6D9A74AFF2B0B3BF75
:1013E0009AFDDE522DDEADBF2F6C6A2C44B4A2BF35
:1013F0000D5555555555D53FFF8300922449C23FA1
:101400006E204CC5CD45B73F513DD0A0660DB13FD4
:10141000EB0D76244B7BA93F11DA22E33AAD903FE6
:1014200000000000000000004661696C65642074E3
:101430006F20636F6E6669677572652074686520DA
:101440006F75747075742074797065206F66204EA6
:101450004D45412073656E74656E63657320746FCE
:1014600020616C6C20666F726D6174730D0A0000F0
:101470004661696C656420746F20636F6E6669678E
:101480007572652074686520737570706F7274650D
:101490006420474E535320736174656C6C697465A6
:1014A000206E617669676174696F6E2073797374F9
:1014B000656D7320746F204750532B426569446FEC
:1014C000750D0A00436F6E6669677572696E6720F5
:1014D00074686520737570706F7274656420474E10
:1014E000535320736174656C6C697465206E61760A
:1014F00069676174696F6E2073797374656D7320A9
:10150000746F204750532B426569446F750D0A0074
:1015100054696D65325F0000636F756E745F73654B
:101520006D70686F72655F0073656D70686F72656E
:101530005F00000065633830305F6461746155702E
:101540006C6F61006D757465785F65633830304429
:10155000617465006D757465785F727334383552E7
:10156000656344617465000064656661756C7454FC
:1015700061736B00636F6D6D756E69636174696F24
:101580006E000000735F6D6573736167654461741D
:10159000655F6C6F636174696F6E0000BC15010854
:1015A0000010002034020000F63A00085816010826
:1015B000341200204C720000F49A0008811365BABE
:1015C0001408E9B6800E0833392E39382E33372EF9
:1015D0003138300710C17E4E554C4CE76865636862
:1015E000756E00095261646D696E3132333210429A
:1015F00001037524F41AAA0101141ED8110108F47C
:101600000401212C120108C06904510B130C043889
:10161000C80A63647A75706461746514B7323032D5
:1016200031215A801101015A33392E39382E323185
:10163000312E32343412151A2F3E1B612F34A94239
:1016400000111A656E7472616C4374725379732E53
:0816500062696E0A1410988112
:040000050800293195
:00000001FF
